:0A0000000C94380C0C9400000C94D2
:10000A0000000C9400000C9400000C9400000C9466
:10001A0000000C94FD5C0C9400000C9400000C94FD
:10002A0027140C9400000C9400000C9400000C940B
:10003A0000000C9400000C94D9130C9400000C944A
:10004A00A2590C9400000C94DE590C9400000C94F4
:10005A0000000C9400000C9400000C9400000C9416
:10006A0000000C9400000C9400000C9400000C9406
:10007A00575B0C9400000C949B5C0C9400000C944D
:10008A0000006B65696E204B72656469740054697F
:10009A006D656F757400504C55200000000001001A
:1000AA000200040008001000200040008000000147
:1000BA000002000400080010002000400080000137
:1000CA0002040810204080002404C10B80100000A4
:1000DA002804C10B821F00003204C10B81030000F7
:1000EA003A04C10B010403004404C20B01060500D3
:1000FA004E04C40B018000005A04CB0B020F00000F
:10010A006204C50B020F00006A04C70B020FD0126B
:10011A007204C90B011000007C04190C01100000C4
:10012A008604CA0B000100008E04CD0B01080100F1
:10013A009804CE0B03080100A604CF0B03070000A6
:10014A00AE04E50B017F3F00B804E40B0106000092
:10015A00C204D00B03040000CA04E30B01641E00AE
:10016A00D604D10B00010000E204D20B000100000A
:10017A00EE04E20B01020000FA04D30B00010000B6
:10018A000805D40B020F00001405D60B020FE70373
:10019A001E05180C016300007C051A0C01100000F2
:1001AA0086051B0C010202002A05D80B0308010070
:1001BA003005D90B030800003605DA0B03080000E6
:1001CA003C05DB0B030800004205DC0B03080000BA
:1001DA004805DD0B030800004E05DE0B030800008E
:1001EA005405E60B040A2E005C05F00B040A2E00E7
:1001FA006405FA0B040A2E006C05040C040A2E008E
:10020A0074050E0C040A2E0000000000FF00000016
:10021A00537061727465202000008E0500029605F5
:10022A0004049C050807A2050C05A2058C06A8056E
:10023A008009B005100BB805500CC2054003CA0569
:10024A00140AD4051808DC051C01000000025465D4
:10025A0073740000546F74616C2000006A610000BE
:10026A006E65696E0000580043616C696272617460
:10027A00696F6E004F4B00004B653A00496E3A00B9
:10028A0054696E79200062616400454550524F4DB1
:10029A002000446174612000496E6974000053743F
:1002AA006F700000567320312E353700310B312024
:1002BA0041424300320B322044454600330B33207F
:1002CA00474849004D0A4D0000000000340B342015
:1002DA004A4B4C00350B35204D4E4F00360B36201D
:1002EA00505152002B0A2B0000000000370B372018
:1002FA0053545500380B382056575800390B3920BB
:10030A00595A2F002D0A2D0000000000430C43000B
:10031A0000000000300B3020202E2C002C0A2C006C
:10032A00000000003D0A435200000000210C580062
:10033A002D0B2D002B0B2B004D0A4D0028006000C1
:10034A009800D00008014001808182838400002146
:10035A0088898A8B8C8D8E8F00004A014600320074
:10036A002100004B004A01460032004D0000960071
:10037A004A0146003200540000E1004A01460032B8
:10038A00003D0000F0000000320050002D0000F097
:10039A0000500032005000470000F000A000320078
:1003AA0050004B0000F000F000320050002B00001B
:1003BA00B400040038003800217002008700C80029
:1003CA00640032003D6602000800C8006400320082
:1003DA00216A02004B004A01460032004D0000002B
:1003EA0001000100E60063004D0000000000A000CB
:1003FA001B00007105D700A0001A020071056900F0
:10040A000000180400730569001E0119060073052F
:10041A0050726F64756B742000005F4944005F522C
:10042A0073323332494400005F526F74617465005D
:10043A005F54617374656E5800005F54617374652C
:10044A006E5900005F44656661756C744B6579008E
:10045A002A436F64653000002A436F6465310000E7
:10046A002A436F64653200002A4D61784D6F6475C6
:10047A006C005F4572774D6F64756C002A5469731E
:10048A00636845005F4D795465726D4E72005F4D29
:10049A0061737465725465726D7300005F454D6FC8
:1004AA00646500005F4543726564577472005F5269
:1004BA0073304D6F646500005F5634756E643500A5
:1004CA005F50756C736554696D6500005F41736BAD
:1004DA0043726564697400005F53656E64446562C3
:1004EA00697400005F4372656469744D6F646500E6
:1004FA005F4372656469744D6173746572002A544E
:10050A0061626C655374617274002A5461626C652D
:10051A00456E64002A4669727374426F6E50000019
:10052A002A4A6F6231002A4A6F6232002A4A6F628F
:10053A0033002A4A6F6234002A4A6F6235002A4A17
:10054A006F6236002A4A6F6237005F4572726F72B5
:10055A0031005F4572726F7232005F4572726F725C
:10056A0033005F4572726F7234005F4572726F7248
:10057A0035005F4672656967616265005F4B6F6D42
:10058A006D61000054617374657200004C69745A9D
:10059A0000004C656974540050756C730000546116
:1005AA0073742030000073657269656C6C00736542
:1005BA007269656C20320000546173742032000045
:1005CA0054617374207061720000466F6C676554E1
:1005DA0000005377697463680000706F7274696F02
:1005EA006E696572656E00002E666F6C6765000045
:1005FA00506F7274696F6E656E2073696368657295
:10060A006E0066616C73636865722054697363680F
:10061A002000206765737065727274005469736391
:10062A006820766F6E204B2000004665686C657204
:10063A00200056656E74696C20616B7469760000DF
:10064A00435349204E722000436F64652000546969
:10065A00736368200000436865662D4D656E7500FA
:10066A004B206C697374656E00004B206C6F657368
:10067A006368656E00004B20647275636B656E007B
:10068A0054206C697374656E000054206C6F657336
:10069A006368656E00005420647275636B656E0052
:1006AA0053797374656D0000506F7274696F6E00D0
:1006BA004B726564697465004B7265642E436C7293
:1006CA0000006D616E2E506F7274696F6E0050611A
:1006DA0072616D657465720050726F64756B7465D2
:1006EA0000004B656C6C6E65720056656E74696CC1
:1006FA0065004572726F72004F70742E0000496D6A
:10070A0070756C7300004162726563686E756E671E
:10071A0000004D6F64756C20000073656300496DBD
:10072A007000507231005072320046756E63740068
:10073A00547970003A20563A2020302B203000009D
:10074A003A20544F3A2000003A2050733A200000D1
:10075A0053703A00730049004B204D6F6465204A7C
:10076A006F62204A6F62466C616773004B2000001B
:10077A004D6F646520004A6F6220000056202020D9
:10078A004572722050676C20496D7020544F0000EA
:10079A0020563A005061757365002E202C30414274
:1007AA00433144454632474849334A4B4C344D4E0F
:1007BA004F35505152365354553756575838595A5F
:1007CA002F39306006316A06327406338006348A5D
:1007DA000635940636A00646AA0641B20643BA066C
:1007EA0044C2064ACC060000000030AA0637580266
:1007FA0039D80638E20642EC0645F4060000000045
:10080A00FC062F0C000500000207320C0003000052
:10081A000807300C000500009800310C0014000095
:10082A000500C11100000300D90B00000300C1112B
:10083A000300170E0300D90B00000500E0080000B2
:10084A000A00C1110A00170E0A00D90B0A00C111C9
:10085A000A00170E2800D90B00000000F80000005B
:10086A00FF000000FF0000007F80001E0F80007F55
:10087A00E7C0007FFFE0003FFFE00007FFC0000184
:10088A00FFC00001FF800001FF0003FFFE0007FF19
:10089A00FC0007FFF00003FFF00003FFFE00001F4B
:1008AA00FFC001FFFFF001FFFFF801FFFFF8007F23
:1008BA00FFF80007FE00003FFF00007FFF80007F77
:1008CA00FF80007FC100001FE000001FF000001F32
:1008DA00F000000FE0000007C0000007C00000079A
:1008EA00C0000007800000030000000300000002AF
:1008FA00000000000000000000000000E00000000E
:10090A0000000003900000000000000E1800000024
:10091A000000003808000000000000C018000000B5
:10092A00000003807000000000000C01C0000001FC
:10093A008006300700000003C00F401C00000006BC
:10094A00E01DC0700000000C3039C1C00000001862
:10095A001871C7180000001C0CE1DC7C0000000EB6
:10096A0007C3F1C40000000703860706000000035E
:10097A00800E1C0200000001C01C300300000000B1
:10098A00E03818010080000070700FC183C00000B9
:10099A0038E003E08E6006001DC00020FC200F0036
:1009AA000F8000307030198007000010003030C00E
:1009BA000000001800E0606000000008038060305A
:1009CA000000000C0E003018000000043800180C5B
:1009DA0000000006E0000C06000000038000060389
:1009EA0000000000000003018000000000000180F8
:1009FA00C000C0C060C030C030C030C030C030C0DD
:100A0A0030C030C030C030C030E030703018300CE8
:100A1A0030043FFC3FFC0000000000000000000022
:100A2A000000000000000000000000000000070CA9
:100A3A00182022204D994D401140489147202220EC
:100A4A0018C007000000070C1F3FEE3F7277727F45
:100A5A00FF7F777F783FEE3F1FC00700000000004E
:100A6A0000000C183DEE3F3FEE3F1FC80F07000283
:100A7A0000000000000000000000000207080F1F2D
:100A8A00CE3F1FC80F070002000000000000000050
:100A9A000007080F0F880F376F7F7FFF7F326007CD
:100AAA000F800000000000000002000207080F1F6C
:100ABA00CE3F3FEE3F1AC0070F8000000000000043
:100ACA000000000000000006000F0F0006000000F2
:100ADA00000000000000FFFFFFFFFFFFFFFFFFF91C
:100AEA00FFF0F0FFF9FFFFFFFFFFFFFFFFFF00002E
:100AFA00000000000600091088101088100900067E
:100B0A00000000000000FFFFFFFFFFFFF9FFF6EF04
:100B1A0077EFEF77EFF6FFF9FFFFFFFFFFFF000028
:100B2A0000000E01006A1E33286161886133001ECD
:100B3A00000000000000000000078C0C186618185E
:100B4A006C0C078003030C0F030003000000020073
:100B5A0003038C0302CC0202800202000E1E001E56
:100B6A000C00000000000C000E0B08090CC40E0B50
:100B7A004C0938C478784C3103CC0301800000005A
:100B8A00020202271FCC18306770306C181FC22768
:100B9A000200020000000000001000181C001E1FC6
:100BAA00081F1F001E1C0018100000000000000093
:100BBA00000088010388070F881F0F880703880130
:100BCA0000800000000000000207080F1FC0020298
:100BDA0000020200021FC80F0700020000000008FE
:100BEA001919881919881919881919881919800061
:100BFA00198819000000000E1F36CC6666CC6636CE
:100C0A00CC1E06CC0606CC0606CC06000000000860
:100C1A001F30C03030081F30CC301F8C0000CC3061
:100C2A001F8000000000000000000000000000001B
:100C3A000000000000000E1F1FEE1F00000002004F
:100C4A00070F8C1F0200020200020200021FC80FD7
:100C5A000700021FC00000000207080F1FC002029F
:100C6A00000202000202000202000200000000006C
:100C7A00020200020200020200020200021FC80F62
:100C8A000700020000000000000000000108010146
:100C9A00CE3F01C801010000000000000000000072
:100CAA000000000004000C1C0E3F1C000C04000095
:100CBA00000000000000000000000000000000002A
:100CCA000000400040400040400E7F00000000004D
:100CDA0000000000088C1838EF7F38EC18088000F4
:100CEA0000000000000000000000000000000207F1
:100CFA00080F1FCE3F7FF000000000000000000038
:100D0A0000000000000F7F3FEC1F0F800702000069
:100D1A0000000000000000000000000000000000C9
:100D2A0000000000000000000000000000000600B3
:100D3A00060F000F0F000F0F000606000600000046
:100D4A000600060000000000001988191988190019
:100D5A000000000000000000000000000000000683
:100D6A00060666063FFC0C0CC819198C7F33003343
:100D7A003300000000000600061F8C3F3600363F95
:100D8A008C1F06CC063FC81F0600060000000000A4
:100D9A0000001338387E3801C80307000E1C0E38CD
:100DAA0070EE600000000000070D881919801B0E04
:100DBA00001E3E063333C8313BC61E0000000E003B
:100DCA000E0E000606000C000000000000000000E5
:100DDA000000000000000380060E000C1C001C1C12
:100DEA00001C1C001C0C000E0608030000001C005E
:100DFA000607000303880303880303880303000725
:100E0A0006001C000000000000000C3636C81F0F48
:100E1A000C3F0F081F36CC3600000000000000000F
:100E2A0000000000060006060C3F3FC0060600064A
:100E3A0000000000000000000000000000000000A8
:100E4A00000000000000000E0E000E06000C00005C
:100E5A0000000000000000000C3F3FC0000000003E
:100E6A000000000000000000000000000000000078
:100E7A00000000000000000E0E000E00000000013D
:100E8A000000370000EC010380070E001C380070D8
:100E9A006000000000000F8E3F30676060FB6163F6
:100EAA0033666C33787036303FE80F000000030079
:100EBA00071F001F030003030003030003030003CB
:100ECA001FEE1F0000001FCE3F707360607E00019E
:100EDA00C80307000E1C00387FFF7F0000001FCEEA
:100EEA003F7073600037000FEC0F006300603770CB
:100EFA003FEC1F00000001CC0307CC0E1CCC38705D
:100F0A00CC607FFF7F00CC0000CC000000007FFF98
:100F1A007F600060600C7F3FE7000033006037703D
:100F2A003FEC1F00000003CC070E001C3800307F86
:100F3A00CE7F7073606037703FEC1F0000007FFF48
:100F4A007F00660000CC000188010300030600064A
:100F5A000C000C0000000F8C1F38E630306E381F72
:100F6A00CE3F7073606037703FEC1F0000001FCEE9
:100F7A003F7073606037703FFF1F006E0001C80347
:100F8A001F001E0000000000000000000E000E0EF0
:100F9A0000000000000E000E0E000000000000001D
:100FAA00000000000E000E0E00000000000E000EF1
:100FBA000E000606000C00CC010380070E001C3848
:100FCA0000381C000E07080301CC000000000000D6
:100FDA0000000000000E3F3FE000000E3F3FE0002F
:100FEA000000000000003000381C000E0708030152
:100FFA00CC010380070E001C3800300000001F8C53
:10100A003F70E66060EC01038007060006060000F8
:10101A000600060000001FCE3F306B676FBB6D6D88
:10102A00BB6D6DBE6F67C0703FCC0F00000006003D
:10103A00060F000F0F081919881930CC3F3FC660F8
:10104A006066600000007F087F61CC6060CC617FD1
:10105A008C7F60E660606E607FC87F0000000F8C46
:10106A001F38E630600060600060600060306E38F3
:10107A001FC80F0000007F087F61CC606066606057
:10108A00666060666060CC617F807F0000007FEEF2
:10109A007F6000606000607F887F60006060006041
:1010AA007FEE7F0000007FEE7F6000606000607F5F
:1010BA00887F6000606000606000600000000FCE02
:1010CA001F38603060006063EE63606660306638C7
:1010DA001FEE0F0000006066606066606066607FF9
:1010EA00EE7F6066606066606066600000001F8870
:1010FA001F0600060600060600060600060600068B
:10110A001F881F00000000660000660000660000DD
:10111A006600006660606C703FC81F000000606E69
:10112A006061C86367006E7C007C6E0067638C61D7
:10113A0060E660000000600060600060600060605F
:10114A0000606000606000607FEE7F000000606EFB
:10115A007070EE7979E66F6F6666666660606660E3
:10116A006066600000006066707066786C666C6627
:10117A00666663666361EE6060E6600000000F0801
:10118A001F39CC3060666060666060666030CC395A
:10119A001F800F0000007F8C7F60E66060666060E1
:1011AA00EC7F7F80606000606000600000000F08D4
:1011BA001F39CC3060666060666060666333CC3924
:1011CA001FE60F0000007F8C7F60E660606660604B
:1011DA00EC7F7F8067638C6160E6600000001F8C93
:1011EA003F70E6606000703F8C1F00E600606E7022
:1011FA003FC81F0000003FCC3F0600060600060657
:10120A0000060600060600060600060000006066E4
:10121A0060606660606660606660606660606C30D0
:10122A003FC81F000000606660606C3030CC301927
:10123A00881919800F0F000F06000600000060666B
:10124A006060666060666060666666666F79EE70AA
:10125A0070E66000000060666030CC3019800F06CE
:10126A0000060F081930CC30606660000000606626
:10127A006030CC301988190F000F060006060006E8
:10128A000600060000007FEE7F00CC000180030606
:10129A0000060C00183000307FEE7F0000001F8827
:1012AA001F18001818001818001818001818001825
:1012BA001F881F00000000004060007038001C0EEC
:1012CA000007038C0100E7000030000000001F88BF
:1012DA001F01880101880101880101880101880133
:1012EA001F881F0000000200070F8C1D38E770607E
:1012FA0030000000000000000000000000000000B4
:10130A0000000000000000000000000000000000D3
:10131A000000007FFF7F00000707000706000603A2
:10132A0000000000000000000000000000000000B3
:10133A0000000000000C1F3FE6001FEE3F606660E1
:10134A007FEE3F00000060006060006060086F7F11
:10135A00CE70606660606E607FC87F00000000002B
:10136A000000000000081F3FC67060006060067041
:10137A003FC81F00000000660000660000661F3FAD
:10138A00EE716066606066703FEE1F00000000004C
:10139A000000000000081F3FC6707FEC7F600070ED
:1013AA003FC81F00000007880F1C00181800187F8C
:1013BA00007F180018180018180018000000000014
:1013CA0000000000000E1F3FE670606E703FE61FCF
:1013DA00006E003FC83F60006060006060006F7F81
:1013EA008C7160CC6060CC6060CC60000000000052
:1013FA000006000600000E0E00060600060600069D
:10140A001F881F0000000000000188010008030374
:10141A0088010188010188010188191F800F3000A5
:10142A00303000303008313380373E003E370833E1
:10143A0031CC300000000E000E060006060006063B
:10144A0000060600060600061F881F0000000000AE
:10145A00000000000008597FCE7F666666666666F1
:10146A0066666600000000000000000000083F3FBA
:10147A00CE30306630306630306630000000000012
:10148A000000000000081F3FCE70606660606E704A
:10149A003FC81F00000000000000000000087F7F16
:1014AA00CE6060666070EC7F6F80606000600000F4
:1014BA0000000000000E1F3FE67060666070EE3F9D
:1014CA001F6600006600000000000000000C373FA5
:1014DA00E6383000303000303000300000000000C4
:1014EA000000000000003F7F80607F083F01880104
:1014FA007F803F00000000001818001818007F7F46
:10150A0000181800181800181F880F0000000000A3
:10151A0000000000000660606660606660606E70D1
:10152A003FE61F00000000000000000000066060A7
:10153A006C3030C81919800F0F0006000000000037
:10154A00000000000006666666666666666F6C3FA7
:10155A0039C810000000000000000000000C607193
:10156A00C83B1F000E1F083B71CC60000000000042
:10157A0000000000000C3030C81919800F0F000657
:10158A0006000C0C0018000000000000000C7F7F11
:10159A00800306000C1800307FCC7F00000003CCCB
:1015AA00070E000C0C000C1C00381C000C0C000C64
:1015BA000E0C0703C0000600060600060600060019
:1015CA0000060600060600060600060000003C00AB
:1015DA003E070003030003038C0103800303000397
:1015EA0007003E3C00000000001C6C3663800000CF
:1015FA0000000000000000000000000000000000E1
:10160A000000000006000F198C306066607FEE7FD4
:10161A0000000000000000001E0060077E0700F0C6
:10162A001EF060F77EF7FBDE1F00E007FF0700F8F9
:10163A001FF8E0FFFFFFEA0000EB2000EC0C00EDD2
:10164A00C400E84000E93800F10100F2100027A3C5
:10165A000040000041000042010043130044100012
:10166A004526004608004751004802004912004A30
:10167A0018004B19004C1400501900512F00522C1D
:10168A0000533E00543F00553F00562E0057770046
:10169A00580B005906005A07005B0D005C1D005DDF
:1016AA00CC001B1B001A0100242F00255700238D94
:1016BA00001836001901000100001F8800FD05000E
:1016CA001F8000FD05001F9000FD05001FD000FDD2
:1016DA000500170500360000283800FD2800283CC0
:1016EA0000160800FF0000000000000000000000D3
:1016FA00000000000000000000002564002B003EEE
:10170A003E0049443D00202047433D002020363416
:10171A006B002D2D2D2D00204C00533F0000583119
:10172A003939313030004D42005053004D31004FAD
:10173A0031005350004350004459006275737900D8
:10174A004D5000256400202000433F003A20004D00
:10175A0049004D42004D43004D50004D4C004F4E44
:10176A0000002530325800253034580025366400F0
:10177A002533642E25303264002535640025640043
:10178A002532640025336400444400004B230042A0
:10179A005300422100424600542300544F0049524C
:1017AA00004D5A0042510042520043530056530022
:1017BA00564300494C00426600004B230054230064
:1017CA00424500434500424100445300434200233E
:1017DA00502241534349492D492F4F222C22312E61
:1017EA003030222C323030382D30312D30313B0020
:1017FA0023482245636F222C22312E3030222C328C
:10180A003030382D30312D30313B0023532245639F
:10181A006F222C22312E3030222C323030382D30AB
:10182A00312D30313B00504F00504632333B50553A
:10183A00002564002B302B303B0025640025303214
:10184A0058002E3030004F4E00006D696B726F7475
:10185A006F756368000001002D4E414E00000100C3
:10186A00E20E60180000F894EE27ECBBF1E0F5BF39
:10187A00E5BFE0936C00F8E1F1BDE1BD8DE0A2E0C7
:10188A00BB27ED938A95E9F780E090E1A0E0B1E00B
:10189A00ED930197E9F7E8E6F8E1859195910097CC
:1018AA0061F0A591B59105901590BF01F0010590E1
:1018BA000D920197E1F7FB01F0CFEFEFEDBFE0E109
:1018CA00EEBFC0E0D3E00C949E150A9902C0E1E095
:1018DA000895E0E00895A0913D0CA13031F40E94F2
:1018EA005F6B0E9416630E94706B0895A0913D0C75
:1018FA00A13031F40E945F6B0E947A6B0E94706B78
:10190A000895E881E03011F01C9A01C01C9832C099
:10191A000E947E6B0E947E6B0E94836BEFE3F0E075
:10192A000E94886B08951A93A0910403A43081F44D
:10193A00E0910F04E093100410E0183048F4ABE093
:10194A001A9FF001EE59FC4F0E948E6B1F5FF5CF74
:10195A003FC0A0910403A43039F4E881E093100455
:10196A00E0E0E0930F0406C0E881E0930F04E0E0B2
:10197A00E0931004219608951A93A0910403A430C9
:10198A0019F110E0143000F50E94926B3196E4913F
:10199A00EA93DFDFE0E0E09310040E949B6BEBE048
:1019AA00F1E00E94A56B0E94A56BFA93EA930E944C
:1019BA00926BE491EA930E94926B32960E94AA6B10
:1019CA000E9410431F5FDECF0E94AD6B0E94B26B74
:1019DA00199108952A970E94CF7C30E010E000E028
:1019EA0047ED50E028E0E091190CE03019F020E1D1
:1019FA0049E650E0321710F00C94420D0E94B66B83
:101A0A00E130A0F10E94B66BE03870F0EEE00E947F
:101A1A00BC6BE4E0F7E1FA93EA930E94B66BEF70CD
:101A2A00EF5F0E94C46B09C0ECE0EA9392DFE0E743
:101A3A00F2E004900E82E0E0EF830E949B6BA02FFD
:101A4A00B0E0E7E3F0E00E94497AE40FF51F0E9454
:101A5A00A56BFA93EA93EDE2F0E0FA93EA930E9417
:101A6A00B66BEA930E947E6B0E94CE6B1F5F1430A6
:101A7A0011F410E00F5F3F5FBDCF0E94AD6B0E9473
:101A8A00A2480E94D67C619608950E94D46BECE02D
:101A9A00EA935FDFEAEBF3E00E948E6BEBE0EA93F6
:101AAA0058DF0E94D86B0E94DD6BEAEAF0E00E94E0
:101ABA00E26BE0913A0CF0913B0CE491EA93E091ED
:101ACA003A0CF0913B0C31960E94E96B0E9410434C
:101ADA0001E00E94EC6B0E94EF6B11F00F5FF9CFEF
:101AEA000E94FD6B031718F4E0E0E093C0050E9422
:101AFA00FD6B11E00E94046C0E94EF6B11F015302F
:101B0A0008F021C00E94D86B0E94076CE0E4F0E064
:101B1A000E94497A3496FA93EA93E2EEF0E00E9440
:101B2A00E26B0E94046C0E940A6CE491EA930E94A0
:101B3A00046C0E940A6C31960E94E96B0E94104361
:101B4A003F5F1F5FD7CF0E94B26B0E94D87C36C41A
:101B5A0027970E94CF7C22E354E0A0910403A4308B
:101B6A0011F426E453E010E0143010F00C94080E3F
:101B7A0000E0051710F00C94060EE12FEE0FEE0FA1
:101B8A00E00F3E2F0E94046C0E94166C3196E4917D
:101B9A000E94BC6B0E94046C0E94166C3296FA93E7
:101BAA00EA930E947568ED85E03039F4AF81A1327D
:101BBA0010F4E0E0EF83E0E0E887A02FBB27E22FF4
:101BCA00E85FF0E00E94497A3896FA93EA930E9415
:101BDA00076CEAE3F0E00E94497AE55BFF4F0E9456
:101BEA001B6C0E94A56BFA93EA930E94046C0E94F4
:101BFA00166CE491EA930E947E6B0E94CE6B0F5F93
:101C0A00B8CF1F5FB1CF0E94B26B0E94D67C2E96CE
:101C1A00089522970E94206CA13059F40E94256CE5
:101C2A00ABE2B1E00E94747A2E2F57E1E2ECF0E0C9
:101C3A0008C00E94256C0E94296C2E2F53E0E7EE03
:101C4A00F0E0EE83FF830E942E6CA0911908A13068
:101C5A0081F4E9ECF0E00E94456C0E944C6C0E9411
:101C6A00516CEBE2EA93E7E0F7E10E94AA6B0E946B
:101C7A001043E3E0F0E00E94456C0E94576C0E941A
:101C8A00516C0E945C6C0E94606C3F5FE091C10BDA
:101C9A00AFEE0E94537AF0E0EE83FF8311E0E09109
:101CAA00C20B1E17C0F500E0E091C10B0E1788F5B4
:101CBA000E94666C59F10E946D6CE09310040E94B8
:101CCA00EC6BAE81BF810E94497A33960E941B6CED
:101CDA000E94076C0E94497ADF010E94776C0E9479
:101CEA007A6CEA85FB853497FA93EA930E94516CE1
:101CFA000E945C6C0E94606C3A930E942A20EF3F1B
:101D0A0029F0ADE05A9FF0010E947F6C3F5F0F5FA0
:101D1A00CBCF1F5FC4CF0E94AD6B0E94B26BCAC00B
:101D2A0022970E94CF7CE2E5F7E0EE83FF8340E052
:101D3A00443190F4AE81BF8111960E94876C13964C
:101D4A00EFEFEC93AE81BF81EC93EE81FF81349685
:101D5A00EE83FF834F5FECCFE091C10BA0EF0E94AF
:101D6A00537A2E2F0E94256CA0E4B1E00E94747A67
:101D7A005E2F0E942E6C21FE23C00E948C6C0E9452
:101D8A008C6CEFEAF0E0FA93EA930E94916C0E945D
:101D9A005C6C0E94606C0E94976CE6EBF0E0FA9330
:101DAA00EA930E948C6C0E944C6C0E94916CEFE743
:101DBA00EA93E9E0F7E1FA93EA93E0E0F0E011C090
:101DCA000E948C6C0E948C6CE8EEF0E0FA93EA9325
:101DDA00E52F0E949E6CFA93EA930E945C6CEAE8F3
:101DEA00FBE0FA93EA930E9410433F5F11E0E0910F
:101DFA00C20B1E1710F00C94590F00E0E091C10BB2
:101E0A000E1710F00C94570F0E94666C11F40C9484
:101E1A00540FA0919A0BE0E8EA23E03821F0A09150
:101E2A00E20BA23019F40E946D6C0AC00E94A16CE8
:101E3A00E03011F4E0E001C0E8E0E0930F04E7E0ED
:101E4A00E0931004A02FBB27E22FF0E00E94497A0A
:101E5A003396FA93EA930E94776C0E94076C0E9469
:101E6A00497A3396FA93EA930E94516C0E94916CD4
:101E7A000E945C6C0E94606C4E2FA0911E08E32F9A
:101E8A000E94A66CEA0FFB1F43833A930E942A2002
:101E9A00EF3F29F0ADE04A9FF0010E947F6C3F5F5F
:101EAA000F5FACCF1F5FA3CF0E94AD6B0E94B26BD6
:101EBA000E9421350E94D67C28960895E1E0E0939D
:101ECA000D04E2E0E0930E04E0E0E0931004ECE09D
:101EDA00E0930F04E2EDF3E00E948E6BEAE0E093F8
:101EEA000F04E6ECF3E00E948E6B0E94A24808956C
:101EFA001A93A981A43029F4A0E021FCA1E0A03022
:101F0A0009F426C0E9810E94AD6C0490E9810E941F
:101F1A00B36CE491A02DAE1BA2501A2F0E94976CAD
:101F2A00E4EBF0E0FA93EA93EB810E94B36C0E942F
:101F3A00FC7A3296FA93EA93EAE3F0E00E94BB6CE9
:101F4A00EFE7EA93E9E0F7E10E94AA6B0E941043E7
:101F5A001881229608951A930A930E94C26C0E94CD
:101F6A0017180E94A16C0E2FE6E4F3E00E94FC7A97
:101F7A0033971E2F0E947E6B0E947E6B0E94836B9A
:101F8A000E94C76C0A930E94D064ECE3F0E00E94BE
:101F9A00CC6C0E940D46E2E0E0930E04E091980BAF
:101FAA00EF70E09310040E94D36CEFE0E09310040A
:101FBA00AA81A13051F40E94DB6C0E94DD6B0E9461
:101FCA00F245ECE8F0E00E94E06C21FE0DC0E4E08E
:101FDA00EA938EDFEEE4F3E00E94E46CE0E5F3E0DE
:101FEA000E94E46C0E94BC489EDC82C0E8810E9488
:101FFA00B36C0E94E46CEA810E94AD6C0E94E46CAE
:10200A000E944946E881EA9373DFC6C11A930A938C
:10201A00EC81EA93EBDF1AEEEC810E94AD6C04903E
:10202A00EC810E94B36CE491A02DAE1BA2500A2F42
:10203A00AC81A43029F4A0E021FCA1E0A03009F48D
:10204A0009C01EEAAA81BB811B96E0E0EC93EC81F1
:10205A00EA934EDF0E946D6CE0931004EC810E94BB
:10206A00E96CFF93EF930E948C6CEE810E94B36C33
:10207A000E94FC7A31960E94BB6C0E94EC6BFA9328
:10208A00EA93EC85E058EA930E947E6BED85FE8523
:10209A00FA93EA930E941043AF91BF91EC93EC81BB
:1020AA000E94B36C0E94E46CEE810E94AD6C0E94A7
:1020BA00E46C0E94BC4819810881259608950E9403
:1020CA00EF6C0E94296C8F010E947E6B0E947E6BCE
:1020DA000E94836B0E94F26C0E94DB6C0E94F245A4
:1020EA00EA81EA930E9417180E94D36C0E94F96C45
:1020FA0019810881239608950E94EF6C0E94296C29
:10210A008F010E947E6B0E947E6B0E94836B0E94ED
:10211A00F26C0E94DB6C0E94F245EC81FD810E9408
:10212A00E06CAA81BB810E94C57C24F4A030E0E166
:10213A00BE070CF006C0EA81FB81FA93EA930E947B
:10214A00AB40AA81BB81A130E0E1BE0724F0A030F8
:10215A00E1E1BE070CF00AC0A6EEBBE0EA81FB8112
:10216A00E150F0410E94036D0E940B6D0E94F96CD0
:10217A0019810881269608950E94EF6C0E94296CA5
:10218A008F010E947E6B1A930A930E94BC48E0E07A
:10219A00E0933C0C099119910895E881EA930E9411
:1021AA0017180E94F71EE03051F10E94116D0E942B
:1021BA007E6B0E94156D0E94D36C0E94196DE88196
:1021CA00EA930E947720E8830E941D6D3B9734F0C2
:1021DA000E941D6D0E94286DE9E40BC0A3EEB6E0D3
:1021EA000E942C6D0E942F6D0E94346D0E94396DE1
:1021FA00E3E7EA930E948B45E2E0E0930E04CCC049
:10220A000E944F64E0E0E0930F04A0910403A4301D
:10221A0019F4EEEDF3E002C0EAEEF3E0FA93EA9382
:10222A000E94F14208950E9419460E944F640E943A
:10223A00A264E1E0E0930D040E94116DE6E0F0E093
:10224A000E943D6DEEEAF2E00E94E06C0E947E6B15
:10225A00E7E0F0E00E943D6DECE0F7E10E94E06CFF
:10226A000E94416DEA930E94B840E0E1F7E10E94C2
:10227A00E06CE0910403EA930E94B840E6E1F7E1DA
:10228A000E94E06C08952A971A930A930E947E6B23
:10229A000E947E6B0E94836BE4E6F0E00E94886BEA
:1022AA0000E010E01530B0F4053020F40E94466DCD
:1022BA00E03009F40DC00E947E6B0E94EC6B0E9414
:1022CA003D6D0E944D6D0E94466D0E94526D0F5FDA
:1022DA001F5FE8CF0E94546D0E94F245E2E8F2E0E7
:1022EA000E94E06CE091410CEA930E94B840E091B0
:1022FA00400CEA930E94BE400E94D86B0E94DB6C9D
:10230A000E94F245E6E8F2E00E94E06CE0912306C2
:10231A00EA93E5E0EA930E946E40E091190CE030FE
:10232A0079F10E94D86BE2E0F0E00E943D6DE09105
:10233A0028060E94576D0E948C6C0E94F245E0911B
:10234A002806E295EF70E695E695AE2FE09129060C
:10235A00EE0FEE0FEA0F0E94576D0E94DD6B0E948E
:10236A00F245E0912906E295EF70AE2FE0912A0638
:10237A00E295E07FEA0FEA93E6E0EA930E946E4074
:10238A00198108817DC1E881E064E7B9369A349BF6
:10239A00FECF349AE4B1F5B121960895E881F98126
:1023AA00AA81BB81AE17BF071CF4EA1BFB0B06C050
:1023BA00A881B981EA81FB81EA1BFB0B2496089567
:1023CA0028970E94D17CEFE0E0936100E1E00E944F
:1023DA005D6DE5E00E94646D0E946B6DE0936F0590
:1023EA00F0937005E0917B05F0917C05E0936D0513
:1023FA00F0936E05E1E0EA93C6DFE0937B05F09384
:10240A007C05EFE0E0936100E8E00E945D6DEAE0A0
:10241A000E94646D0E94706DE0936B05F0936C05E9
:10242A00E0917905F0917A05E0936905F0936A05E0
:10243A00E0E0EA93A8DFE0937905F0937A050E9439
:10244A00706DA0916B05B0916C05EA0FFB1FA0910E
:10245A007905B0917A050E94756D8F010E946B6DA6
:10246A00A0916F05B0917005EA0FFB1FA0917B0543
:10247A00B0917C050E94756D9F01E0916B05F0910A
:10248A006C050E947C6DFF93EF930E94706D0E9411
:10249A007C6DAF91BF91EA0FFB1FFF93EF93E09121
:1024AA007905F0917A050E947C6DAF91BF91EA0F90
:1024BA00FB1FE0937505F0937605E0916F05F091A7
:1024CA0070050E94826DFF93EF930E946B6D0E94CC
:1024DA00826DAF91BF91EA0FFB1FFF93EF93E091DB
:1024EA007B05F0917C050E94826DAF91BF91EA0F46
:1024FA00FB1FE0937705F0937805A0917505B091DD
:10250A007605E4E1F0E00E941B7A0E2EA091770591
:10251A00B0917805E4E1F0E00E941B7AE02919F015
:10252A000E94C044ABC000937105109372052093BA
:10253A00730530937405A0916405A63428F4E091DC
:10254A006405EF5FE09364050E94886D989724F410
:10255A000E948D6D98970CF00EC0A0916405AA3068
:10256A0019F4E1E0E0936105A0916405A83219F439
:10257A00E2E0E09361050E94886D999724F00E9439
:10258A008D6D99970CF47AC0E0916705EF5FE0933F
:10259A0067050E94926D0E94886D0E94976D0E9445
:1025AA009E6D0E94A36D0E944E7A7F936F93FF9354
:1025BA00EF93A2E0B0E00E94177B0F010E94926D98
:1025CA00DF01F001EA1BFB0BAF91BF918F919F9145
:1025DA000E94AC6D0E949E6D0E94B16D0E948D6D2D
:1025EA000E94976D0E94B66DAC81BD818E819F81DC
:1025FA00EFE3F1E060E070E00E944E7A7F936F9320
:10260A00FF93EF93A6E0B0E00E94177B0F010E94B0
:10261A00B16DDF01F001EA1BFB0BAF91BF918F9106
:10262A009F910E94AC6D0E94B66DE0911204E03059
:10263A0049F4E885F985E0935905F0935A05EC8148
:10264A00FD810AC0EC81FD81E0935905F0935A059A
:10265A000E94A36D0E94DE79E0935B05F0935C050E
:10266A00E0915905F0915A05FA93EA93E0915B05D6
:10267A00F0915C05FA93EA930E9448440E94D87C40
:10268A002C9608951A930E941946E2E0E0930E04EC
:10269A00E2E3F0E00E94A56B0E94BB6DE2E7F2E084
:1026AA000E94E06CE4E1EA930E941640E0E9F1E05E
:1026BA000E94BF6DE4E1EA930E941640A09167056B
:1026CA00A13010F0A895FACF10E0143010F00C9455
:1026DA00C813E2E0E0930D040E94C36DDF010E947B
:1026EA00E46CFD0132960E94E46C0E940D460E9441
:1026FA00C36D3496E491EA930E948B45E1E0E0933E
:10270A000D04A0916705AF3110F4A895FACFEAE05D
:10271A00EA930E9416400E94C36DDF0135960E941B
:10272A00FC7ABF01FD010E94C96DDB010E94277B73
:10273A000E94D06D0E94076CE8E2F0E00E94497A9C
:10274A00E65AFF4F0E94BB6D0E94C36D0E94C96D7D
:10275A000E94286DA0916705AE3110F0A895FACFB6
:10276A000E94C36DDF010E94E46CFD0132960E9453
:10277A00E46CE8E1F0E0FA93EA93E8E2F0E00E9420
:10278A00886B1F5FA2CF0E94D06DEAEFF0E00E9433
:10279A00BB6DEEE7F2E00E94E06CE0EDF7E00E942C
:1027AA00BF6D0E9419465FC10E94D56D0A93E4E687
:1027BA00E2BF78940E940A4403DEE6B3AFEFEA2749
:1027CA00E093410CE091400CE03009F002C0E09146
:1027DA00410CE0933008A2E6BBE00E94E46DE09170
:1027EA00620BE77031F4A0910A04E0E4EA27E0936F
:1027FA000A04E091620BEF7131F4A0910A04E3E854
:10280A00EA27E0930A040E94EE610E941621E2B3CD
:10281A00EF700E2EA0911408B0911508EFE0F0E0C9
:10282A00AE27BF27EA23FB230E94F779E029E2BB00
:10283A00E0911408E07111F41D9A01C01D980991E4
:10284A00199114C00E94D56DE6E0E4BDE0B1E295AD
:10285A00EF70AE2FE0916300E071EA2B1E2F0E9409
:10286A00C76C0E94ED200E94C8611991E991EFBFDF
:10287A00F991E991B991A99199918991799169917E
:10288A00F9901990099018950E94ED600E9478615C
:10289A000E94744C0E94351E08951A93A8950E94AE
:1028AA001E42E13011F00C94B314E091C605E150D8
:1028BA001E2FA091C505A13021F40E94EA6DE030D7
:1028CA0009F40CC0ADE01A9FF001E15FFC4FBF01B3
:1028DA00E081E260DB01EC930E94F16DA091C505F5
:1028EA00A23011F0A43089F40E94EA6DE093DB056E
:1028FA000E94F66D31F0FD01E15FFC4FE081E2706C
:10290A0009F403C01A930E94FF6DA091C505A33074
:10291A0019F41A930E94DD26A091C505A53029F461
:10292A00E091C605EA930E940A27A091C505A8303E
:10293A00A9F4E0E0EA93E091C605EF77EA930E94F2
:10294A00EA171E2F1F3F51F0E0E0EA930E9416405B
:10295A00E12FE058E093DB05E0932D06E0910A04AD
:10296A00E07821F1E0910A04EF77E0930A040E94EB
:10297A00E548E0910A04E07131F0E0910A04E2705E
:10298A00EA930E94F244E4EEEA930E943D62A09127
:10299A003D0CA13021F4A0911908A43009F406C015
:1029AA00E0EBEA930E943D62E093400CA0913C0C5C
:1029BA00A13039F4E0913E0CF0913F0C0E94036E75
:1029CA0009F401C0D9DB60DF4EC01A930E94194690
:1029DA00E1E0F0E00E94AA6B0E94F24510E00E943A
:1029EA000D6E0E947E6B0E94C76C0E94F245E091B8
:1029FA002008E03049F4EEE5F2E00E94E06C0E9423
:102A0A00136E0E94396D1E5FA0912008A130F0F06C
:102A1A00E0912008E150EA930E944618A091B30B76
:102A2A00AD3229F40E941C6E0E94C17C79F0E3EB5E
:102A3A00FBE00E940B6DE6E0F0E0FA93EA930E9455
:102A4A00296E0E941C6E0E94396D1E5FE09120085B
:102A5A00EF5FE09320081C3020F4A0912008AB30EF
:102A6A0008F001C0BECF199108951A930E94194621
:102A7A00E981E03019F4E0E0E0931E08A981A23070
:102A8A00A9F410E0A0911E08A13010F01C3008F043
:102A9A000DC0E0911E08E150E0931E080E942D6EC1
:102AAA0019F40E943B6E09F01F5FECCF0E940D6E75
:102ABA0010E00E947E6B0E94C76C0E94F245A091B2
:102ACA001E08A03408F50E942D6E19F40E943B6E70
:102ADA00D1F0E0911E08EA930E9417180E94D36C65
:102AEA000E947E6B0E94296E0E94466E0E94286D8B
:102AFA00E8E7EA930E948B450E94196D0E944B6E8B
:102B0A000E94396D1E5F05C0ECE1F7E10E94E06C9E
:102B1A001E5FE0911E08EF5FE0931E081C3020F450
:102B2A00A0911E08A13408F001C0C3CF18812296D3
:102B3A000895E0E0E5BFE0936D00E0936C00EBBB25
:102B4A00EFEFEABBE0E0E8BBE7BBE5BBEFEFE4BBD6
:102B5A00E0EFE2BBE1BBE0E2E3B9ECEBE2B9E0E0D3
:102B6A00E0936200E0936100EFE0E0936500E09398
:102B7A006400E0E0E0BFE7E0E3BFE4E6E2BFE0E0F4
:102B8A00E1BFEFBDEEBDEDBDECBDE7BDE6BDEBBD02
:102B9A00EABDE9BDE8BDE0937900E0937800E3E09F
:102BAA00E5BDE6E0E4BDE0E0E3BDE0938B00EAE0EA
:102BBA00E0938A00E0E0E0938900E0938800E093E4
:102BCA008100E0938000E2E1E0938700E4E3E09390
:102BDA008600E0E0E0938500E0938400E0938300C0
:102BEA00E0938200E0936A00E0E3EABFE0E4E9BF31
:102BFA00E8BFE1E4E7BFE0E0E0937D00EBB9E8ED90
:102C0A00EAB9E6E0E0939500E0E0E0939000E7E6B9
:102C1A00E9B9E0E0E0939B00E8EDE0939A00E6E092
:102C2A00E0939D00E0E0E0939800E3E3E0939900ED
:102C3A00E0E8E8B9E0E0E0BDE0E4E7B9E7E8E6B9F2
:102C4A00E0B5EF7EE0BDE0E2E0937000E0E0E09303
:102C5A007200E4E4E0937400EFE1E1BDEFE0E1BD6E
:102C6A000E947F590E94DB670E94E3447894E1E066
:102C7A00EA930E94860C0E94416DE53128F0A9E092
:102C8A00B0E0E0E00E942F7BCEDA21E030E0E0EE17
:102C9A00EA930E943D62E09331080E94546E3F5FBE
:102CAA00A0913108A43511F03A3008F001C0EFCFF5
:102CBA0030E0E0EBEA930E943D62EF3F19F0E1E079
:102CCA00E0933D0C0E94546E3F5FA0913D0CA030F2
:102CDA0011F43A3008F001C0ECCF0E94DB6C0E947C
:102CEA00D86B0E94F245EAE8F2E00E94E06CA091FB
:102CFA003108A43551F4E2EEEA930E943D62E09372
:102D0A003108EA930E948B4508C0E0E0E09331085D
:102D1A0020E0E0E9F2E00E94E06CA0913D0CA130D5
:102D2A0021F4E1E2F7E10E94E06C96D0E03079F418
:102D3A000E94DB6CE9E0F0E00E943D6DE4E9F2E01C
:102D4A000E94E06CE0E9F2E00E94E06C20E00E9460
:102D5A00926D0F01A2E0B0E00E94177B0E161F06CB
:102D6A0054F40E94B16D0F01A6E0B0E00E94177BF7
:102D7A000E161F060CF086DC203071F40E94DB6C04
:102D8A00EAE0F0E00E943D6DE8EAF2E00E94E06CC1
:102D9A00A8950E94576EFCCF0E9408360E94DB6CF1
:102DAA00E9E0F0E00E943D6DECE9F2E00E94E06C9F
:102DBA000E94BC1AE03019F0E2EAF2E002C0EEE743
:102DCA00F2E0FA93EA930E94A1450E940062E1E0D0
:102DDA00EA930E94164000E010E00436E0E01E0785
:102DEA0024F40E947861E03009F005C00E94546E14
:102DFA000F5F1F4FF2CF0436E0E01E072CF0A091C0
:102E0A006705AF3108F03EDC48DD0E947B310E9445
:102E1A00EC1CFACFFFCF0E945A6E17FD02C0103089
:102E2A0011F4E0E058C3E12F56C30E945A6E17FD11
:102E3A0010E01A3008F41F5F0E94676E4CC30E94AC
:102E4A005A6E17FD02C0103011F4E0E044C311506D
:102E5A000E94676EE1E03FC31A930A9310E0E4E62A
:102E6A00F0E00E94BF6DA8950E945762E03021F4FD
:102E7A00E0EA0E94726E09F002C001E001C000E0BF
:102E8A000E9468621F5F003011F4153008F001C01B
:102E9A00E6CFE02F0991199108950E94776E3FC4F9
:102EAA000E94776E0E94846E0895A881B9810E945B
:102EBA00C57C24F4A83EE3E0BE070CF005C00E94DE
:102ECA00876E0E94C86208C3E0E006C3EA81E03068
:102EDA0011F4EFEFEA83A881B9810E94C57C24F43A
:102EEA00A83EE3E0BE070CF006C00E94876EED81A3
:102EFA00EA930E94F5625AC10E94D17C20E030E038
:102F0A00283EE3E03E077CF4A8953A932A93CDDF66
:102F1A001E2F1F3F29F0EFEFEA933A932A93D6DF49
:102F2A002F5F3F4FEDCF0E94D87C4DC01A930A9372
:102F3A00E0E0F0E0E093420CF093430CAA81A03465
:102F4A0058F40E94906EE55FFB4F8F010E94976EC6
:102F5A00E2E4FCE00E94A06EE091420CF091430C86
:102F6A0023C11A931FEF1F5F1A93E0DFA981BA8169
:102F7A00EA17FB0711F0113408F001C0F4CFE12F72
:102F8A00188114C11A930A93A091C10BE091C20B44
:102F9A00EA9FF001A0911E08EA0F0E2F013408F0F3
:102FAA000FE310911E08101758F41A93BFDFAA8175
:102FBA00BB81EA17FB0711F4E12F03C01F5FF3CFB0
:102FCA00EFEF19810881249608950E94CF7C10E0C2
:102FDA00103418F50E94076CE8E2F0E00E94497A82
:102FEA00E050FC4FAF01E0EAEA93FA0170960E94C2
:102FFA00A46EEC713E2FE0EAEA93FA013F960E9432
:10300A00A46E0E2FEF81E31719F4EE81E01709F091
:10301A0002C0E12F03C01F5FDBCFEFEF0E94D67C17
:10302A00289608951A930A93E091890BAA81EA17C0
:10303A00C1F0A03468F40E94906EE050FC4F8F01FA
:10304A000E94A86E0E94A06EEA81E093890B09C0D3
:10305A00EFEFE093890B0E94B36E0E94B86EE09383
:10306A00940BA2C01A930A930E94906EE050FC4FF0
:10307A008F01AA81A03420F40E94A86E0E94846E57
:10308A0093C01A930A93E091B20BAA81EA17A1F0AE
:10309A000E94C26E40F40E94CE6E0E94A06EEA8127
:1030AA00E093B20B09C0EFEFE093B20B0E94D96E26
:1030BA000E94B86EE093BD0B77C01A930A930E94E0
:1030CA00C26E20F40E94CE6E0E94846E6DC01A9366
:1030DA000A93E091330CAA81EA1751F10E94DE6E3D
:1030EA0008F50E94976EE4E3FCE00E94A06EEA8174
:1030FA00E093330CE0E0E0932B06A091350CA1306D
:10310A0020F0A091350CA83008F00BC0A8EDBBE068
:10311A00E091350C0E94E86EAE0FBF1FEC91E09370
:10312A002B0606C0EFEFE093330CE0E0E093340C9B
:10313A003BC01A930A930E94DE6E30F40E94976E87
:10314A00E4E3FCE00E94846E2FC01A930A93E09194
:10315A002E0CAA81EA17C1F00E94EB6E70F4E0EA25
:10316A00EA930E94DD6B1A930A93EFE2FCE00E9455
:10317A00A06EEA81E0932E0C07C0EFEFE0932E0CCD
:10318A000E94F56E0E944A680FC01A930A930E9421
:10319A00EB6E50F4E0EAEA930E94DD6B1A930A930D
:1031AA00EFE2FCE00E94846E19810881239608955B
:1031BA000E94F56E0E944A68E881EF5FE093300C46
:1031CA00D4C124970E94CF7C0E94FC6E0E944A6858
:1031DA00AA85A03478F5AB85A13010F0A63008F0A6
:1031EA0007C0EB850E94E86E0E94036F0E94166F6B
:1031FA00EB85E030F9F4E0E0EE83EF83E887E987D6
:10320A0040E050E020E030E02530E0E03E0784F482
:10321A00F9010E94036F0E94166F0E94466E4E0FBC
:10322A005F1F0E944B6E0E941B6F2F5F3F4FECCFB8
:10323A000E94266F3AC11A930A93AB81A13010F00B
:10324A00A63008F01CC0EB810E94E86E0E94FB7950
:10325A000E94F779DF01EA810E94376FE8E0F0E027
:10326A000E94497AE050FA4E8F01E0EAEA930E94FE
:10327A00D86B1A930A93ECE1FCE00E94846E1981E0
:10328A0008810C94331E0E94D17CEC810E943B6F12
:10329A00E83109F454C00E94406F309729F00E9427
:1032AA00406F0E94456FEC830E94EB1E0E2F10E0C8
:1032BA00101710F00C94A4190E94496F82DFAEE136
:1032CA00BCE00E94E46DA091200CB091210C809189
:1032DA00220C9091230C0E944E6F0E94D979E093A0
:1032EA00200CF093210C6093220C7093230C0E9403
:1032FA00496FA1DFE0EAEA93EE810E94E86EEE0FE1
:10330A00FF1FE050F04F0E94A46EE270B1F4ED810D
:10331A00E093240C0E94406F309729F4EC81F0E08E
:10332A00EF5EF84D02C00E94406FE093250CF093C7
:10333A00260C0E94556F0E945A6F1F5FB9CF0E94D8
:10334A00D87C269608951A930A930E94606FECE23D
:10335A00F0E00E94676F0E946B6F0E94706F10E02E
:10336A001034D8F41A935EDEE0912108EA931A9396
:10337A0028DF0E94796FEA0FFB1F0F010E94796F05
:10338A000E94816FDF01CB010E944B6E0E94D979A6
:10339A00D0010E94F77A1F5FE3CFA0911908A330EA
:1033AA00B9F500E00031A0F50E94EC6B0E94866F2F
:1033BA0069F510E01A3050F5E02FE05DEA93E4E297
:1033CA00F7E10E948B6FE12FE05D0E94926FE1F4BA
:1033DA000E94976F0E949E6FEA0FFB1FFF93EF9365
:1033EA000E949E6F0E94816F7F936F93FF93EF936A
:1033FA000E94DB5DAF91BF918F919F910E94D97915
:10340A00AF91BF910E94F77A1F5FD4CF0F5FCACFE7
:10341A0010E01A3090F40E949E6F0E94816FA09172
:10342A002808B091290880912A0890912B080E94B7
:10343A00D9790E94706F1F5FECCF0C94791E249784
:10344A000E94CF7CEA85EA9371DD9F01022E032A4E
:10345A0039F13A932A9385DD1E2F40E050E0E0E0EF
:10346A00EE83EF83E887E987AA851A17B1F4012F5B
:10347A00003498F40A935ADD2E173F0761F4EB855E
:10348A00EA930A939EDE0E94466E4E0F5F1F0E94C9
:10349A004B6E0E941B6F0F5FEBCF0E94266F05C019
:1034AA00EB85EA93EB85EA938CDE0E94D67C2C9618
:1034BA0008951A93A895A981A63068F40E94FC6E13
:1034CA000E944A6810E0103430F4E981EA931A93B2
:1034DA00B2DE1F5FF8CF1881229608951A9311E081
:1034EA00163020F41A93E5DF1F5FFACF71C3E1E0CB
:1034FA00E093340CE093350C38C0A8950E94D96E3D
:10350A00EAE1F2E0FA93EA930E94D86B0E943A68E1
:10351A000E94A56FE093BB0B0E94AC6FE093BC0BBB
:10352A00E0E0E093BD0B21C0A895E9E8FBE00E942A
:10353A00B36FE9E2F0E00E94676F0E94B36EEAE1BE
:10354A00F4E0FA93EA930E94D86B0E943A68E88101
:10355A00EF5FE8830E94A56FE093920B0E94AC6F25
:10356A00E093930BE0EBE093980B219608950E9469
:10357A00CF7C0E94B86FE03228F0AAE0B0E0E0E029
:10358A000E942F7B00E089DCA091BE0BB091BF0B9B
:10359A00A633E2E1BE0741F110E01A3030F41A9383
:1035AA00ACDF1A938ADD1F5FF8CF10E0103430F4D5
:1035BA001A93BADF1A9356DD1F5FF8CF10E010385E
:1035CA0030F41A9394DF1A93B4DD1F5FF8CF86DFC5
:1035DA00A9E0B0E0E0E00E942F7BE6E3F2E1E093AD
:1035EA00BE0BF093BF0B01E010E0183210F00C9400
:1035FA004F1B0E94BD6F9F010E94BD6FAF010E94C9
:10360A00C76F3496E491E03011F0E13069F4D901E2
:10361A00AC910E94C76F3596E491EA1720F40E9494
:10362A00C76F0E94CE6F34C0E23091F4DA010E9473
:10363A00ED7AE031A7E2FA0714F4FF2342F40E947C
:10364A00C76F36960E94FC7ADA01ED93FC9320C08C
:10365A00E33049F4D901AC91AF3F21F40E94C76F1E
:10366A000E94CE6F15C0E43099F4D901AC91AF3FF6
:10367A0079F400E00E94C76F3596E4910E1740F482
:10368A000E94C76F0E94CE6F2F5F3F4F0F5FF2CF2E
:10369A001F5FABCF05DC10E0153060F41A9355DDDF
:1036AA00A0912F0CA63020F01A9382DD1A936DDDBB
:1036BA001F5FF2CFE02F0C941020E881EF5FE883C0
:1036CA00A881A43610F0E0E0E883E8810C948D200C
:1036DA000E942C6DA5E0B0E00E94497A30960C94C5
:1036EA008D20A091370CBB27E091360CA6C0F9DFDC
:1036FA00329774F00E94D36FE091360C0E94DA6F11
:10370A000E94846EE091360CEA93D7DFE093360C80
:10371A0008950E94D36FE091370C0E94DA6FFA93F2
:10372A00EA930E9416630895E4E2FCE00E94E26FC5
:10373A000E94D36FE091370C0E94DA6F0E94846E68
:10374A00E091370CEA93B9DFE093370C08950E94B1
:10375A00D17CE0E0E093360CE093370C10E030E0E7
:10376A00343680F5A8950E94D36F3A93B1DFFA9365
:10377A00EA93E4E2FCE00E94A06E00E0A091240C2F
:10378A00A13010F0A03808F001C001E0E12FE030CC
:10379A0041F4013029F43093370C3093360C11E0A0
:1037AA000FC0E13031F4003019F43093360C12E0D6
:1037BA0007C0E23029F4013019F43093370C13E0D2
:1037CA003F5FCECF49C21A93A091CF0BA870B9F030
:1037DA0010E0E981FA810E94076CAE17BF077CF4FA
:1037EA00ED81E093240CEB81FC81E851FC4F0E94AF
:1037FA00E96FE0E0F0E00E945A6F1F5FEACF18819C
:10380A000C941220E881EF5FE883A881A43610F0B7
:10381A00E0E0E883E8810C948D20E881E150E883B8
:10382A00A881A43610F0E3E6E883E8810C948D20A1
:10383A00A091390CBB27E091380CF0E031960E9438
:10384A00EE6FEC59FF4FDF01E4E6F0E00E94A67A42
:10385A0008950E942C6DA5E0B0E00E94497AE050DC
:10386A00FE4F0C948D200E94F36FE881EA93C0D139
:10387A000C948D201A9340DBE1E0E093860BA8C1FB
:10388A00A89510E0143680F41A93ABD1A091290CB4
:10389A00AF3F31F40E94F66FAF3FEFEFBE0711F072
:1038AA001A93E1DF1F5FEECF0E94FB6F689420F846
:1038BA008FC10E94D17C1091390CAD81AA23CAF51F
:1038CA00E091380CE11719F0AD81AA230AF030C053
:1038DA001A9387D10E94F66FEE81FF81EA17FB07E0
:1038EA0029F4E885A091290CEA1709F01EC00E9464
:1038FA000170EC81FD810E94E379EA17FB0744F429
:10390A000E9406700E940F70E0E0EC83ED830BC00A
:10391A000E940670EC83FD83E0E0F0E00E940F70E5
:10392A00E0E0E093290C1A9363D10E941470C8CF87
:10393A0046C0E091380CE11729F0AC81BD810E94A4
:10394A00C57C0CF01BC01A934CD10E94F66FEE8115
:10395A00FF81EA17FB0729F4E885A091290CEA17E9
:10396A0009F009C00E9406700E940F701A9340D194
:10397A00E0E0EC83ED830E941470DBCFAC81BD8163
:10398A000E94C57C1CF454DF33970CF418C0E885F8
:10399A00E093290CEE81FF810E941970EC81FD8170
:1039AA000E940F70E091380CEA9322D1E091380C12
:1039BA00EA9328DFE093380CE0E0EC83ED83689427
:1039CA0020F8EC81FD810E94D87C299608951A93EB
:1039DA00A091440CA03059F4E091470CF091480CA6
:1039EA00FA93EA93E8EBFBE00E941E7009F40BC01D
:1039FA00E1E0E093440CE091380CE093460CE0914E
:103A0A00380CE093450CA091440CA13011F00C94B1
:103A1A006F1DE091390CA091460CEA1711F40C9431
:103A2A00601DE091460CEA93F8DEE093460CEA93B7
:103A3A00D8D0A091290CA13010F0A03808F034C0D9
:103A4A00E091450CEA93E9DEE093450CA091460C1F
:103A5A00EA1749F1EA93CCD0E091E20BE030E9F4BD
:103A6A0010E01530D0F4ABE01A9FF001DF01E35209
:103A7A00FA4FE081E03049F0FD01E452FA4FE0816B
:103A8A00AE2FE091460CEA1709F005C00E94247097
:103A9A00A091450CA0831F5FE4CF0E94F36FE091D1
:103AAA00460CEA93A5D006C00E94F36FE091460C3B
:103ABA00EA939ED00FC0E091450CE093390CE0E008
:103ACA00E093440C689420F80E942D64E093470C1C
:103ADA00F093480C7DC01A93A8951091390CE09187
:103AEA00380CE117C1F00E942A700E94C57C64F468
:103AFA00EB81A091290CEA1739F40E94F66FE9814B
:103B0A00FA81EA17FB0709F003C0E12F1881A6C062
:103B1A000E941470E4CFEFEF1881A0C00E940170D8
:103B2A000E94C57C84F4E0912B06E87031F4E091A0
:103B3A002E08A091290CEA1731F40E942E700E94D7
:103B4A00456FE03408F001C05AC10C94EB20A895E7
:103B5A00E091380CA881EA1761F0E8810E9433707D
:103B6A0019F0E8810C948D20E881EA934BDEE88312
:103B7A00EFCFEFEF0C948D201A93A8951091390C82
:103B8A00E091380CE117E1F00E942A700E94C57C8E
:103B9A008CF4E0912B06E87031F4E0912E08A091A4
:103BAA00290CEA1739F40E94F66FE981FA81EA17BB
:103BBA00FB0709F002C00C94D2200E941470E0CFD7
:103BCA00EFEF0C94D3201A931091390C1A93BFDF9C
:103BDA0019910895E881EA9315DEE883EA93B7DF3D
:103BEA0097C20E94D36F0E943A700E94A06E90C240
:103BFA000E94D36F0E943A700E94846E89C20E940A
:103C0A00D17C0E94FB6F10E030E0343628F5A8958D
:103C1A003A93E7DF00E0A091290CA03808F401E00C
:103C2A00E12FE03041F4013029F43093390C30931C
:103C3A00380C11E00FC0E13031F4003019F4309340
:103C4A00380C12E007C0E23029F4013019F430933D
:103C5A00390C13E03F5FD9CF0E94D87C249608958F
:103C6A000E944370A43009F43FC010912E080091BD
:103C7A00530CE0913008E03059F0E0932E08689434
:103C8A0024F80E944870E0E0E0932F08E0E520C0A5
:103C9A00E0912F08E03021F0E0932E08E2E518C009
:103CAA00E0E0E0932E08E093530CE091C40BE0307F
:103CBA0031F0E091C40BE150EA930E946C18A09194
:103CCA00340CA17039F0E091C40BE0932E08E4E4BF
:103CDA00E093530CA0912E081A1721F4A091530CCB
:103CEA000A1711F0689423F80991199108950E940E
:103CFA004E70EBE0EC93EC81D8011696EC93EB81D5
:103D0A00D8011796EC93D8011896E0E0F0E0ED930D
:103D1A00FC93D80112960E945B70D80114960E94F7
:103D2A005B700E94607001C10E944E70ECE0EC93DF
:103D3A000E94607034C21A9318E0113108F5E091BC
:103D4A001408F0911508A981BA81EA27FB27BF0157
:103D5A000E946C70E623F723309781F00E946C7002
:103D6A00A981BA81EA23FB23309731F01A93E0E064
:103D7A00EA931A93BCDF02C01A93D6DF1F5FDDCF26
:103D8A000DC2A0911A0CA93030F0E0915B0CA09101
:103D9A005A0CEA1709F414C0E0915B0CE03021F4E4
:103DAA00E3E6EA93C1DF08C0E0911A0CEA93E0E087
:103DBA00EA93E3E6EA939BDFE0915B0CE0935A0C0B
:103DCA000895A0919A0BECE1EA230895A0919A0B29
:103DDA00A07411F0E2E00895A0919A0BA07809F07E
:103DEA00F5C10DC0A091890BAF3F09F4EFC1E9DF1E
:103DFA00E43009F4EBC1E5DFE03109F4E7C1E1E0C1
:103E0A0008950895A881AF3F11F4E0E081C1D9DF98
:103E1A00E43011F4E1E07CC1E0E07AC1A881A2308B
:103E2A0019F4CFDFE83011F0E1E072C1E0E070C1CF
:103E3A00A881B981AC91A130A8F0A881B981AC91CF
:103E4A00A43180F4A881B981EC910E947770EB5F6C
:103E5A00FC4FE081EF770E2EA881B9811296EC9182
:103E6A00E01509F002C0E1E011C1E0E00FC1A8814C
:103E7A00A13118F0E881E051E883E8810E947C7062
:103E8A000E948670A091D00BA13018F0A881A430AE
:103E9A0009F006C0E0EBF0E00E94FC7A0E9486700E
:103EAA0037C1A881A13010F0A63008F006C0E88119
:103EBA000E949170E15CF94F2AC1E0E029C1A88112
:103ECA00A13010F0A63008F006C0E8810E94917077
:103EDA00EC5BF94F1CC1E0E01BC10E94D17CEC8174
:103EEA00EA93EDDFEF731E2F1030E1F0EC81EA93D5
:103EFA00E6DFE0743E2FE12FE150A1E00E94EF7966
:103F0A00A0912306EA230E2F303011F4003009F075
:103F1A0002C0E1E008C0303011F0003009F402C0FC
:103F2A00E1E001C0E0E00E94D87C259608950E9455
:103F3A00CF7C00E00530A0F50A930E94AA180E94DF
:103F4A009670A7E10A9FF001EE5CF94F0E94B36FE9
:103F5A00E4E1F0E00E94676FE091300CDA015096DC
:103F6A00EC93A0912F0CEFE3EA23AE2FE091320CF1
:103F7A00E295E07FEE0FEE0FEA0FDA015596EC9329
:103F8A00E091300CE1503E2F3F3F41F0E091310C7F
:103F9A000E949D70DA015196ED93FC930F5FCACF90
:103FAA0010E01034C0F51A930E9417181A932ADFEA
:103FBA00E13079F5E0919D0BEA9373DFE1500E2F22
:103FCA000F3F39F10E949670E12FDA011396EC93B4
:103FDA00E0919D0BDA011496EC93E091A30BF0911A
:103FEA00A40BDA011696ED93FC930E944E6FA4E699
:103FFA00B0E080E090E00E944E7ADF01CB01E091D0
:10400A00A30BF091A40B0E94AC6DDA011A96ED9302
:10401A00FC931F5FC6CF0E94D67C26960895A09176
:10402A001908A23031F0A83021F0A73011F0A530DC
:10403A0009F40AC00E94606FEFEFF0E00E94676F18
:10404A0076DFE0E0E093A20608951A93E981E0584A
:10405A00E98310E01530C0F4A3E21A9FF001EB5592
:10406A00F94FE081AE2FE981EA1749F4F001EC55E6
:10407A00F94FE081AE2FE0912E08EA1709F002C04D
:10408A00E12F03C01F5FE6CFEFEF18812296089554
:10409A000E94D17CED81EA93D8DF1E2F1F3FF1F0F9
:1040AA00A3E21A9FF001ED55F94F9F01D90112962B
:1040BA00EC91EF77EC93EC81D901EC930E94777045
:1040CA00EF5EFC4FBF01E081EF77DB01EC93EC81FF
:1040DA000E947770E15FFC4FA1E0A083E12F0E946C
:1040EA00D87CDCC40E942C6D0E94A37061F4E0911C
:1040FA004D0CEF5FE0934D0C0E942C6DED55F94F7E
:10410A00A0914D0CA0830E942C6DED55F94FE081D2
:10411A00219608951A931FEFE091D40BF091D50BD5
:10412A00A981BA81AE17BF073CF0E091D60BF09196
:10413A00D70BEA17FB070CF412C00E94A8700E9462
:10414A005A171E2F103031F01F3F21F0E0912E0830
:10415A00E11729F4E1E0E0935B0CE0E01FC0E0E046
:10416A00E0935B0C1AC01A930E94A870D3DF1E2F2B
:10417A00103099F01F3F39F4ECE0F6E0FA93EA9335
:10418A00EB81FC8106C0E6E2F6E0FA93EA930E942C
:10419A00AD70FA93EA930E948110E12F1881239659
:1041AA000895E0916505E03009F00895E0912C0644
:1041BA00E03009F008950AC0E0916605E03009F0A0
:1041CA000895E0912D06E03009F00895E0E00895A1
:1041DA000E94D17CE0912606F0912706AC81BD8130
:1041EA00EA27FB279F0110E0153090F4F901E170EE
:1041FA0049F0A7E11A9FF001EF5CF94FDF01EC915A
:10420A00EF5FEC93D9010E94B0709F011F5FECCF62
:10421A00EC81FD81E0932606F09327060E94D87C64
:10422A003DC428970E94CF7C3091260610E01530B5
:10423A00B8F5A7E11A9FF001EB5BF94F0081E12F76
:10424A00A1E00E94EF792E2FE22FE32391F00038AC
:10425A0010F0003C08F001C00F5F003C31F4E22F7F
:10426A00A0912306EA2BE0932306003808F400E81D
:10427A000FC0003408F40F5F003439F4EFEFE2277F
:10428A00A0912306EA23E0932306003808F000E011
:10429A00A7E11A9FF001EB5BF94F00831F5FC7CFBD
:1042AA00E0E0E0932C06E0E0F0E0E0931608F093FB
:1042BA001708E0915B0CE03021F0E0911A0CEA93C8
:1042CA00D6DDE0911D08EF5FE0931D08E091E30B56
:1042DA00A0911D08EA1751F4E091E30BF0E0A0E089
:1042EA00B1E00E94107BEA1BE0931D08A091190817
:1042FA00A13019F0A93009F096C0A091620BB091D3
:10430A00630BE4E1F0E00E94A67A309719F4E1E049
:10431A00E0931F0846DFE03019F04EDFE07809F439
:10432A0062C04ADFEF775E2F5A930E9417180E94E5
:10433A00776CED55F94F5081503011F40C94F821F7
:10434A0051DDE13031F4E0911A08EA9367DDE0309B
:10435A0009F449C00E94B5700E94376FEC91EC7164
:10436A00EC3021F4E0911D08E07851F40E94BA7013
:10437A00EC91EA937CDD0E94BF70EC91EA9377DDC1
:10438A000E94BA70AC91A63070F5A3EEB6E00E9416
:10439A00776C0E942F6D0E94E46D0E94BA70EC91B6
:1043AA00EA937FDD1E2F1130F0F00E94C4700E9444
:1043BA00C770CF010E94C4700E942F6D6D917C91CD
:1043CA00E12F0E949170EF5CF94F0E94CC70E60FCA
:1043DA00F71FDC01ED93FC93E12F0E949170EF5CD3
:1043EA00F94FA0E0A08310E01530E8F40E94CF70E6
:1043FA0013965C915F3FA9F05A9374DE5E2F0E9478
:10440A00D9700E94C4700E94C770BF010E94C47014
:10441A000E942F6D0E94DF70AE81BF811296E0E08C
:10442A00EC931F5FE1CFA0911908A23039F0A830B0
:10443A0029F0A53019F0A73009F0E2C100E00530F3
:10444A0010F00C940524A3E20A9FF001ED55F94FF0
:10445A00EA87FB87AA85BB85AC91A03019F0A281B7
:10446A00A07809F0CBC1AA85BB8513960E94ED7A84
:10447A00309771F0AA85BB8513960E94EC700E9452
:10448A00F27029F4AA85BB8513960E945B70B6C1A7
:10449A0093DEE03021F00E94F27009F4AFC120E00F
:1044AA0030E0333010F00C94B0230E94FC70DF012E
:1044BA000E94046C0E94036DE887F987A181A270AB
:1044CA0021F4A481B581109709F410C1E885F98512
:1044DA00A181A47011F40C94D222A181A87021F4B4
:1044EA000E94E332E03009F457C00E940271EBE007
:1044FA00EC93A885B9850E940F71A885B985139692
:10450A00EC91AC85BD851796EC93EC85FD853896C4
:10451A000F01E885F985A181E1E0EA230E9416717D
:10452A00ED93FC93A885B98514960E94ED7AAC8523
:10453A00BD851296ED93FC930E941971AC85BD85D9
:10454A001496ED93FC93A02FEAE0EA9FF001E30FA3
:10455A00EF5F0E941F71E885F985A085B185E2E0C9
:10456A00F0E00E94497AA885B9851896ED93FC93E4
:10457A000E941971309739F4A885B9851896E8EE22
:10458A00F3E0ED93FC93E885F985A181E8E0EA2B55
:10459A00A885B9851196EC936EC0E885F985A18145
:1045AA00A17031F4A885B98514960E94EC7043C0B5
:1045BA000E94287176DCE1501E2F0E94CF7012965D
:1045CA00EC91E03001F5AE81BF8153960E94E46D13
:1045DA00EE81FF81A189B289109751F0038814886E
:1045EA00AE81BF8151960E94ED7AE015F1050CF07B
:1045FA0009C00E94576C1CDCE03011F00E942D713A
:10460A000E9435710EC0E885F98534960E943D7185
:10461A000E9416710E94EE6F0E94457153960E9485
:10462A005B70E885F985A581AA232AF4A885B9854E
:10463A0014960E945B70A885B985EC91EC71EC30F8
:10464A0021F4E0911D08E078B1F4E885F985A481A8
:10465A00B5815E971CF4A181A07209F404C0E885B3
:10466A00F985A28106C00E94287101DCE885F985D6
:10467A00A381AA93FCDB0E941971309791F0A88557
:10468A00B98518960E94EC700E941971309749F406
:10469A000E94576CCDDBE03011F00E942D710E9410
:1046AA0035710E94287119DCE03001F10E94576CC3
:1046BA00BFDBE03049F00E942D71AA85BB85EC91E1
:1046CA000E9477700E947F6CAA85BB851296EC9136
:1046DA00E058AA85BB851296EC93E3E0E0932406A2
:1046EA000E942871ECDBEF73E0932506A885B98553
:1046FA0014960E94ED7A309761F52F5F323048F5B3
:10470A00A885B98516960E94ED7A309789F0E885D2
:10471A00F985A681B7810E944C71AA85BB8513963B
:10472A00ED93FC93A885B98516960E945B7011C01B
:10473A000E94FC70DF01E32FEF5FF0E00E94036D3F
:10474A00E887F987A181EDEFEA23A885B985119653
:10475A00EC933F5FA6CE233011F00C9403240E9401
:10476A00E332E03069F00E940271E8E0EC93AA8536
:10477A00BB850E940F71AA85BB85EC910E941F71AF
:10478A000E94576C55DBE03011F00E942D71AA850A
:10479A00BB85E0E0EC93EA85FB85A581ECE1EA23A1
:1047AA00E83061F50E94416DAE2FEA85FB85E38D05
:1047BA00EA1741F4EA85FB85E48DE150EA930E9409
:1047CA001A171CC00E94E332E030C1F00E94027145
:1047DA00E3E0EC93AC85BD85EFEFEC931896EA85A0
:1047EA00FB85E38D0E945171AC85BD851296EA85E1
:1047FA00FB85E48D0E9451710E9455710F5F1FCE97
:10480A000E945B7149F4A0911908A23021F0A830E6
:10481A0011F0A53009F401C050C010E0153010F0B5
:10482A000C9462240E94CF7013965C915F3F11F43E
:10483A000C9460240E94D970AE81BF81BD010E9490
:10484A00DF70EE81FF8138960E943D710E9461718E
:10485A000E9445710E94ED7ADF010E94C57CB4F482
:10486A00EE81FF81A681B7810E94C57C7CF4AE816E
:10487A00BF810D901C90AE81BF8116960E94ED7A81
:10488A00D001AE1BBF0B0E94C57C0CF014C0AE81D8
:10489A00BF81BD010D901C90EE81FF81A681B78179
:1048AA00F001EA1BFB0BDB01ED93FC935A93E5E065
:1048BA00EA930E943C421F5FB1CFE0911C08E030AE
:1048CA0041F4E0911608F0911708E0931408F09368
:1048DA0015080E94D67C2E9608950E94D17CA0913C
:1048EA00C10BE091C20BE150EA9FF001EF5F1E2F6E
:1048FA002FE330E000911E08A091180CA13080F03F
:10490A00E091180CE150A0911E08AE1728F0E09132
:10491A00180CE1503E2F04C0E091180CE2502E2FE3
:10492A00EC81E03049F1EF3F51F4A0911E08A11B40
:10493A00A31720F0E0911E08E11B0E2F1DC0EE3FC9
:10494A0059F4E12FA0911E08AE0FA21720F4A091EE
:10495A001E08EA0F0E2F10C0EC3F49F4A091180C64
:10496A00A13020F0E091180CE1500E2F05C0AC8167
:10497A00A1501A9FF0010E2FE0911E08E01751F086
:10498A000A930E941718A0918A0BAD3209F4032FDB
:10499A0000931E080E941946A0911908A83019F41C
:1049AA000E94950E02C00E940E0E0E94D87C259687
:1049BA0008950E94CF7C05DAE03111F40C94502559
:1049CA0020E030E040E050E010E0133060F50E9453
:1049DA0065710E942F6D0E94ED7A309711F10E9445
:1049EA0068710E947C702E2B3F2B0E946871EA939B
:1049FA0074DAE03029F0E3E0E0932406E0E04CC00A
:104A0A000E946F710E947C702E2B3F2B0E946F7147
:104A1A00EA9363DAE03029F0E3E0E0932406E0E089
:104A2A003BC01F5FD2CF00E0053058F5A3E20A9FD2
:104A3A00F0010E94A37019F110E0133000F50E94F2
:104A4A00FC70DF010E94AD700E947671AE0FBF1F2D
:104A5A001296EC910E947C704E2B5F2B0E94FC7088
:104A6A00DF010E94AD700E947671AE0FBF1F1396D0
:104A7A00EC910E947C704E2B5F2B1F5FDECF0F5F85
:104A8A00D3CFF901E423F523309729F0E1E0E0934D
:104A9A002406E0E001C0E1E00E94D67C2696089553
:104AAA001A93E091510CE03011F40C94AA25E0918C
:104ABA00E40BE13059F4A091510CA13311F4EFE069
:104ACA0001C0E0E0EA930E94175A3FC0E23059F46D
:104ADA00A091510CA13311F4E6E001C0E5E1EA939B
:104AEA000E94175A32C0E53061F4A091510CA133EB
:104AFA0019F4E091990B01C0E0E0EA930E94175A79
:104B0A0024C0E330B1F410E0173040F40E94AD70D5
:104B1A00E15CF64F0E947D711F5FF6CFA091510CA8
:104B2A00A13311F4E1E301C0E0E3EA930E94175ACA
:104B3A000CC00E948171E9E4EA930E947F5EE091D1
:104B4A00510C0E9488710E948D7187C422970E941D
:104B5A00CF7C30E0A0911908A23029F0A83019F0D2
:104B6A00A53009F021C1A985A03410F00C94D826EB
:104B7A00E0912E08E03009F417C1E9850E943B6FE5
:104B8A00E03131F4E1E3E093510C8ADFE1E00CC15A
:104B9A0029D9E03009F408C110E01530A0F4A3E2E5
:104BAA001A9FF001DF010E94A37041F0FD01EB554D
:104BBA00F94FE081AE2FE985EA1709F002C0E0E07B
:104BCA00F3C01F5FEACFF5DEE03011F40C94D8266B
:104BDA0010E0A3E21A9FF001ED55F94FEE83FF832F
:104BEA00AE81BF81EC91E03011F00C94D12613967E
:104BFA000E945B7000E0033010F00C94A026A3E240
:104C0A001A9FF001E855F94FDF010E94EC6B0E94F0
:104C1A00036DAF01DA0116960E945B700E949271D1
:104C2A00DA011296EC930E949971DA011396EC93C9
:104C3A00A0919A0BEEEFEA23DA01EC930E94A0719D
:104C4A00DA011196EC93BDD8E43139F0FA01A18169
:104C5A00E2E0EA2BDA011196EC930A93DFD8E0300E
:104C6A0011F40C948226FA01A281AA931AD9E1506E
:104C7A002E2F2F3F81F0A7E12A9FF001EF5CF94F19
:104C8A00A0E0A083A7E12A9FF001EE5BF94FA0E024
:104C9A00B0E0A083B1830E94A8710E942F6D0E9488
:104CAA00ED7ADA011496ED93FC93013040F00E94FC
:104CBA00A8710E942F6D0E94ED7A309709F00EC0FC
:104CCA00AE81BF811596E02F0E94E86E0E94767130
:104CDA00AE0FBF1F1196EC91E062EC93AE81BF81DB
:104CEA005A96EC91E062EC93023030F40E94AB7178
:104CFA00DA0116960E94517104C0DA0114960E94D4
:104D0A005B705FD8EC3019F4E0E0E0931D080E9474
:104D1A00B2710E949D70DA011896ED93FC93FA0124
:104D2A00A281A63030F0A181E4E0EA2BDA011196E3
:104D3A00EC930F5F60CFA0911908A23011F0A53053
:104D4A0019F4A885AF3F08F007C0E0912E08EA934E
:104D5A00EA85EA930E944819E885AE81BF81EC93FF
:104D6A00E0912E08AE81BF811196EC93E985AE8160
:104D7A00BF811296EC93A885A43138F4E8850E9485
:104D8A007770E15FFC4FA1E0A083AE81BF811696E8
:104D9A00EC91ED7FEC9331E01F5F303011F4153068
:104DAA0008F001C016CFE32F0E94D67C2A960895F8
:104DBA000E944370A23021F0A0911908A53021F475
:104DCA000E94B9710E94FF6DA0911908A830C9F418
:104DDA000E94B971E1E0EA930E947C46E091E20BFD
:104DEA00E03069F4EA810E94C471E081EF771E2FF6
:104DFA00ABE01A9FF001EA51FA4FA0E0A083689451
:104E0A0020F8198108812396089564970E94206CDE
:104E1A00A23039F4E0912E08EA93EB8DEA930E94CE
:104E2A004819A0911908A83011F00C9480270FEFA7
:104E3A0020E0253050F4A7E12A9FF001EE5CF94FFB
:104E4A00E081AE2FEA8DEA1709F402C02F5FF1CF95
:104E5A00A7E12A9FF001E15DF94FAF01DA0115964A
:104E6A000C910F3F11F40C9480270E94CA71108193
:104E7A000E942A700E94C57CECF4ACE2BCE00E945D
:104E8A00EC700E94D0710E940170A083B1831A93C2
:104E9A000E94FD1DABE00A9FF001E252FA4F3081F9
:104EAA000A93FE0137960E94D6713A93FE0137960D
:104EBA000E94DA710E94E071F1F40E94CA71AFEFA8
:104ECA00A083DA011396EFEFEC93DA011596EC93CF
:104EDA000E94D0710E94E671E0E0F0E00E940F703B
:104EEA00E0E0E093290C1A930E94FD1D0A930E94A8
:104EFA00FB0F689420F80E94D67C6B9608951A934B
:104F0A0010E01031B0F4A7E11A9FF001EC5BF94F01
:104F1A00E081EF73AE2FE981EA1729F41A930E9410
:104F2A00721FE03009F403C0E1E01881E0C01F5F9E
:104F3A00E8CFE0E01881DBC01A93E091540CF091BD
:104F4A00550CFA93EA93E4EFF1E00E941E70F9F02F
:104F5A000E94EB7110E01530D0F4A091580CAF5FAD
:104F6A00E5E00E94A37AE093580CEF5FEA93C7DF6B
:104F7A00E03059F0E3E0E0932406E091580CF0E0C9
:104F8A00EF5FFF4EE093250668C21F5FE4CF65C25C
:104F9A001A93E0912306E093500CE8E7F0E0FA93C5
:104FAA00EA93ECEDF0E0FA93EA930E94494610E0A6
:104FBA001530D8F4E12FEF5FEA93A1DFE03099F0E2
:104FCA000E947E6BE12FEA5FF0E00E943D6DE4E310
:104FDA00F6E00E94E06CA6EEBBE00E94AD700E9473
:104FEA00036D0E940B6D1F5FE3CF37C2A5DFE0910F
:104FFA002406E13029F4ECE3F6E00E94F2713CC0A9
:10500A00E23029F4E8E9F0E00E94F27135C0E330B9
:10501A0051F4E4E3F6E0FA93EA93E0912506F0E02E
:10502A00E050F04F29C0E43019F4EAE4F6E01FC07A
:10503A00E53031F4E0912506EA930E94641020C01D
:10504A00E63019F4E2E5F6E012C0E73029F4ECE8BC
:10505A00F0E00E94F27110C0E83029F4ECE0F6E0CA
:10506A000E94F27109C0E93059F4E6E2F6E0FA93D7
:10507A00EA93E0912506F0E0FA93EA930E94811000
:10508A00E0E0E09324060895A881B9811196E1E051
:10509A00EC930E942E70A881B9811296ED93FC932D
:1050AA000E94EB1EA881B9811796EC930E94416D6C
:1050BA00A881B98118960E945171E091C605A8810C
:1050CA00B981EC93E091290CA881B9811696EC93E9
:1050DA00E091890BA881B9811A96EC93E091AC0B07
:1050EA00F091AD0BA881B9811496ED93FC932296A9
:1050FA00089564970E94D17CA091E20BA230E1F45A
:10510A00EB8DEA930E9417180E94EB1EACE2BCE0FA
:10511A000E945171AAE2BCE0EB8D0E945171E091AC
:10512A002E08E093290C0E94406F309721F00E94CC
:10513A00406F0E94197014C0AA8DAF3F09F4CAC00B
:10514A00EA8DEA930E94F61DAB8DAF3F29F40E94C7
:10515A002E700E94456FEB8FEB8DEA930E94171811
:10516A000E94EB1E0E2FA98DAF3F21F00E94F71E61
:10517A00E03009F001C0AEC00E9401700E94EC6BE1
:10518A00AE17BF071CF015DCE13009F0A3C0A091EF
:10519A00D10BA03021F4A091E20BA23011F50E94AC
:1051AA00416DE13041F00E94E332E03021F00E948B
:1051BA00F932E03009F002C00E94F7710E94416D95
:1051CA00E13021F40E94E932E03009F409C00E947A
:1051DA000372EE55F84FFA93EA9356DF0E9409726A
:1051EA0077C0EB8DEA93EA8DEA93B0DC1E2F11307B
:1051FA0011F00C946D29A091D30BA13059F4E091D0
:10520A002E08EA930E942E70FA93EA93EFEFFFEFCB
:10521A000E940F720E9401700E94EC6B0E94EE6F56
:10522A000E940F70689420F8A091E20BA03019F444
:10523A00A88DAF3F09F437C00E941372EE51FA4F9E
:10524A000E940170A083B183E88D0E94E96C3081CD
:10525A00E88DEA93FE0135960E94D671E88D0E9488
:10526A00E96CE081EA93FE0135960E94DA710E94A8
:10527A00E61EE03131F00E941372EA51FA4FA1E0C2
:10528A0005C00E941372EA51FA4FA2E0A0830E945D
:10529A001372EC51FA4FFF93EF930E942D64AF9172
:1052AA00BF91ED93FC930E94E07119F4E0E0E09362
:1052BA00290CEA8DEA930E94FD1DE0912E08EA93DB
:1052CA000E94406F0E941872FA93EA930E94E81BA8
:1052DA00E1E001C0E0E00E94D87C6C96089569DBA9
:1052EA00E13041F40E94E332E03021F00E94F932C9
:1052FA00E03009F007C00E94406F0E9419700E94B6
:10530A00F77130C338C30E94D17C0E941B721F3FC1
:10531A0011F40C94D929E091510CE03011F00C945D
:10532A00D8291A930E941718E5E0E09324061093EF
:10533A002506A0911908A23031F40E9424720E9415
:10534A00B820E03009F00EC0A091520CA13331F41C
:10535A00E0912E08EA931A930E944819E1E3E09338
:10536A00510C1DC2A0911908A83091F40E94406FF7
:10537A000E9428720E2F0A930E945B333E2F1A93C3
:10538A000A93EFEFEA933A93B4DEE03009F007C2EA
:10539A00A0911908A53021F4A2DFE03009F0FFC17D
:1053AA00E0E3E093510C06C0E0E3E093510CE4E043
:1053BA00E0932406F4C1E0913F090E942C720895FB
:1053CA001A93E6E0EA930E94175A0E948171A0910B
:1053DA003F09A83539F4E8E2F7E10E943872E0E0C3
:1053EA000E948D71A0913F09A33509F510E0A091A3
:1053FA001908A83021F0A23011F0A53009F411E300
:10540A00E3E5EA930E947F5E1A930E947F5EE0E8DA
:10541A00EA930E947F5EE0E8EA930E947F5EE0E8FA
:10542A000E948871E093510CE0E00E948D71A09176
:10543A003F09A93491F4A091E40BA43019F4E0E0F7
:10544A00E093510C0E943C72E09325060E9446723A
:10545A00EC91E093520C57DF23DB199108950E94D7
:10546A00D17C0E944B72E2E3F0E0E0934B0CF093A4
:10547A004C0CA0913F09A73741F4E3E4F9E00E94FC
:10548A0052720E9457720E942C72A0913F09A03357
:10549A0010F0AA3308F025C0209126083091270879
:1054AA00EFE3F9E00E945272E2E0EA930E94255E7D
:1054BA000E2F013090F00E945772E09325060E9449
:1054CA0057720E945B720E941B720A931A930E947F
:1054DA0048192093260830932708E2E5EA930E94A8
:1054EA00175A5DC1A091E40BA33069F4E091490C0D
:1054FA00F0914A0CFA93EA93E0914B0CF0914C0C20
:10550A000E941E7009F40FC0E0E0E0933909E5E457
:10551A00EA930E94175A0E944B72E8ECF0E0E0937B
:10552A004B0CF0934C0C08950E94C26C0E94AD0D76
:10553A000E9460720E947E6B0E947E6B0E94F245FE
:10554A00A0911B08A23021F4E0EAF0E00E94E06C8E
:10555A00A0911B08A13021F4E2E5F6E00E94E06C7C
:10556A00E0911B08E03021F4E8E5F6E00E94E06CE7
:10557A000E946A720E94AA6B0E94F2450E946D7292
:10558A000E947272FA93EA93E0915F05F0916005C6
:10559A000E9478720895E1E003C0E0E001C0E2E011
:1055AA00E0931B08C1DF08950E94E61EEC3109F062
:1055BA00E2C1E091990BE33631F4A0911908A230C7
:1055CA0009F4EBDF17C0E23631F4A0911908A230D2
:1055DA0009F4E5DF0FC0A091C505A23011F0A6308D
:1055EA0021F4E091990BEA9378D9A091C505A430EA
:1055FA0009F4D1DFB7C11A930A93A0E023FCA1E012
:10560A00A03019F0AA81A03009F014C0E89423F858
:10561A00E7E0E09318080E943445A0913008A030D2
:10562A0019F40E947C7209F405C00E9481729AD70B
:10563A00E89424F824FE24C00E948672EAE5F0E089
:10564A000E948D7219F0AA81A130C9F4B7D7E0304F
:10565A00B1F00E9493720FEF1FEF0E9424720E9412
:10566A008F20E03021F40091260810912708EB8161
:10567A00EA93E0912E08EA931A930A9373D70BC020
:10568A000E948672ECE2F1E00E948D7221F40E947F
:10569A009A72E0932F081981088183C00E94116DC4
:1056AA000E947E6B0E94156D0E947E6B0E947E6B2B
:1056BA000E94F245E4EEF5E00E94E06CE0911A08DF
:1056CA000E949E72E2EFF5E00E94E06CE2E0E09355
:1056DA000E0408950E94606FE0ECF0E00E94676F8C
:1056EA00E881E03009F406C0A0911A08AF5FE3E050
:1056FA000E94A37AE0931A08E1E0E0934D0C0E941D
:10570A009C1F26C20E94D17C10E0103410F00C9429
:10571A00D42B0E94AD70ED55F94F30813F3FE9F12E
:10572A001A930E94171800E00E94A2720E942F6D1D
:10573A000E94ED7A3B9794F00E94A5720F010E9495
:10574A00A2720E942F6D0E94AB720E94B1720E94D7
:10575A00376FEC91EE7FD001EC9301E00E94B672B4
:10576A000E942F6D0E94ED7A759794F00E94A5729F
:10577A000F010E94B6720E942F6D0E94AB720E94A6
:10578A00B1720E94376FEC91E160D001EC9301E0B5
:10579A00013019F41A930E9437181F5FB6CF0E947E
:1057AA00D87C249608950E944370A93011F40E946F
:1057BA00B97223FE06C0E7E0E09318080E948172DE
:1057CA00D1D60E944C42E030A1F1E0E00E94C072C2
:1057DA00103838F5113231F4E7E0E09318080E94E6
:1057EA008172C0D61D3439F40E94C7720E949F5F2D
:1057FA00E3E0E09318081B3271F40E94CC72EAE2EB
:10580A00EA93E3E3F7E1FA93EA93E0911A08E05D99
:10581A00EA930E949F5F1F3219F4E1E0EA935DD890
:10582A003DDF103830F00E94D2721A930E9477201E
:10583A00BBDE0E94E1200E2F003810F40C94652C78
:10584A000F770034E0F5E0911F08E03069F00A9321
:10585A000E947720A0911908A13019F40A930E9496
:10586A00D210E0E0E0931F08E091590CE01739F1FB
:10587A000A930E9417180E94BA70AC91A83028F4B3
:10588A000E94BF70AC91A830A8F0E02FEF5FE093C0
:10589A00A2060A930E9477200E94BA70EC91EA93BA
:1058AA000E94BF70EC91EA93E091A206EA930E94EB
:1058BA007C1E03C0E0E0E093A2060093590C0EC0E0
:1058CA00A091590CAF3F51F0E091A206E03019F0D7
:1058DA00EA930E94991EEFEFE093590C09911991EE
:1058EA000895A881A03310F0AA3308F01DC00E94C1
:1058FA00D6720E94DB72AAE0B0E00E94497ADF0108
:10590A00E8810E94E072EA0FFB1FE0932408F093FB
:10591A002508E2E0E0930E040E946A720E94AA6BD4
:10592A000E94156D0E946D72A881A33451F40E94E1
:10593A0060720E946A720E94AA6B0E94156D0E9490
:10594A006D7206C1E091C70BF091C80B0E94E37219
:10595A0011F4E2E00895E091C50BF091C60B0E94A4
:10596A00E37211F4E1E00895E091CB0BF091CC0BD6
:10597A000E94E37211F4E0E00895EFEF0895E0E089
:10598A00E0931B08A0911908A23021F40E9419463D
:10599A000E940E0EA0911908A83009F442D6A091CF
:1059AA001908A53009F441D10895E2E0EA930E946A
:1059BA001640E2E0E0930E04E881EA9392DFA881C0
:1059CA00AF3721F4E0912B06E37009F403C0E2E05B
:1059DA00E0931808A881A13239F0A33421F40E9477
:1059EA00D672109709F004C0A0911908A23009F0E4
:1059FA000FC0A0911B08A33009F4D1DDA0911B08A8
:105A0A00A23009F4BCDFE0911B08E03009F4C5DDDF
:105A1A00A881AD3311F00C94692D0E943445E091B0
:105A2A001B08E030A1F4E0912408F0912508FA93CC
:105A3A00EA930E94B820E03041F4E0912408F09102
:105A4A0025080E945B729BDF01C0A7DD3DC0E130E3
:105A5A0069F478DFEF3F41F0E3E00E94E7720E94C9
:105A6A00C7720E94ED7201C08ADF2EC0E230F1F4E3
:105A7A000E94D672A034E0E0BE07B4F4E091240894
:105A8A00EA930E94F472E2E0E0930E040E947E6BB5
:105A9A000E947E6B0E94F2450E94D36C0E94630FA3
:105AAA00E3E0E0931B0801C07ADD0EC0E33061F445
:105ABA00E0912408EA930E941718E0912408EA93D7
:105ACA00EEEFEA9343D86BDDA881AD3409F463DDC8
:105ADA00A881A43521F4A0911908A23009F001C0C7
:105AEA005CDDA881AB3221F4EEEFEA930E947224C6
:105AFA00A881AD3221F4EFEFEA930E947224A881C3
:105B0A00A73421F4E1E0EA930E947224A881AB341D
:105B1A0021F4ECEFEA930E9472241AC00E94142026
:105B2A000E941946E0E0E0931B08A881A13039F4ED
:105B3A000E947C7221F0A091CA0BA03009F402C025
:105B4A002CDD06C00E940E0E0E9424720E948F2035
:105B5A00219608951A930A930E94B9720E94F872C4
:105B6A0091F10E94007378F10E94D2721DDDE0303B
:105B7A0051F50E9408730E944D20EF3F09F0EFC4CF
:105B8A000E9424720E94B820E03021F40E94F71E7D
:105B9A00E13009F018C00E94E61EE83119F40E94AB
:105BAA000D7309F001C0DBC40E9408730E94AB2583
:105BBA000E2F013021F4A091990BA03009F403C0F3
:105BCA001A930E946410A0912E06AF3F61F11091C2
:105BDA002E06EFEFE0932E061A930E9417180E94E2
:105BEA0024720E94B820E03021F40E94F71EE130AE
:105BFA0009F019C00E94E61EE83119F40E940D73DB
:105C0A0009F001C0ACC41A93EEEFEA930E94AB25E7
:105C1A000E2F013021F4A091990BA03009F403C092
:105C2A001A930E9464105EDC9AC40E9414200E9497
:105C3A009C1FE89421F8E0E0E0931E080E94147388
:105C4A000E9419460E947E6B0E947E6B0E94F2455A
:105C5A00E09132060E94526DE09133060E94526D25
:105C6A000E947E6B0E94DB6C0E94F245E0913F0627
:105C7A000E94526DE0913906F0913A060E94286D11
:105C8A0008950E94D17C0E94B972B0D90E944C42F8
:105C9A00E03049F00E94007330F00E94D27284DC36
:105CAA00E03009F41CDBE091560CF091570C0E948D
:105CBA00036E11F40C94C12E0E9414730E947E6B21
:105CCA00E2E0F0E00E941B73E0913706F09138069B
:105CDA000E94286DE0913B06F0913C060E94286DD7
:105CEA0000E0053010F00C94C12EA7E10A9FF001E4
:105CFA00E15DF94F9F01F901A381AF3FD9F1D901C4
:105D0A001A960E94346D7F936F93FF93EF930E94CC
:105D1A001E73AF91BF918F919F910E940B7A0E943F
:105D2A004E7ADF01CB010E942373D9011C96ED93B1
:105D3A00FC93F90104841584D9011E960E94ED7A18
:105D4A00E015F105B9F0F90104841584A685B78533
:105D5A00F001EA1BFB0BE093AC0BF093AD0BBFDA3F
:105D6A00E13041F4D9011C960E94ED7AD9011E96C0
:105D7A00ED93FC930F5FB5CFB5DB0E94D87C10C4BE
:105D8A000E94D17C0E94B9720E94F87211F40C949C
:105D9A00582F0E944F420E2F0A9307DE003820F038
:105DAA00A091C605A03808F429C00F770A930E946B
:105DBA002A730E9428721E2FA091E20BA03011F4C0
:105DCA001F3F09F416C030E0353098F4ABE03A9F33
:105DDA00F001E452FA4FE081E11749F43A9FF001E9
:105DEA00E252FA4FE081EF5FE093C605232F3F5F4F
:105DFA00EBCF0A930E9408732A9354C0A091E20B36
:105E0A00A03021F4003810F0053808F00AC00F77E6
:105E1A000E94CA711081EFEFEA930E9408730A93F5
:105E2A0068D9A091E20BA03011F0003808F43BC009
:105E3A000F770A930E941718B7DBE030A1F50E948A
:105E4A002D730E944D20EF3F19F00E94D87CA8C301
:105E5A000E94F71EE13039F50E94EB1EE03049F44A
:105E6A000E942D730E94AB25E03011F00E9432731C
:105E7A001AC00E94E61EE83141F40E940D7321F017
:105E8A000E942D730E94AB250EC0A0911E08E02F20
:105E9A000E94A66CAE0FBF1F1C910A930E94087342
:105EAA00EFEFEA9326D9A0912E06AF3FF9F00091C1
:105EBA002E06EFEFE0932E060A930E942A730E94A1
:105ECA0028721E2F0A931A93EEEFEA93EFEFEA93E2
:105EDA0010D91F3F41F4A0919D0BA03021F4A0914D
:105EEA00A00BA03009F002C00E94327320FE0AC043
:105EFA00E89420F8E091E20BE03019F4EAD33BD5BC
:105F0A0001C09AD530E0353080F5ABE03A9FF00118
:105F1A00DF01EA51FA4FE081E03049F0AC51BA4F63
:105F2A000E943873E8EEF3E00E941E7099F4ABE029
:105F3A003A9FF001EA51FA4FE081E23051F43A9F78
:105F4A00F001EC51FA4FDF010E94ED7A0E94036ED4
:105F5A0009F409C0ABE03A9FF001EA51FA4FA0E018
:105F6A00A083689420F83F5FCECFBCDA0E94D87C29
:105F7A0017C30E94206CA33011F40C947731E0917E
:105F8A003908ED3411F00C94A030E0913A08EA3562
:105F9A0011F00C94553024FC83C0E0913B08E05387
:105FAA002E2FE0913C08E0533E2FEDE3F8E00E94EB
:105FBA0052720E944672AC91AB3429F40E943D732E
:105FCA000E94AF5D0E2F0E944672AC91A43529F44F
:105FDA000E943D730E94AF5DAF01E091CD0BE317C4
:105FEA0031F5E0E0E0934F0C0E949372409326084B
:105FFA0050932708A0912F080A1759F0E7E0E09379
:10600A00180800932F0820934E0CE0E0E0932E0826
:10601A000DC0A0914E0C2A1721F0A0912D08A03096
:10602A0009F004C02093180820934E0C35C0A091A3
:10603A002F08A03049F4A091CE0B0E94046CE853BB
:10604A00FF4FE491EA2309F40CC0E7E0E093180853
:10605A0020934E0CE0E0E0932E08E0913808E0939C
:10606A004F0CE0913808A0914F0CEA17A9F440931D
:10607A0026085093270800932F080E949372A09134
:10608A004E0C2A1721F0A0912D08A03009F004C067
:10609A002093180820934E0C273011F40E94487060
:1060AA00E0913A08E93439F4E7E00E94E7720E9485
:1060BA009A72E0932E08E0913A08E23439F4E4E067
:1060CA000E94E7720E949A72E0932E08E0913A08C1
:1060DA00E03519F4E1E0E0931808E0913A08EC346D
:1060EA0049F4E4E0E0931808E0913B08E053EA93AE
:1060FA000E943A15E0913A08E334E9F4A0913B088A
:10610A00A13320F0A0913B08A93308F014C00E94E3
:10611A004073E0912108EA930E945E1AE0913808E0
:10612A00EA93E6E3F7E1FA93EA930E946B6F0E941F
:10613A00007B0E94925FE0913908E03521F4A0913A
:10614A001908A13009F003C00E94CC72A7DAE091C5
:10615A003908EF3459F4E0913A08EE3439F4E09111
:10616A003808EA93E9E3F7E10E944673E0913908B7
:10617A00E33569F5E0913A08EF3349F5A0913B0818
:10618A00A03320F0A0913C08A03308F420C00E945C
:10619A004073E0913C08E0531E2FA0912108A630DD
:1061AA0010F41A3008F013C0103011F40E94A81924
:1061BA00E0913808EA93ECE3F7E1FA93EA930E9454
:1061CA009E6F0E94816F0E94007B0E94925FE09105
:1061DA003908E33411F00C943F31E0913A08EF3377
:1061EA0011F00C943F31E0913C08E03319F4EFEFE1
:1061FA00E0932208A0913B08A033F8F00E94407374
:10620A00A0912108A630C8F4E0912208EF5FE0933C
:10621A002208E0912108EA93E0912208EA930E9479
:10622A00241AA0911E0CB0911F0C109721F4A09172
:10623A002208A03408F001C0E7CFE0912208EA93CF
:10624A000E9417180E944C73EFE3F7E10E9438721C
:10625A000E94466E0E9451730E9456730E944B6EB2
:10626A000E94007B0E9456730E94B36E0E94175FC1
:10627A000E94665FE0913908E434A1F5E0913A089A
:10628A00E43481F514E0E1E0E0933809103538F49C
:10629A000E94AD70E95CF74FE081E03208F41AC061
:1062AA000E94AD70E95CF74FE081E33259F40E9435
:1062BA00AD70E85CF74FE081E053EA930E94175A09
:1062CA001F5F06C00E94AD70E95CF74F0E947D71A6
:1062DA001F5FDCCF0E944C73E2E4F7E10E94387240
:1062EA000E94665F0E94D67C269608951A930A93A6
:1062FA000E945B7111F40C94E931E0E0E0935B0CCD
:10630A00E0911808EF770E2F009318080E9419469B
:10631A000E94DB6C0E94DD6B0E94F245013021F085
:10632A00A0911908A13009F00DC0EAEFF5E00E942A
:10633A00E06CE8D9E4EFF1E0FA93EA930E946B4249
:10634A000E941946073049F40E941420E0E0E093C5
:10635A001B080E9405110E94CD27043031F4E5E4A0
:10636A00F7E10E94E06C0E94C10C083019F40E9407
:10637A005C7357D1053019F40E945C7356DC013006
:10638A0039F40E9469730093190888D90E940E0E85
:10639A00093059F40E9469730E940E0E0A93E1E0D3
:1063AA00EA9329D9E1E0E0935B0C023029F40E94D8
:1063BA005C73E1E0EA93B2DB033011F40E94C93F57
:1063CA00009319080E94C61EA0911908A73011F05F
:1063DA000C949532E091540CF091550C0E94036E86
:1063EA0021F0A0911B08A03009F00AC00E94EB71AD
:1063FA00E091500CA0912306EA1711F00E94CD27D4
:10640A000E944C42E030E9F0E2E00E94C0721A9326
:10641A0068DA1D3409F4BFD81D3399F40E94344553
:10642A0091DAEF3F41F0E3E0E09318080E94C77267
:10643A000E94ED7206C0E7E8E0931808E0E0E093F6
:10644A001B08A0912E08A03031F0E0912E08A091EF
:10645A002D08EA1709F455C0E0912E08E150EA9395
:10646A000E946C18A091340CE1E0EA23E13021F497
:10647A00E0912B06EF7C09F429C0E0E0E0932D08B7
:10648A00E0914E0CE03019F0E09318081EC012E0BB
:10649A00E0912B06EC7009F018E0E091C40BA09192
:1064AA002E08EA1781F0E0912B06E07439F011E02A
:1064BA00EAE2EA93EAE4F7E10E944673E0912B06E6
:1064CA00E07809F019E0109318081BC00E941946D9
:1064DA000E9405110E94DB6C0E94DD6B0E94F2454E
:1064EA00EBE4EA930E948B45E0912E08EA930E941E
:1064FA00B840ECE1F6E00E94E06CE0912E08E093EF
:10650A002D08A0912E08A03021F4A0912D08A030CA
:10651A0009F406C0E0E0E0932D08E7E8E0931808E4
:10652A00A0911908A33011F40E94CB3DA09119083B
:10653A00A13009F438D9A0911908A23009F40ADB6C
:10654A00A0911908A83009F41BDCA0911908A530FC
:10655A0009F497DBA0911908A93009F424D9099103
:10656A00199108950E947473E652F84FA6E0A08329
:10657A000E947473E752F84FAB81A0830E94747330
:10658A00E152F84FAA81A0830E947473E552F84F32
:10659A00A881B981A083B1830E9455710E94744C6D
:1065AA00249608950E947A73A881B981AC91A53086
:1065BA0020F0A881B981E0E0EC9389C0A09113088A
:1065CA00BB27E091120805C0A0911108BB27E091F2
:1065DA001008F0E031960E94EE6F3596DF01E5E093
:1065EA00F0E00E94A67A08951A9310911308E09198
:1065FA001208E117A1F0ABE01A9FF001E652F84F3A
:10660A00E081E13011F0E23011F4E1E04DC0EDB784
:10661A00FEB7FA93EA931F93C5DF1F91E8CFE0E034
:10662A0043C01A930E941420ECEDF5E00E94B36F68
:10663A000E944C6C0E944A6810E0153068F40E946F
:10664A002470AFEFA083ABE01A9FF001EE51FA4F2E
:10665A000E94E6711F5FF1CF10E0153048F4A7E100
:10666A001A9FF001EC5CF94FAFEFA0831F5FF5CFE3
:10667A00E0912B06E37019F00E947C7209F402C0C3
:10668A00689401C0E89421F8EFEFE0932C08E091B8
:10669A00E20BE03029F41DD06ED1E89420F804C052
:1066AA000E9419460E94950E199108951A9310E0B6
:1066BA00153058F40E942470E081AE2FE981EA1760
:1066CA0011F4E12F03C01F5FF3CFEFEF1881229679
:1066DA00089522970E94CF7C00E0053058F40E946A
:1066EA008073A0E00E948673E152FA4FA0E0A08373
:1066FA000F5FF3CF00E00530C0F50E94CA71E08158
:10670A00EF3F89F10E94CA71E0810E943370B9F0AB
:10671A000E94D071DF010E94ED7A0E940170EA178F
:10672A00FB0751F00E94D0710E940170A083B183CF
:10673A000E948B73A1E0A0830E94807312C0ABE019
:10674A000A9FF001EA51FA4FE081E03061F40E94B9
:10675A00CA71AFEFA0830E94D0710E94E6710E94B5
:10676A008B73A1E0A0830F5FC6CF0E94E81D1E2F86
:10677A001F3F11F0E1E001C0E0E0E0935B0C1F3F36
:10678A0011F40C941A3450E000E0053048F40E94E9
:10679A00CA71E0811E1711F451E002C00F5FF5CFF4
:1067AA005030E1F500E00530C8F50E94CA71E08179
:1067BA00EF3F91F50E94CA7110830E94D0710E9426
:1067CA000170A083B183ABE00A9FF001E052FA4F57
:1067DA00A091290C0E948673EF51FA4FFF93EF9311
:1067EA000E942E700E94456FAF91BF91EC930E9458
:1067FA008B73A1E0A0830E948073A1E00E9486733C
:10680A00EC51FA4FFF93EF930E942D64AF91BF9121
:10681A00ED93FC9351E002C00F5FC5CF503029F0D1
:10682A001A930E94EF1D1E2FAACF30E0353010F0C8
:10683A000C946034A7E13A9FF001E15DF94FEE83D1
:10684A00FF8350E000E0053048F5503029F5ABE011
:10685A000A9FF001EF51FA4F20812A930E941718DC
:10686A000E948073E081E13059F42A930E94071F45
:10687A00E13031F4A32FAF5FE0919D0BEA1709F0E5
:10688A000BC0E22FAE81BF811396EC93E02FAE814D
:10689A00BF811596EC9351E00F5FD5CF503049F484
:1068AA00AE81BF811396EFEFEC93AE81BF8115964F
:1068BA00EC933F5FBBCF0E94D67C0C9408370E94B2
:1068CA00D17CAC81BD81EBE4EC93EC81FD81319606
:1068DA00FA93EA930E949173E052FA4FE0810E9480
:1068EA00C46B00E00E949A73EC91E03011F00F5FE4
:1068FA00F9CF0E949A73E0E2EC930F5F0E94A073B3
:10690A000E947A6C0E949173EE51FA4FDF010E9445
:10691A00346D0E94A573EE81ABE0EA9FF001EF515E
:10692A00FA4F10811A930E94171800E00E949A7376
:10693A00EC91E03011F00F5FF9CF0E949A73E8E70B
:10694A00EC930F5F0E949A73E0E2EC930F5F30E0E2
:10695A003A3060F40E94A073EA0FFB1F0F01AAE805
:10696A00BBE00E94AC730F5F3F5FF2CF0E949A7345
:10697A00EC930C944D3764970E94D17C00E010E0B0
:10698A00153040F40E942470E081EF3F09F40F5F54
:10699A001F5FF6CF053021F0A0912C08A03009F432
:1069AA0006C0E0E0E0932C08EA930E94B00F10E0E2
:1069BA00153088F5ABE01A9FF001E152FA4FE081F9
:1069CA00E03039F11A9FF001E352FA4FE081E030EA
:1069DA00B1F01A93FE0135960E94D671ABE01A9F68
:1069EA00F001EF51FA4F30813A930E9417181A9327
:1069FA00FE013596FA93EA930E940B100AC01A9385
:106A0A000E94FB0FABE01A9FF001E152FA4FA0E09F
:106A1A00A0831F5FCDCF053021F4A0912C08A130AF
:106A2A0009F406C0E1E0E0932C08EA930E94B00F53
:106A3A000E94D87C689608950E94CF7CA091E20BB0
:106A4A00A23011F40C94E93830E0343168F40E9431
:106A5A00B3730E94B773DA011296E0E0EC93DA019D
:106A6A00EFEFEC933F5FF1CF0E94E81D0E2F0F3F2F
:106A7A0011F0E1E001C0E0E0E0935B0C0F3FA1F10F
:106A8A000E942E70FA93EA930E94C7171E2F1F3F87
:106A9A0031F1A0911E08E12FEA1B3E2F3431F8F4A0
:106AAA000E94B3730E94B773FA0132960F01E08114
:106ABA00AE2F0E94BD73B0E0EA0FFB1FD001EC932A
:106ACA00FA01A281A43620F0DA011296E3E6EC93E9
:106ADA00DA01AC91AF3F19F4E02FDA01EC930A9393
:106AEA000E94EF1D0E2FCACF0E94491430E03431A4
:106AFA0010F00C9406360E94B3730E94B773FA0121
:106B0A00A381AF3F11F40C9404360E94C2730E9411
:106B1A003B6FE83139F40E94C273EA930E9410175E
:106B2A00E03009F408C00E94C273EA930E94101769
:106B3A00DA011296EC93A0919A0BA07839F4FA0133
:106B4A000280DA011196EC91E01509F458C0DA01D5
:106B5A0013962C91ADE02A9FF001EF5EFC4F0F01D6
:106B6A00DA011296EC91D001EC930E94C273EA9377
:106B7A000E942A20EF3F29F0ADE02A9FF0010E94EF
:106B8A007F6CDA011296EC91E03089F00E94C773AB
:106B9A00DF010E94A16CEC93ADE02A9FF001E25F55
:106BAA00FC4FDF01E091980BEF70EC9313C00E9449
:106BBA00A16CE03021F40E94C773A0E003C00E94D8
:106BCA00C773A8E0A083ADE02A9FF001E25FFC4F03
:106BDA00A7E0A0830E94C273EA930E942A20EF3F93
:106BEA0019F0ECE0E0930F04DA011296EC91DA0165
:106BFA001196EC932A93E1E0EA930E947C463F5F68
:106C0A0076CF0C94E938E7E0E09318080E9452170F
:106C1A00A8950E94AC1BA8950E94041EA895EFEFA8
:106C2A00E093B20BE093890BE093330CE0932E0CC4
:106C3A00E0932E060E94CD73EC7F29F0A8E0B0E025
:106C4A00E0E00E942F7B089524970E94D17C0E9445
:106C5A006541E0E1F7E00E94B36F0E94F3410E94B0
:106C6A008D41E0912108E03061F0ECEEF6E00E94FF
:106C7A00B36F0E94F341E09121080E94D2730E94EF
:106C8A00D6730E948D410E94A81900E00A30A0F430
:106C9A000A930E9446180E94D96EEFE0EA930E9476
:106CAA00CD41E02FA3EAB6E00E94DA730E94816F19
:106CBA000E94DE730F5FEACF0E94A141EEE5F2E087
:106CCA00FA93EA93EFE0EA930E94F3410E94136E6B
:106CDA000E94DE730E94A3410E948D4110E0103190
:106CEA0010F00C9404370E94416DE117E1F5ECE1D4
:106CFA00F7E00E94B36F0E94F3410E94C76C0E94A2
:106D0A00D673E0E0E0931E08A0911E08A03448F56F
:106D1A00E0912108EA93E0911E08EA930E94241A5E
:106D2A000E94466E3097B9F0E0911E08EA930E94DD
:106D3A0017180E94466EFA93EA930E94E4730E941F
:106D4A00F3410E94B36EEAE0EA930E94CD410E94A9
:106D5A004B6E0E94DE73E0911E08EF5FE0931E08FF
:106D6A00D3CF0E94E9730E94AD700E94866F11F022
:106D7A000C940237ECE1F7E00E94B36F0E94F341F2
:106D8A000E94C76C0E94D6730E94ED73E0E30E94D2
:106D9A00926F29F40E94976F0E94AF5D9F010024B1
:106DAA000216030644F50E943D730E94DB5D0E94B1
:106DBA00B66D0E943D730E94F5733A932A930E941E
:106DCA00E4730E94F3410E94F973EAE0EA930E9495
:106DDA00CD41EC81FD816E817F810E94DE730E942C
:106DEA00ED73E1E30E94926F29F40E94976F0E946B
:106DFA00AF5D9F01D4CF0E94E9731F5F70CF0E94DD
:106E0A0066410E94D87C289608950E94D17CAD8163
:106E1A00BE812C910E94FE730E94C76C0E94EC6B8B
:106E2A000E943D6DECE3EA930E948B45EC81EA9364
:106E3A000E94E4452A93ED81EA930E945840EEE3CA
:106E4A00EA930E948B450E9472720E9418720E94F5
:106E5A0078720E940374333409F431E2313320F03A
:106E6A00EC81E05DE31708F407C0E32F0E94E072AB
:106E7A00E853FF4FE4912E273D3311F0313209F4E4
:106E8A0001C0CACF3D3319F4AD81BE812C93E32FE3
:106E9A000E94D87C279608950E94CF7C20E0AF817B
:106EAA00B8855C910E94FE730E94C76C0E94EC6BCD
:106EBA000E943D6DE2E0EA930E94E4455A930E94E3
:106ECA00B8400E9472720E9418720E9478720E94E0
:106EDA000374303310F03A3308F00EC0203009F44E
:106EEA0050E021E0A52FEAE00E94A37AAAE0EA9FF7
:106EFA00F001E30FE0535E2F3B3211F4533608F0F2
:106F0A0001C05F5F3D3211F4513008F401C05150A5
:106F1A00333429F4203009F431E250E020E03D33E3
:106F2A0019F4EE81E51708F005C0AF81B8855C91C8
:106F3A0030E020E03D3311F0313209F401C0B4CF22
:106F4A003D3319F4AF81B8855C93D2C00E94CF7CDF
:106F5A0020E0AF81B8854D915C910E94FE730E943A
:106F6A00C76C0E94EC6B0E943D6DAE81A23051F459
:106F7A00E6E0EA930E94E445FA010E9451730E94F6
:106F8A00974008C0E5E0EA930E94E4455A934A9381
:106F9A000E94A2400E9472720E9418720E94787225
:106FAA000E940374303310F03A3308F01EC02030C8
:106FBA0011F440E050E021E04031E7E25E0734F0AE
:106FCA00DA01E0E1F7E20E94A67AAF01493BEBE081
:106FDA005E0724F0DA010E94DB72AF01DA010E9437
:106FEA0008740E940D74D097AD013B3221F44033EE
:106FFA00E5E75E070CF002C04F5F5F4F3D3221F4B8
:10700A000024041605060CF002C0415050403334E7
:10701A0031F4203009F431E240E050E020E03D3321
:10702A0011F0313209F401C09ACF3D3321F4AF8116
:10703A00B8854D935C935CC00E94CF7C0E94FE731E
:10704A0020E050E04FEF0E94C76C0E94EC6B0E9458
:10705A001B73EF81F885FA93EA93E885EA930E9415
:10706A00B845E52FE10FF0E00E9418720E9478728D
:10707A000E940374303310F03A3308F021C03053C1
:10708A00431729F04F3F09F05F5F20E005C0A22FA8
:10709A00AF5FEA2FE3702E2FE52FAF81B8850E94EC
:1070AA0012740F01E32FA4EAB7E00E94DA73AE0F5D
:1070BA00BF1FE22F0E941274E491D001EC93432F78
:1070CA003B3219F4EE815E1708F002C05F5F4FEFA2
:1070DA003D3211F4513008F402C051504FEFEE81A5
:1070EA005E1720F4313211F03D3309F401C0ABCF01
:1070FA00E32F0E94D67C299608951A930A93A091A9
:10710A009A0BECEDEA231E2F00E00D3040F40E94AA
:10711A0016740E941A74E11711F00F5FF6CF0E94DD
:10712A001674EA0FFB1F0E94FC7A0E94E06CE02FA3
:10713A0049C4AAE9BBE00E942C6DAE0FBF1FEC91B7
:10714A00E17011F4E3E701C0E9E4EA930E948B4598
:10715A00219608950E94CF7C0E94FE730E94C76CFC
:10716A000E94EC6B0E941B73C8DF5E2F0E94727232
:10717A000E9418720E9478720E9403743D3211F0C4
:10718A00363311F4503009F401C051503B3211F03A
:10719A00333311F45C3008F001C05F5FA0919A0BA1
:1071AA00E1E0EA232E2FE52FA4E2B2E00E94DA738F
:1071BA000E941A74E20FE0939A0B3D3311F03132B8
:1071CA0009F401C0CBCFE32F0E94D67C26960895FE
:1071DA000E94D17C0E94FE730E94C76C0E94EC6BD5
:1071EA000E941B73AAE9BBE0EC810E94376FEC9105
:1071FA00E17019F4E4E2F7E002C0E8E2F7E0FA939A
:10720A00EA930E94A1450E9472720E9418720E941B
:10721A0078720E940374303310F03A3308F010C0C9
:10722A00AAE9BBE0EC810E9412740F01AAE9BBE053
:10723A00EC810E94376FAC91E1E0EA27D001EC9330
:10724A003D3311F0313209F401C0C6CFE32F0E9459
:10725A00D87C259608950E94D46BE1E0EA930E94B7
:10726A00AD0D0E947E6B0E947E6B0E94F2450E94C9
:10727A00B36EEAE0EA93E0DEE13209F46AC40E94FE
:10728A007E6B0E947E6B0E94156DE0EAF0E00E9420
:10729A00E06CE5E9FBE00E94B36F58DEE13209F4E5
:1072AA0058C40E947E6B0E947E6B0E94156DEAE1B3
:1072BA00F2E00E94E06CE091970BEF5F0E2FEDB7C2
:1072CA00FEB7FA93EA930F93EAE0EA93E5DD0F91AA
:1072DA00E13209F43EC400240216030624F4E02F26
:1072EA00E150E093970B0E947E6B0E947E6B0E9496
:1072FA00156DECE2F7E00E94E06CECEAFBE00E941C
:10730A001F7409F426C40E947E6B0E947E6B0E9441
:10731A00156DE0E3F7E00E94E06CEEEAFBE00E9404
:10732A001F7409F416C40E947E6B0E947E6B0E9431
:10733A00156DE4E3F7E00E94E06CE9E9FBE0FA93FB
:10734A00EA93E3E60E94287409F403C40E947E6B60
:10735A000E947E6B0E94156DEAE3F7E00E94E06CE2
:10736A00F9DEE13209F4F5C310E0133010F00C94A1
:10737A00733A0E947E6B0E947E6B0E94156DE12F0C
:10738A000E949E72EEE3F7E00E94E06C0E942D7468
:10739A000E94F245ADE9BBE00E94AD700E947A6C92
:1073AA00E0E10E94287409F4D4C3E9E0F0E00E9405
:1073BA00AA6B0E94F245A0EABBE00E94AD700E944F
:1073CA007A6CE0E10E94287409F4C3C30E947E6BC0
:1073DA000E947E6B0E94156DE12F0E949E720E9490
:1073EA0031741A93F5DEE13209F4B3C30E942D74A5
:1073FA000E94357451F40E9465710E943F74E2E064
:10740A000E94437409F4A5C309C00E9465710E94D1
:10741A003F74E0E00E94437409F49BC30E947E6BB0
:10742A000E947E6B0E94156DE12F0E949E72EAE413
:10743A00F7E00E94E06C0E942D740E94F245A9EACE
:10744A00BBE0EE27A10FBE1F2C913327EDB7FEB785
:10745A003197FA93EA933F932F93E0E0EA9376DD2C
:10746A002F913F91E13209F474C3A9EABBE00E946B
:10747A00AD70EA0FFB1F2083123070F50E947E6BFD
:10748A000E947E6B0E94156DE12F0E949E72E2E5BA
:10749A00F7E00E94E06C0E942D740E94F245A0EB76
:1074AA00BBE0EE27A10FBE1F2C913327EDB7FEB725
:1074BA003197FA93EA933F932F93E0E0EA9346DDFC
:1074CA002F913F91E13209F444C3A0EBBBE00E9443
:1074DA00AD70EA0FFB1F20831F5F47CF3AC30E949C
:1074EA00D17C10E01A930E94F4720E9448740E94A0
:1074FA007E6B0E94F2450E944D6D0E9431740E947B
:10750A00D36C0E94406F0E94286D0E947E6B0E947D
:10751A00DB6C0E94F2450E944E6F0E94396DE7E0D3
:10752A00F0E0FA93EA930E94DB6C0E94F245E09144
:10753A00AE0BF091AF0B0E940B7A0E94396D0E943C
:10754A007E6BE2E0F0E00E943D6DEAE5F7E00E9422
:10755A00E06CE091970BEF5FEA930E94B840E7E096
:10756A00F0E00E94CC6C0E94F245C7DD0E94196DC2
:10757A00E091990BE03029F0E091990BEA930E948F
:10758A00B84000E0033010F00C94093B0E947E6B77
:10759A00E02FED5FF0E00E943D6D0E949271EA9348
:1075AA000E94B840EBE2EA930E948B450E949971CF
:1075BA00EA930E94B8400E94196D0E94A07159F482
:1075CA000E94A8710E942F6D0E94346D0E944C7413
:1075DA00EEE5F7E00AC00E94A8710E942F6D0E9492
:1075EA00ED7A0E94286DE0E6F7E0FA93EA930E94AA
:1075FA00A1450E94196D0E94B271EA930E94BE4091
:10760A000E9450740F5FBECF0E944F423E2F3B3202
:10761A0011F4103408F001C01F5F3D3211F411302B
:10762A0008F401C011503D3439F41A930E94171816
:10763A0012DE1A930E943718313209F053CF89C2E9
:10764A000E94D17C10E00E941946012F0E947E6B95
:10765A000E947E6B0E94F245E2E6F7E00E94E06C2F
:10766A0031E03C3018F51038F8F40E947E6B0E9425
:10767A00046C0E943D6D1A930E946C180E944D6D15
:10768A000E94196DA091340CE3E00E945374A091FA
:10769A00350CE7E00E945374E0912B06EA93E8E088
:1076AA00EA930E94584013953F5FDBCF0E94C10CBA
:1076BA000E944F423E2F3D3411F00C94A33B0E948E
:1076CA00C26C0E94AD0D102F1038C0F51A930E949B
:1076DA006C180E947E6B0E947E6B0E94156DE6E715
:1076EA00F7E00E94E06C0E944D6D0E9431740E9486
:1076FA00546D0E94F245EAE7F7E00E94E06CE4E389
:10770A00FCE0FA93EA93E3E00E94287409F421C2A8
:10771A000E94546D0E94156DE0E8F7E00E94E06C4B
:10772A00E5E3FCE0FA93EA93E7E00E94287409F49F
:10773A0010C21A930E949E181F5FC6CF313211F0F1
:10774A00103808F001C07FCF04C20E94D46B0E9497
:10775A0048740E947E6B0E94F245E6E8F7E00E94B8
:10776A00E06C10E01530F0F41A930E94AA180E94F7
:10777A007E6B0E94296E0E944D6D0E943174E091C9
:10778A002F0C0E945874E091320C0E945874E091B8
:10779A00300C0E945874E091310CEA930E94BE406A
:1077AA001F5FE0CF0E944F420E2F0D3411F00C9450
:1077BA001D3C0E94C26C0E94AD0D10E01530C0F550
:1077CA001A930E94AA180E947E6B0E947E6B0E94E6
:1077DA00156DEAE9F7E00E94E06C0E944D6D0E9487
:1077EA00317430E03430F8F40E94546D0E94156D03
:1077FA000E94046C0E94F979E65FF74F0E94FC7AB6
:10780A000E94E06C0E94046C0E94F979E65FF74FCF
:10781A000E945C74FD013596E4910E94287409F473
:10782A0098C13F5FDFCF1A930E94CA181F5FC6CF65
:10783A0090C11A930A930E941946E1E0EA930E94C2
:10784A00AD0D00E0083210F00C94E73C0E948D0C5C
:10785A000E947E6B0E947E6B0E94F2450E94EC6B36
:10786A000E945F740E94FC7A31960E94E06C0E942A
:10787A00196D0E94EC6B0E945F743496E491E038B3
:10788A00A9F40E94416D1E2FEDB7FEB7FA93EA9351
:10789A001F93E0E1EA9300DB1F91E13209F492C001
:1078AA00E12FA9E0B0E00E942F7B88C0E238A9F45A
:1078BA000E94B86F1E2FEDB7FEB7FA93EA931F9393
:1078CA00E0E1EA93E9DA1F91E13209F47BC0E12FA2
:1078DA00AAE0B0E00E942F7B71C0E138E1F40E9477
:1078EA00CD731E2FEDB7FEB7FA93EA931F93E3E029
:1078FA00EA93D2DA1F91E13209F464C00E948D0C36
:10790A000E94CD73E11731F0E12FA8E0B0E00E94A8
:10791A002F7BFFCF53C0E03069F40E94EC6B0E94CA
:10792A005F7432960E94E46CE1E00E94287409F4C4
:10793A0049C044C0E13069F40E94EC6B0E945F7454
:10794A000E945C74FD013596E4910E942874D1F17D
:10795A0035C0E23061F40E94EC6B0E945F7432968B
:10796A000E94E46CEFE00E94437461F127C0E330A7
:10797A0071F40E94EC6B0E945F740E945C74FD01BA
:10798A003596E491EA9341DAE132E1F017C0E43046
:10799A00A9F40E94EC6B0E945F7432960E94FC7AF2
:1079AA00E0935C0CF0935D0C0E9418720E945F7465
:1079BA003596E491EA9340DBE13221F00E945517B3
:1079CA000F5F40CF099119910895E8810E949E7234
:1079DA00E6E5F7E10E94E06C0C9439401A930E94A4
:1079EA00C26C0E94AD0D10E0133010F00C944B3DA8
:1079FA000E947E6B0E947E6B0E94156D1A93E5DFD2
:107A0A00ECE0F0E00E94AA6B0E94F2451A9391DB27
:107A1A000E942D740E94357449F40E9465710E9477
:107A2A003F74E2E00E94437489F108C00E946571C4
:107A3A000E943F74E0E00E94437441F1123020F545
:107A4A000E947E6B0E947E6B0E94156D1A93BDDFA9
:107A5A00EEE9F7E00E94E06CECE0F0E00E94AA6B2D
:107A6A000E94F2450E945074EAE0F0E00E94AA6B7C
:107A7A000E94F245A0EBBBE00E94AD700E947A6CB6
:107A8A00E3E60E94287411F01F5FAECF19910895A2
:107A9A000E94D17C10E01A930E94F4720E944874EA
:107AAA000E947E6B0E94F2450E944D6D0E943174C5
:107ABA000E94D36C21E000E0033080F5E3E0F0E0BF
:107ACA000E941B6C0E943D6D0A937FDF0E94A07189
:107ADA0049F40E94A8710E942F6D0E94346D0E9481
:107AEA004C7408C00E94A8710E942F6D0E94ED7A02
:107AFA000E94286D0A931DDB2F5F023068F4E7E0CD
:107B0A00F0E00E941B6C0E943D6D0E94AB710E94C6
:107B1A00526D0E9450742F5F0F5FCECF0E944F426A
:107B2A003E2F3B3211F4103408F001C01F5F3D3282
:107B3A0011F4113008F401C011503D3439F41A938C
:107B4A000E9417184BDF1A930E943718313209F036
:107B5A00A2CF0E94D87C249608950E94C26C0E94EB
:107B6A00AD0D0E947E6B0E947E6B0E94F245ECEE88
:107B7A00F6E00E94E06CE1E0E0932108E1E2F8E03F
:107B8A00FA93EA93E5E0EA9387D9089522970E9447
:107B9A00CF7C0E944F420E2FE0911B08E03011F07B
:107BAA000C94773F0132D1F4ECECF7E0A0913A0C57
:107BBA00B0913B0CEA17FB0761F4E7E0E093180881
:107BCA00EAE2EA93E9E5F7E10E94B36F0E949F5F58
:107BDA00A9C0E0E0E093C0050E9464740D3331F45B
:107BEA00E091C005F0E00E940A6C04910D3441F462
:107BFA00EAE2EA93ECE5F7E10E94B36F0E949F5F25
:107C0A00063449F4E4EFF7E0E0933A0CF0933B0CC6
:107C1A00E0E0E093C005003311F00B3229F4E09163
:107C2A00C005EF5FE093C0050D3229F4E091C0056D
:107C3A00E150E093C005013329F48FDFED3311F4ED
:107C4A000E946B74033329F488DFED3311F40E9428
:107C5A002936063329F4E0E0E09321080E94293608
:107C6A00043329F4E0E0E09321080E946B74A091A8
:107C7A002308A13010F40C94113F023301F56DDF93
:107C8A00ED33E9F40E947874D1F4E0912108EA9383
:107C9A000E945E1A30E0303190F40E94046C0E9417
:107CAA00866F59F4E32FE05DEA93EFE5F7E10E946E
:107CBA008B6FE0E3EA930E94C15F3F5FECCF05332D
:107CCA0031F5E0E0E09321080E94787401F511E0B3
:107CDA001630E8F41A930E945E1A30E03031A8F4A4
:107CEA000E94046C0E94866F71F4E32FE05DEA93B0
:107CFA00EFE5F7E1FA93EA93E12FE05DEA93E0E337
:107D0A00EA930E94C15F3F5FE9CF1F5FE1CF013471
:107D1A0069F4EAE2EA93E2E6F7E10E944673E1E0F7
:107D2A00E09318080E94D67C289608950A3409F42C
:107D3A00AFDE073311F00C94113F0E94C26C0E940F
:107D4A00EF0CE1E0E0931C08E0E0F0E0E0931408B7
:107D5A00F0931508EFE2F6E00E94B36FE3E7F0E074
:107D6A000E94676F0E942D64EE83FF830E948174D4
:107D7A00E8E2F0E00E941E70B9F00E9448110E94E9
:107D8A002D64EE83FF83A091190CA03021F00E948C
:107D9A00E332E03009F408C00E947473E652F84FE7
:107DAA00AEE0A0830E9455710E9486740E946B42C5
:107DBA0040E050E00E94E120E03868F00E94E120B3
:107DCA00EF573E2F313010F0313108F004C0E32F65
:107DDA000E947C70AF015A934A930E94A01E40935E
:107DEA001408509315080091DB05E0E0E093DB05E9
:107DFA00013211F00B3209F401C0B8CF0B3221F471
:107E0A00E1E0EA930E94EF0C013209F0A3CFE0E02F
:107E1A00E0931C08E093DB05A0912308A23011F03F
:107E2A000C94703F093309F404DD053409F48DDC40
:107E3A00083309F454DB023409F402DC0334B1F5E3
:107E4A001091390C0E94194600E0E091380CE117B4
:107E5A0011F00C3008F01DC00E947E6B0E94EC6B82
:107E6A000E943D6D1A930E94F61D1A937CD10E94BE
:107E7A00196DE091290C0E945874E0912C0C0E9413
:107E8A0058740E942E700E94286D0E9414700395E7
:107E9A00DCCF0E94C10C0E944F420E2F013221F00A
:107EAA00E091380CE11709F401C0CCCF043499F4FD
:107EBA000E94787481F4A091D30BA03021F4A09190
:107ECA00D10BA03031F00E948B740E947E6B0E940D
:107EDA00A54E0E943F1CE0911B08E03011F40E945D
:107EEA004A0D49C0E130D1F4A0912008AB3010F41A
:107EFA00013209F405C00E94EA140E94C10C0DC0A7
:107F0A00E0E0E0931E080E948F740E944673E0E04E
:107F1A000E949474E2E0E0931B082DC0E23059F508
:107F2A00013269F4E0E0E0931B080E941946EAE294
:107F3A00EA93ECE5F7E10E9446730E944A0D0B3280
:107F4A0011F00D3359F40E948F74FA93EA93E1E326
:107F5A00EA930E949F5FE1E00E9494740D3259F403
:107F6A000E948F74FA93EA93E2E3EA930E949F5F76
:107F7A00E2E00E949474A0911808A33009F409CE93
:107F8A000E94D67C0C94BE441A93E3E0E09319084D
:107F9A000E9419460E947E6B0E947E6B0E94F245E7
:107FAA00E8E5F2E00E94E06C0E947E6B0E94DB6CC6
:107FBA000E94F245E3E1F6E00E94B36FE0E1F0E0EF
:107FCA000E94676F10E0E091C90B1E1700F50E942E
:107FDA00416DE117D1F0E12FE05DEA93E8E6F7E1C0
:107FEA00FA93EA93E0E3EA93E0E00E94926F49F49D
:107FFA000E94AD70ED5EF94FA1E0A083E12FE05D34
:10800A0001C0EEE2EA930E948B451F5FDCCF0E941B
:10801A006474E0E0E093C005E0931B080E944A0DF7
:10802A0053C2E881E03021F4E0E3F8E00E94997459
:10803A00A881A13021F4EAE2F8E00E949974A881AB
:10804A00A23021F4E6E3F8E00E949974A881A330F3
:10805A0021F4E4E4F8E00E949974A881A43021F4A0
:10806A00EAE4F8E00E949974219608951A930A9313
:10807A00E0E0E0937D05E0937E0510E0143190F492
:10808A0000E0033068F4A3E01A9FF001EC57FA4FBE
:10809A00DF01EE27A00FBE1FE0E2EC930F5FF1CFE6
:1080AA001F5FECCFEDC31A9311E0E981E11780F06D
:1080BA000E94AD70E853FF4FE491AA81EA2319F0B8
:1080CA00E12FE05D01C0E0E2EA9320D51F5FEDCF2A
:1080DA0030C11A9311E0E981E11778F00E94AD707E
:1080EA00E853FF4FE491AA81EA2311F0E1E301C0CA
:1080FA00E0E3EA930BD51F5FEECF1BC12A97A0914D
:10810A001B0CA13038F0EA85FB856C857D850E94C1
:10811A004C7407C00E949E740E94A2740E949E74AE
:10812A00FDD427C12A970E949E740E94AB740E94B4
:10813A00B4740E949E74F2D41CC12A970E949E7441
:10814A000E94C7740E94CE74E9D420C12A970E9463
:10815A009E74E7E8F7E10E94D3740E9451730E946B
:10816A00CE74DCD413C12A970E949E74EAE8F7E120
:10817A0005C02A970E949E74EEE8F7E1FA93EA9303
:10818A00EE850E94C46B0E949E74C8D42B960895F3
:10819A000E94D17C10E0E1E3E0933709E89431F8DA
:1081AA00EA930E944C5FE2E9F7E10E94387200E02C
:1081BA00E09182050E17E0F40E94EC6BEC57FA4F3F
:1081CA00E081E03258F4E3E2EA930E947F5E0E9483
:1081DA00EC6BEC57FA4FE081E05D05C00E94EC6B56
:1081EA00EC57FA4FE081EA930E947F5E0F5FE0CF7F
:1081FA000E94D8749F010E9452143A932A93E8EC81
:10820A00F0E0FA93EA930E9438640E2FA0E031FC62
:10821A00A1E0A03011F4003009F001C0ECCF31FE2A
:10822A0009C0E0E0E0938205E89431F8E1E00E94B9
:10823A00D87CF8C41F5F123008F4ADCFE0E0E093B9
:10824A0082050E94D87CEEC4E0918105E03021F4D9
:10825A00E881EA930E94175AA0918105A13069F436
:10826A00A0E09299A1E0A13021F4A8950E94576E4E
:10827A00F7CFE881EA930E94C85CA0918105A230F9
:10828A00F1F4E0918205F0E0EC57FA4FA881A0835F
:10829A00E0918205EF5FE0938205E0918305EF5F4D
:1082AA00E0938305A03218F4EF5FE0938305A09171
:1082BA008305A83320F06CDFE0E0E09383052CC44B
:1082CA0008950E94E9730E94E97322D0EBE1EA93D0
:1082DA00BBDFE9E6EA93B8DFA0918105A13061F43A
:1082EA00E8ECF0E00E94BF6DE0919A00E069E0934B
:1082FA009A00E9E1E0939900A0918105A23021F466
:10830A0047DFE0E0E0938305E0E0E093810508952C
:10831A00EDE0EA9399DFEAE0EA9396DF08951A938B
:10832A0010E0E9811E1728F4EA81EA938DDF1F5FC6
:10833A00F8CF188123960895EDE201C0EDE3EA93A0
:10834A00E8E2EA93ECDFE4DF08952A97A0911B0C98
:10835A00A13038F00E949E740E94AB740E94B474DB
:10836A0004C00E949E740E94A274FE010E94B36F10
:10837A000FD02E9608952A970E949E740E94C77461
:10838A000E94DC74FE010E94B36F02D02C960895FD
:10839A001A930A9310E0EA81E03011F408E201C06E
:1083AA000A81AB81BC81EE27A10FBE1FAC91A03020
:1083BA0011F0101708F007C0AB81BC810E94E1746C
:1083CA000E94E674EECFEA81E03039F0EA811E17A6
:1083DA0020F4E0E20E94E674F9CF27C01A930A93C8
:1083EA0010E0EA81E03011F408E201C00A81E12FCD
:1083FA00AB81BC810E941274E491E03011F0101735
:10840A0008F009C0E12FAB81BC810E941274E4918B
:10841A000E94E674ECCFEA81E03039F0EA811E1757
:10842A0020F4E0E20E94E674F9CF198108812596CA
:10843A000895E091C405A091C305EA17B1F00E941E
:10844A00EB740E942F6DEC91E093C6050E94EB74C9
:10845A000E94C770E181E093C505A091C4050E94FE
:10846A00F174E093C405E1E00895E0E008950E9404
:10847A00F674A981A0830E94F6743196A881A0831C
:10848A00A091C3050E94F174E093C3053DC3E09136
:10849A00DB0508951A93E091DB05E03059F40E9458
:1084AA0052140E945B7121F4A091DB05A03009F0FF
:1084BA0001C0F5CF1091DB05E0E0E093DB050E94F7
:1084CA005B7109F011E2E12F199108950E94D17CA4
:1084DA000E942D648F010E945214EC81FD81E00FED
:1084EA00F11FFF93EF930E942D64AF91BF91AE1BD2
:1084FA00BF0B9D010024021603061CF40E945B7147
:10850A0009F001C0E8CFE0E00E94D87C26960895E1
:10851A001A93E9810E94C4710E94FC74E05FFC4FC7
:10852A00108117FF05C0E12F0E940375A0E0A08308
:10853A0016FF05C0E12F0E940A75A0E0A083E98119
:10854A00ADE0EA9FF001E05FFC4F0E94FC74E15F3E
:10855A00FC4FA0E0A0831881D7C20E94D17C30E0F2
:10856A00EE81ADE0EA9FF001E05FFC4F108116FF5B
:10857A0017C0E12FEF730E2F0E94117511F03A30D8
:10858A0008F009C00E941975DF010E94046C0E945C
:10859A001F753F5FF1CF0E9419750E940D74EC930D
:1085AA0017FF17C0E12FEF730E2F0E94117511F0FC
:1085BA00343108F009C00E942575DF010E94046C5D
:1085CA000E941F753F5FF1CF0E9425750E940D74AE
:1085DA00EC930E94D87C41C2E881F9810E94E46C44
:1085EA00EA81FB8132960E94E46CEC81FD8134962B
:1085FA000E94E46CEE81FF8136960E94E46CE88565
:10860A00F9853896E491EA93E985FA8539960E94C4
:10861A00E96B01D079C2A0970E94CF7CEDA5FEA597
:10862A00A9A9BAA9EA0FFB1FAF01E5E0F3E0EE83BF
:10863A00FF8310E01431C0F5AE81BF81AC91A03048
:10864A0049F1EE81FF81A381B481EFA5F8A9EA1768
:10865A00FB0701F5EE81FF81A181B281E9A9FAA99F
:10866A00AE17BF07BCF0EE81FF81A181B2814A1724
:10867A005B0784F00E942B75AE0FBF1FE9A9FAA908
:10868A00AE17BF073CF00E942B75AE0FBF1F4A17EB
:10869A005B070CF402C01A933BDFEE81FF813D9623
:1086AA00EE83FF831F5FC6CFE5E0F3E0EE83FF832F
:1086BA0010E0143110F00C940544AE81BF81EC91A6
:1086CA00E03011F00C94FE43EAA5EC93E9A9FAA96B
:1086DA00AE81BF811196ED93FC93EFA5F8A9AE8107
:1086EA00BF811396ED93FC93EDA5FEA5AE81BF81E4
:1086FA001596ED93FC93EBA5AE81BF811796EC938B
:10870A00E0910904A0910F04EA27AE81BF8118966F
:10871A00EC93E0911004AE81BF811996EC93E0913D
:10872A001104AE81BF811A96EC93AE81BF811B966C
:10873A000E94876C1C96E0E0EC93E887E8A5F9A50F
:10874A00309741F00E9436750E943B75E4E1EA9346
:10875A000E94A968EEA1FFA1309751F00E943675D8
:10876A00E8A5F9A5FA93EA93E4E1EA930E949568E9
:10877A00E0E0EC8F0E9436750E9480683E2F3B3005
:10878A00C8F000E00E942575E081E03011F0053064
:10879A0008F002C00F5FF6CF0E942575E081E03035
:1087AA0049F40E9425750E944075E058AE81BF8148
:1087BA001B96EC93E0E0EA8B3130C8F000E00E94AF
:1087CA001975E081E03011F0043108F002C00F5F42
:1087DA00F6CF0E941975E081E03049F40E941975BC
:1087EA000E944075E05CAE81BF811B96EC93E12F3D
:1087FA0008C0EE81FF813D96EE83FF831F5F59CF4C
:10880A00EFEF0E94D67CE39608951A930A930E948A
:10881A004B753097A9F1E0916205E03061F50E944D
:10882A004B75049000926205E0916205E03031F4E4
:10883A00E0E0F0E00E949974E0E01AC00E945075EE
:10884A000E944B750E94FC7AF595E7958F01D80135
:10885A00E0E0F1E00E94747AE0938700D801E0E05A
:10886A00F1E00E94A67AE09386000E945075E0E447
:10887A00E0938B0005C0E0916205E150E093620548
:10888A000991199108950E94D17C00E025E033E016
:10889A0010E01431B8F5D901EC91E03079F1119674
:1088AA000E94ED7A0E94587524F5D90113960E9408
:1088BA00ED7AAC81BD81EA17FB07DCF4F90101808E
:1088CA001280D90115960E94ED7AE00DF11DAE8154
:1088DA00BF81AE17BF076CF4F90103801480D90178
:1088EA001796EC910E946171AC81BD81AE17BF07EA
:1088FA000CF004C0E12FEF5F0E2F04C0235F3F4F3F
:10890A001F5FC7CF003049F0E0916305E01721F0FF
:10891A00A0916305A03009F401C022C0A0916405AA
:10892A00A53079F40A93E1E0EA93A1DD00936305A7
:10893A0000936505D901EC91E0936605E3E0E093C5
:10894A006105A0916405AE3119F4E4E0E093610594
:10895A00A0916105A33018F0E5E0E093680507C02F
:10896A00E0E0E0936405E09361050E945D750E9472
:10897A00D87C28960895E0916305E03091F0A091A3
:10898A006405A93220F4EA93E2E0EA9370DDA0914B
:10899A006405AD3330F0E0916305EA93E4E0EA93CD
:1089AA0066DDE0E0E0936105E09364050E945D7591
:1089BA00E0E0E0936305E0936705089535D156DB5F
:1089CA000895EA81E0937F05E881E0938005E091CC
:1089DA000A04E061E0930A0425C10E94CF7CA091B9
:1089EA007F05A43120F4A0918005A33008F033C09C
:1089FA00E0917F05F0E0ACE0B0E00E94497A8F0197
:108A0A00E0918005F0E0A4E1B0E00E94497A9F017C
:108A1A000E946375ECE0F0E00E946875F0E00E9445
:108A2A00F7790E94886BEE81E030A9F0E0917F052A
:108A3A00A3E0EA9FF001EC57FA4FDF01E0918005CD
:108A4A000E94376F4C9155270E9463754A93EFE055
:108A5A00EA930E9452670E94D67C27960895E09175
:108A6A000A04E07141F0E2E0EA93B7DFE0910A0418
:108A7A00EF7EE0930A0408950E946D75AF3EE0E030
:108A8A00BE0744F4A0910203B0910303AF33E1E0BF
:108A9A00BE070CF039C00E9472750E94496F0E948D
:108AAA005267A0915D05B0915E05549734F4A09188
:108ABA005F05B091600513970CF012C0E0915D0557
:108ACA00F0915E05A3E0B0E00E94217AEC57FA4FDC
:108ADA00A0915F05B0916005EA0FFB1FA981A083F1
:108AEA00E0910D04ACE0EA9FF0010E946D750E94CE
:108AFA0012740E947F75E0915D05F0915E053196D2
:108B0A00E0935D05F0935E0522960895E881EA9365
:108B1A00E0911004EA93B0DF219608951A9310E0C9
:108B2A000E948475E03031F00E948475EA93EEDF8A
:108B3A001F5FF6CF1881E1C31A930A9300E010E091
:108B4A000E948775E03021F00832E0E01E070CF041
:108B5A0007C00E948775EA93D9DF0F5F1F4FF0CFD6
:108B6A00198108815FC01A930A9300E010E0F801A6
:108B7A00AB81BC810E948E7521F0EA810E949375B7
:108B8A000CF009C0F801AB81BC810E949875BEDF68
:108B9A000F5F1F4FECCF1981088110C30E94D17C4F
:108BAA000E946D75EFEEF0E0EA1BFB0B31978F0127
:108BBA000E949D750E9463750E94A57533C00E942C
:108BCA00D17CAC810E94AC750E2F11270E949D7535
:108BDA000E9463750E94A575F1C2EA81FB81E09348
:108BEA005D05F0935E05E881F981E0935F05F093F6
:108BFA006005AA81BB81ECE0F0E00E94497A0E94FC
:108C0A007F75A881B981E4E1F0E00E94497A06C043
:108C1A00EA81FB810E947F75E881F981E093020372
:108C2A00F0930303249608950E94B475143120F436
:108C3A001A936EDC1F5FFACF0E947E6B0E947E6BD6
:108C4A000E94836BEFE3F1E00E94886B10E015301D
:108C5A0048F4A5E11A9FF001E051FB4FA0E0A08380
:108C6A001F5FF5CF10E0143148F4ABE01A9FF00112
:108C7A00EC5EFB4FA0E0A0831F5FF5CFE0910A04F2
:108C8A00EF7EE0930A04EDC30E94B475143100F537
:108C9A00ADE01A9FF001BF01E85FFC4FDF010E94BF
:108CAA00ED7A0F01DF01EB81FC81AE17BF075CF0A3
:108CBA00E981FA81E015F10534F0FB01E05FFC4F30
:108CCA00E081E03009F402C01A9322DC1F5FDECF94
:108CDA000E947E6BED81FE81FA93EA930E94836B78
:108CEA00A985BA850E94BC750E94886B66C2A29744
:108CFA000E94CF7CE9A50E94C4718F01D8011B96FE
:108D0A00EC91E03009F415C2D8011B96EC91E9A365
:108D1A00E07859F0FE013696FA93EA93EBA10E94A5
:108D2A000375FA93EA930E946A68E9A1E07459F01C
:108D3A00FE013696FA93EA93EBA10E940A75FA931A
:108D4A00EA930E946A68FE013696FA93EA930E94B1
:108D5A008068E8A3E0910D04EB8FE0910E04EA8F9E
:108D6A000E940D6ED80111962D913C91D80113964F
:108D7A004D915C91D80115960E94ED7AEEA3FFA35E
:108D8A00D8011796EC91F0E0ECA3FDA3D801189650
:108D9A00EC91EC8FE0910E04A0E10E94C175EAA368
:108DAA00FBA30E94C5750E943B750E943B75ECA10E
:108DBA00EA930E94D064D8011996EC91EC8FE030C6
:108DCA0011F4E8E0EC8F0E94C5750E94CA755A93A7
:108DDA004A930E94D1750E94D5750E94DC750E9443
:108DEA00DF750E94C5753A932A930E94DF75EEA13A
:108DFA00FFA10E94E6755A934A930E94CA750E947F
:108E0A00DF75A8A5A130B1F43A932A93FA013196F5
:108E1A000E94DC75FA013196FA93EA930E94D175A1
:108E2A00F90131960E94EB75F9013196FA93EA93AA
:108E3A000E94DF75A8A5A230F1F40E94D57531977A
:108E4A000E94DC75EAA5FBA5E40FF51F3197FA939A
:108E5A00EA930E94D175EEA1FFA1E20FF31F3197A9
:108E6A000E94EB75EAA5FBA5E20FF31F3197FA936F
:108E7A00EA930E94DF75E8A5E03011F40C946E487D
:108E8A00D8011996EC91EC8FE0910D04ACE00E94A8
:108E9A00F0750E94747AED8FA8A1EA1710F40C9469
:108EAA009D47E1E0E0930E04E03021F0ECA1FDA142
:108EBA00B5970CF402C00E94F675AAA1BBA1ECA159
:108ECA00FDA1EA1BFB0BDF010E94B070EAA3FBA322
:108EDA00ABA1AA231AF4E0E0EAA3EBA3A8A10E949B
:108EEA00AC75AEA1BFA1F0E00E94FE75EE8FA8A5F9
:108EFA00A13021F40E9401760E940476A8A5A2302E
:108F0A0031F40E9401760E94E6750E941076E0E034
:108F1A00E9A30E941676AE0FBF1FEC91E03039F03C
:108F2A000E9416760E9498750E941B76F2CFD1C0D5
:108F3A00E1E0E0930E04E03031F0ECA1FDA1E7346A
:108F4A00A0E0FA070CF402C00E94F675E8A1EF8FC0
:108F5A00EAA1FBA1EE0FFF1FACA1BDA1AE1BBF0B87
:108F6A00E3E0F0E00E94747AEAA3FBA3ABA1AA2390
:108F7A0022F4E1E0F0E0EAA3FBA3EF8DE150EF8FEA
:108F8A00EF8DF0E0DE011696AE0FBF1FAC91A03256
:108F9A0019F0AF8DA13008F404C0EF8DE150EF8FC6
:108FAA00EFCFAF8D0E94AC75AE2FEEA1FFA1B0E05E
:108FBA00AE17BF0714F7EF8DE03011F4ED8DEF8F88
:108FCA00AF8DECE00E94F0750E94FE75EE8FA8A5A9
:108FDA00A13021F40E9401760E940476A8A5A2304D
:108FEA0031F40E9401760E94E6750E941076E0E054
:108FFA00E9A30E9416760E948E7521F0EF8DA9A131
:10900A00AE1708F007C00E9416760E9498750E9453
:10901A001B76EFCFAF8DE8A1EA1BAE2FED8DEA17D5
:10902A0068F0AF8DE8A1EA1BACE0EA9FF001A091DD
:10903A000D040E94F0750E94FE7501C0E0E0EE8FFB
:10904A00A8A5A130A1F40E940176E20FF31F319680
:10905A000E946875AFE00E94C175E40FF51FDF0139
:10906A00ECA1FDA10E94C77031960E94BB6DA8A514
:10907A00A23089F40E940176E20FF31F0E946875FC
:10908A00AFE00E94C175E40FF51FDF01ECA1FDA15D
:10909A000E943F74BDDD0E941676AE0FBF1FAC91D1
:1090AA00A03219F4E9A1EF5FE9A30E9416760E94A3
:1090BA008E7539F0AF8DE9A1EA1BAE2FED8DEA1757
:1090CA0008F407C00E9416760E9498750E941B76C3
:1090DA00ECCFD8011C96EC91E03029F10E940D6E7C
:1090EA000E94C57595DDF801A485A43698F4EFE0D1
:1090FA00E0931004F801A485AA3028F0A485AA9365
:10910A000E94B84006C0D8011C96EC91E05DEA9333
:10911A00FDDC09C0ECE0E0931004E2E5EA93F6DC3A
:10912A00EDE4EA93F3DCEB8DE0930D04EA8DE09332
:10913A000E040E94D67CAA9608951A9310E0E89429
:10914A0027F8143170F40E94EA6DE03011F00E94A1
:10915A00F16D1F5FA895E12FE37011F40E94491485
:10916A00F0CFEFE0E09310040E9449147AC11A93F9
:10917A0010E01431F8F40E94F66DB1F0A85FBC4F0C
:10918A000E94ED7ADF01EB81FC81EA17FB0764F4A8
:10919A00F001E85FFC4FDF010E94ED7ADF01E9810F
:1091AA00FA81AE17BF070CF002C00E94F16D1F5F73
:1091BA00A895DFCFEFE0E093100418812596089573
:1091CA001A9310E0143190F40E94F66D31F0FD010B
:1091DA00E15FFC4FE081E17009F406C01A93E09167
:1091EA000A04E170EA9383DD1F5FECCF3AC11A9358
:1091FA00EFEF0E948871E093380910E00E94AD7089
:10920A00E15CF54FE081EF3F31F00E94AD700E94C2
:10921A0023761F5FF3CF25C11A930A930091CF0BD0
:10922A00AA81A53411F4E0E066C0AA81A23539F416
:10923A00A0913408A13019F40E94267609F405C0D9
:10924A000E94991BE0E0E0933408AA81AB3411F044
:10925A00A33599F4E02FE470E43011F414E001C06E
:10926A0013E0E02FE270E23009F41C5FE02FE170B6
:10927A00E13009F41F5FE12F3EC0AA81A13511F048
:10928A00A13799F4E02FE470E43011F417E001C03B
:10929A0016E0E02FE270E23009F41C5FE02FE17083
:1092AA00E13009F41F5FE12F26C0AA81A33421F01F
:1092BA00A13411F0A23441F413E0E02FE170E1305F
:1092CA0009F41F5FE12F17C0AA81A73741F417E0FD
:1092DA00E02FE170E13009F41F5FE12F0CC0AA8191
:1092EA00A03441F415E0E02FE170E13009F41F5F8A
:1092FA00E12F01C0EFEF19810881239608950E949A
:10930A002C76008011800E94416D0E941671EA1726
:10931A00FB0791F10E942C76DF010E94ED7A0E94F0
:10932A0034760E942C76DF010E94ED7AEC59F44FD4
:10933A00E0810E943C760E9443760E944676E85578
:10934A00F84F0E94CC700E944C760E945076E9E950
:10935A00F7E10E943872E881E03039F00E944676DF
:10936A000E9454760E94B15E02C00E9458760E9402
:10937A0050760E94665F16C0E881E03099F00E943C
:10938A004676EC55F84FDF010E94ED7A0E94456F50
:10939A00E883A881A03430F4EA93E091C605EA9301
:1093AA000E94AB259AC21A930E945C7639F00E94F9
:1093BA004676ED55F84FE081E23009F01CC0A091E5
:1093CA003E09A23429F4E6E0E0933F09E03009F4CB
:1093DA0005C0E1E0EA9393DF0E946276E091600CB7
:1093EA00F091610CFA93EA93E8ECF0E00E948D7236
:1093FA0011F40E9462760E945C7639F00E944676E9
:10940A00ED55F84FE081E13009F02BC0E0E0E09340
:10941A0034080E948171E0E0E0935C0BE2E0EA9399
:10942A000E947F5E0E9446760E9454760E94B15E38
:10943A0010915C0B123011F0133029F4EFE7EA9324
:10944A000E947F5E10581A930E947F5EE3E00E949A
:10945A0068760E946F760E942D64E093600CF09308
:10946A00610C1991089524970E94CF7C2091CF0B0B
:10947A00A0913F09A53411F00C94F64AE0E0E0937C
:10948A0034080E948171E0E0E0935C0BE091D30B19
:10949A00E03029F50E945C7639F00E944676ED5557
:1094AA00F84FE081E13009F01AC0E7E7EA930E9439
:1094BA007F5E0E944676E855F84F0E94CC70FA9378
:1094CA00EA930E9475760E9454760E947576E75553
:1094DA00F84FE081E05D0E9468760E946F76E09125
:1094EA003408E03011F00C94F64A0E94267611F402
:1094FA000C94D04A0E948E1BE1E0E0933408E22FDC
:10950A00E870E83081F40E947A76E8EEF3E00E948F
:10951A00747ADF010E94C57C14F4E1E301C0E0E340
:10952A00EA930E947F5EE22FE074E03411F413E0C4
:10953A0001C012E0E091240C0E94D2731A930E9497
:10954A00EA5EE22FE470E43049F40E947A76E0E1C0
:10955A00F7E20E94A67AAF0114E006C00E947A766A
:10956A000E94DB72AF0113E0E22FE071E03111F4E7
:10957A00415050405A934A931A930E94EA5EE22F4E
:10958A00E072E03211F414E001C013E0E091270C1C
:10959A00F091280C17C018E0E22FE470E43009F4C7
:1095AA001F5FE22FE870E83009F41F5FE22FE072D4
:1095BA00E03209F41F5FE22FE074E03409F41F5F20
:1095CA00E0E0F0E0FA93EA931A930E94EA5EE22F4F
:1095DA00E170E13029F4E0915C0BEA930E947F5E2E
:1095EA0006DEA0913F09A73729F4E2E0E0933408A8
:1095FA00E03009F42BC00E9481710E947F760E949C
:10960A003C721E2F0E945772AF01E1E0EA930E945A
:10961A00255E0E2F0E945C7639F00E944676ED5543
:10962A00F84FE081E23009F00EC00E944676EC5510
:10963A00F84FDF010E94ED7A4E175F0711F40A9383
:10964A005EDE0E946276E0E0E0933408A0913F0972
:10965A00A33421F40E94E332E03009F40BC00E94E3
:10966A0081710E947F760E948B740E947E6B68D300
:10967A000E943F1CA0913F09A13411F0A23421F4A9
:10968A000E9481710E947F76A0913F09A03421F443
:10969A000E94E332E03009F420C00E943C72E8875D
:1096AA00F987E2E0EA930E94255E1E2F0E948576E2
:1096BA000E946B170E9474730E948B76E152F84FD6
:1096CA0010830E947473E652F84FA7E0A0830E94A9
:1096DA0055710E9481710E947F76A0913F09AB3437
:1096EA0039F0A33529F0A13519F0A13709F07AC06C
:1096FA000E94E332E03011F40C94F14B0E94817124
:10970A000E949276E0E4F9E00E945272E22FE2703F
:10971A00E23029F4E4E0EA930E94255E02C0E1E027
:10972A00F0E0E887F987A0913F09A13511F0A13748
:10973A0021F40E9457721E2F02C01091E50BE22FEE
:10974A00E470E43011F4E4E001C0E3E0EA930E943B
:10975A00255EAF01A0913F09A33511F0A13731F47D
:10976A00E885F9850E94E379E887F9875A934A934D
:10977A000E94B6170E2F003420F0A091D30BA1300F
:10978A0011F51A935A934A93EB85FC85FA93EA9357
:10979A000E945E1C0E949676EE83FF83AE81BF8193
:1097AA000E94C57C84F40E948171E6E6EA930E94D5
:1097BA007F5EEE81FF813197EE83FF83AE81BF81A9
:1097CA000E94C57C94F31A935A934A93EB85FC85BD
:1097DA000E940F720CDD06C00E948B740E947E6B81
:1097EA000E945E1C0E94D67C2A9608950E949A7650
:1097FA00E89422F80E944C73E2E7EA930E947F5EA3
:10980A00E0913A08EA930E947F5EEFE0EA930E94B1
:10981A007F5EA0913708AA3219F41A9366D31AC048
:10982A00A0913A080E94AD70EC59F44FE081EA1712
:10983A0021F4E0913A08E03349F40E94076CAC59EC
:10984A00B44FE0913A08EC931A934FD322FC02C02A
:10985A000E94665FC1C20E949A76E0913A08E0537C
:10986A00AE2F0E94AD70EB58F44FE081EA1741F534
:10987A001A933BD3A0913508A23019F40E94A2761C
:10988A0009F402C00E94A876A0913508A33019F401
:10989A000E94A27609F402C00E94A876E0E0E09352
:1098AA003508E093620C0E94AD70EB58F44FBF018B
:1098BA00E081EF5FAE2FEAE00E94A37ADB01EC932E
:1098CA008BC2E881E03019F40E94587606C0E8811C
:1098DA00E8500E94D2730E94B15E219608950E94B8
:1098EA00CF7CA091E40BA63009F45DDD25FC24C2EF
:1098FA000E94A27611F40C94EF4D0E94AE76E752C4
:10990A00F84F9F01D9011196EC91E43071F50E944C
:10991A00B4760E94B7760E94BE76F901A681A0307D
:10992A0021F4A281B381109709F007C0ECE9F7E1AD
:10993A000E9438720E94507615C00E9443760E9497
:10994A00C2760E94C676EFE9F7E10E9438720E9459
:10995A00C9760E94CF76F901A085B185BA93AA93F8
:10996A000E94B15E0E94D576E7C1E730C9F40E9431
:10997A00B4760E94B7760E94BE76E2EAF7E10E94C8
:10998A0038720E94C9760E94C676E5EAF7E10E941B
:10999A0038720E94C2760E94B15E0E94D576CCC10E
:1099AA00E93089F40E94B4760E94B7760E94BE76A6
:1099BA00E8EAF7E10E9438720E94DC760E94C676D5
:1099CA000E94D576B9C1E63029F5EAE2EA930E9407
:1099DA004C5FEBEAF7E10E943872D901EC910E94E0
:1099EA00DF76E091CD0B0E94DF76EBE4EA930E94EA
:1099FA007F5E0E94C2760E94B15EE4E5EA930E940D
:109A0A007F5E0E94C9760E94B15E0E94665F0E94D4
:109A1A00A87692C1E530C9F40E941E730E9434767A
:109A2A00D901EC910E943C760E9443760E94C2764C
:109A3A000E94C676E9E9F7E10E9438720E94C97667
:109A4A000E94B15E0E94D57677C1E83039F50E944E
:109A5A00B4760E94B7760E94BE76EEEAF7E10E94DB
:109A6A003872F901A681AA930E942A73309719F0D5
:109A7A000E94406F04C0D9011696EC91F0E0FA9367
:109A8A00EA930E94B15E0E9450760E94665FD901F5
:109A9A001196E0E0EC930E94A8764EC1E130B9F548
:109AAA00A0911908A53029F4E091CD0BE65F1E2F8D
:109ABA0001C011E0E12F0E94E3760E94AD700E947E
:109ACA00E8760E9443760E94C2760E94C676E1EB4F
:109ADA00F7E10E9438720E94C9760E94CF76D901B6
:109AEA001796EC910E94D2730E94B15EA091190858
:109AFA00A53041F40E94ED76A481B581BA93AA9368
:109B0A000E94225F0E94D8740E94F37615C1E33046
:109B1A00A1F40E941E73F0960E94FE760E941E73A4
:109B2A000E94E876E4EBF7E10E9438720E94C97657
:109B3A000E9402770E94F376FFC0EB3059F50E942B
:109B4A0005770E940877E7EBF7E10E943872F9017E
:109B5A00A681AA93B6DE0E94ED76A781AA93B1DE0A
:109B6A000E94ED76A085B185BA93AA930E94CF761A
:109B7A000E94C9760E94CF76F901A481B581BA9371
:109B8A00AA930E94CF760E94DC760E9402770E94F6
:109B9A00F376D2C0EC3079F40E9405770E940877F8
:109BAA00EAEBF7E10E9438720E94DC760E940277A3
:109BBA000E94F376C1C0EE3069F40E9405770E94D4
:109BCA000877EDEBF7E10E9438720E94D8740E9480
:109BDA00F376B2C00E94267661F0A0913508A030D3
:109BEA0041F4A091D20BA13021F40E94416DE130E1
:109BFA0009F426C0A091850BA03059F0E091870B9B
:109C0A00F091880BFA93EA93E8EEF3E00E948D72E2
:109C1A00B9F4E1E30E94FE76E091760BE05D0E94E2
:109C2A003C760E94416DEA9314D1E09335080E9474
:109C3A00D874E0935E0CF0935F0CE0E0E093850B40
:109C4A00A0913508A03059F0E0915E0CF0915F0CBC
:109C5A00FA93EA93E4E6F0E00E948D7209F025C0D7
:109C6A00A0913508A23019F40E94A27609F402C024
:109C7A000E94A876A0913508A33019F40E94A27612
:109C8A0009F410C0A091620CA33030F00E94A876AB
:109C9A00E0E0E093620C06C00E94AE76E652F84F0E
:109CAA00A8E0A083E0E0E0933508A091860BA130FC
:109CBA0011F00C94A14EE091390CA091380CEA17DE
:109CCA00B1F1EAE20E94FE76E091740BE05D0E9437
:109CDA003C76E091390CEA930E94F61D0E94437685
:109CEA00E091290C0E94D2730E94C676E0ECF7E15B
:109CFA000E9438720E942E700E944C76EAE3EA9320
:109D0A000E947F5E0E94BD730E944C760E9450762C
:109D1A000E94665FE091390CEA930E94381CE09138
:109D2A00390CEA930E94071CE093390C05C0E0E065
:109D3A00E093860B689420F80E94D67C26960895B4
:109D4A001A930A930E94E332E030D9F00E947473A6
:109D5A00E752F84F8F01EC81FD81D8011296ED93FD
:109D6A00FC93EA81FB81D8011896ED93FC93EE816E
:109D7A00D8011696EC93D8011196E4E0EC930E9470
:109D8A0055711981088127960895E091410BEA934C
:109D9A000E947F5EE091420BEA930E947F5E0895E3
:109DAA00F4DF0E940C770E940F770E940F770E94BF
:109DBA00507699C01A930E94AF5D1E2F103021F081
:109DCA00E12FE150E0933F0BE0DFE0913F0BEF5FC3
:109DDA000E94D2730E94C676199108950E94D17C7E
:109DEA0031E00E94147728F00E944672AC91A433A5
:109DFA0008F02AC030E00E944672EC91E270E695C3
:109E0A001E2F0E944672EC91E1700E2FA091590B01
:109E1A001A1729F4E1E0EA27E093590B31E0A091FF
:109E2A005A0B0A1729F0E1E0EA27E0935A0B31E0CE
:109E3A00E0915A0BEE0FE05DA091590BEA0FEA93FD
:109E4A000E947F5E0E943D73E32F0E94D87C249675
:109E5A0008951A9310E00E94267611F40C94764F16
:109E6A000E948E1BE4ECF7E10E943872E091240C08
:109E7A000E94D2730E94C676E7ECF7E10E9438721C
:109E8A00E091270CF091280C0E944C760E945076A3
:109E9A000E947A76A031E7E2BE074CF4EAECF7E1D9
:109EAA000E943872E091250CF091260C13C0EDEC5B
:109EBA00F7E10E943872E9810E949D700E947A76C9
:109ECA00EA0FFB1F0E94E96FE091250CF091260C26
:109EDA00E051F742FA93EA930E94B15E0E945076EB
:109EEA0011E0E12F18812296089524970E94CF7CD1
:109EFA000E941877E0E0EC930E94585DE13010F47C
:109F0A000C946152E091410BEB3441F4E091420B25
:109F1A00E33219F40E94AF5D1E2FCBC2E435B9F4C7
:109F2A00E091420BE33221F40E94AF5DEE83FF839E
:109F3A00E091420BEF3451F40E94AF5D1E2F1A9349
:109F4A00EF81F885FA93EA930E946B17B2C2E23462
:109F5A0011F00C94F750E091420BE13251F4AA85CA
:109F6A00AF3F29F40E948B740E947E6BE9DE0E9447
:109F7A003F1CE091420BE134E1F40E94AF5D1E2FD9
:109F8A00113071F4A0913508A13019F40E94267697
:109F9A0009F402C00E94991BE0E0E093850B09C016
:109FAA00E1E0E093850B0E942D64E093870BF09328
:109FBA00880BE091420BE534A9F4E0EDF7E10E9449
:109FCA0038720E94761BF3973CF00E94AF5D0E94A4
:109FDA00E96F0E941D7701C0E0E3EA930E947F5E69
:109FEA000E945076E091420BE63409F50E942977E7
:109FFA0019F40E94AF5DAF01E885F9850E94456FAB
:10A00A000E2FE091E50BE03011F01091E50B0034D2
:10A01A0020F0A091D30BA13021F40E9435770E9441
:10A02A005E1CAA85AF3F19F40E94357789DEE0915C
:10A03A00420BE23511F00C94B4500E94297719F4BE
:10A04A000E94AF5DAF0130E0A091D30BA03021F4A4
:10A05A000E94416DE13009F027C00E94E932E030E8
:10A06A0011F10E940372EC55F84FA885B985A083B7
:10A07A00B1830E940372E655F84FDF01EA850E9418
:10A08A0051710E940372E855F84F10830E940372BF
:10A09A00E755F84F40830E940372ED55F84FA1E04F
:10A0AA00A0830E94097259C00E94E332E23010F480
:10A0BA000C94B2500E9485760E94701D3E2F3F3F3D
:10A0CA0029F00E940170A417B5070CF412C00E946F
:10A0DA00BD73E41BF50B0E940F700E94E07119F426
:10A0EA00E0E0E093290C3A930E94FD1D689420F861
:10A0FA0003C0E0E0E887E9870E947473E752F84FEB
:10A10A00DF01EA85F0E0EC59F44FE081EC930E941C
:10A11A0074730E948B76EF51F84FDF01EA850E9433
:10A12A0051710E947473E152F84F10830E94747344
:10A13A00E652F84FA5E0A0830E945571E885F9859B
:10A14A00309759F00E948576FA010E94E3790E94BD
:10A15A000F720E9435770E94E81B689422F8E091FA
:10A16A00420BE335F1F50E94AF5DE887F9870E945B
:10A17A00AE76DF01E652F84FE081E23081F4FD016C
:10A18A00EF51F84F008011800E94416D0E941671B4
:10A19A00EA17FB0721F4A0913508A23009F01FC085
:10A1AA000E94AE76E552F84FDF010E94ED7ADF0198
:10A1BA00E885F985EA17FB0779F40E94AE76DF0194
:10A1CA00ED51F84FE081EA93FD01E752F84FE08143
:10A1DA00EA930E94AB2503C0E7E0E0932406689463
:10A1EA0022F867C1E43411F00C945F51E091420BFC
:10A1FA00E33559F4E3EDF7E10E9438720E943C5AC4
:10A20A000E94DF76E1E0E0933809E091420BE03505
:10A21A0011F00C945E510E94397711F40C945E513E
:10A22A0020E00E943F7740F00E944672AC91A23231
:10A23A0019F00E94437709F43CC0E22FE03061F440
:10A24A000E944672AC91A33211F421E004C00E942C
:10A25A0047770E94175A2AC0E13051F40E94467289
:10A26A00AC91A43211F422E001C020E010E01EC03B
:10A27A00E23011F0E330D1F40E9447770E9405647E
:10A28A00EF3F99F0E12FE295E07FEF930E94477745
:10A29A000E940564AF91EA0F1E2F2F5F243021F42C
:10A2AA001A930E94175A20E001C020E00E943D73D1
:10A2BA00B8CFFFC0E33411F00C94CF51E091420BB8
:10A2CA00E534B9F4E0EDF7E10E9438720E94761B9A
:10A2DA00F3974CF00E94AF5DE05FF84D0E94E96F82
:10A2EA000E941D7701C0E0E3EA930E947F5E0E940C
:10A2FA005076E091420BE634D9F441E050E00E94F6
:10A30A00AF5D0E2F0E944B77E13019F40E94AF5DCA
:10A31A00AF01E091E50BE03011F01091E50B1A93D3
:10A32A000E94EC6BE05FF84D0E94EB750E945E1C88
:10A33A00E091420BE335A1F40E944F770E943B6FF4
:10A34A00E83141F4E091890BEA930E941A17689464
:10A35A0020F806C0E885EA93EFEFEA930E94AB255E
:10A36A00E091420BE134A9F4E6EDF7E10E9438727C
:10A37A000E944F77EA930E9417180E94DE24E03069
:10A38A0011F0E1E301C0E0E3EA930E947F5E0E94DC
:10A39A0050768FC0E63511F00C943652E091420B9C
:10A3AA00E33411F00C9435520E94AF5D1E2F113028
:10A3BA0010F40C943552A0911908A13011F0A9306B
:10A3CA0091F50E944B77E03021F0A091A2061A176E
:10A3DA0009F028C011500E94AF5DAF011A930E9484
:10A3EA0077203E2F0E94A2720E94C7700F010E941E
:10A3FA00A2720E942F6D0E9456770E944B77E0301E
:10A40A0071F00E94AF5DAF010E94B6720E94C770E0
:10A41A000F010E94B6720E942F6D0E9456771A93FE
:10A42A000E94D2101DC01630D8F41150A12FEAE0B4
:10A43A000E94537AA3E2EA9FF001E855F94FBF015F
:10A44A00A12FEAE00E94A37AF0E0BB01AAE0B0E003
:10A45A000E94217ADB01AE0FBF1F14960E945B7027
:10A46A0028C0E93431F5E091420BE03551F40E94FD
:10A47A00AF5D1E2FE0E0EA931A930E94EA17E09379
:10A48A002E06E091420BEC34A1F40E94735DE09336
:10A49A0028060E944B77E03021F00E94735DE0931A
:10A4AA0029060E944B77E03021F00E94735DE09309
:10A4BA002A060E94145D20CD0E94D67C2B96089510
:10A4CA00A091570BA03521F4A091580BA03408F0A5
:10A4DA0005C0E091580BEA930E943718A091570BD8
:10A4EA00A33521F4A091580BAA3008F005C0E091D9
:10A4FA00580BEA930E946218A091570BAB3421F4CF
:10A50A00A091580BA03808F005C0E091580BEA93C7
:10A51A000E949E18A091570BA63521F4A091580BC2
:10A52A00A03108F005C0E091580BEA930E94CA18BE
:10A53A00A091570BA43511F40E945517DBD6089544
:10A54A00E3EAF6E0FA93EA93E091410BEA93E0E852
:10A55A00F0E00E94676F08950E945E77A0E0A083F2
:10A56A00E0913F0BE093580BE091410BE093570BBE
:10A57A0008950E94CF7C0E94585DE13010F40C943B
:10A58A00D955E091570BA091410BEA1709F098DFD2
:10A59A00E091410BE33239F5E091420BEC3431F4AE
:10A5AA00CFDFE4E0E09318080E946477E091420B61
:10A5BA00E435C1F4C5DFE091650CE03029F0EF77AE
:10A5CA00A9E0B0E00E942F7BE091660CE03029F010
:10A5DA00EF77AAE0B0E00E942F7B0E946477E7E061
:10A5EA00E0931808DEC2E934E9F4E091420BE4345E
:10A5FA00C1F40E943977A9F010E010E0183178F41C
:10A60A00A3E2B7E00E94AD70EA0FFB1FFF93EF933E
:10A61A000E94735DAF91BF91EC931F5FEFCF0E94D1
:10A62A007B0CBFC2EB34E1F5E091420BE13211F44D
:10A63A0087DF35C0E53211F443DF31C0E33299F4E4
:10A64A000E946A7721F00E9475770E946C180E9416
:10A65A005E77E081EB3429F4E0E0E093340CE09398
:10A66A00350C7ADF1CC0E134D1F40E94AF5D9F0142
:10A67A002093340C0E947B7791F00E94AF5D9F017A
:10A68A00A091340CF901E270F070EA2BE093340CDB
:10A69A000E947B7721F00E94AF5DE093350C81C266
:10A6AA00E33581F5E091420BE13211F449DF29C02B
:10A6BA00E33299F40E946A7721F00E9475770E942A
:10A6CA0046180E945E77E081E33529F4E0913F0B5A
:10A6DA00EA930E94821A40DF14C0EE3491F40E9479
:10A6EA00F57310E01A3068F4A3EBBBE0EE27A10F74
:10A6FA00BE1F0E94AD70ED5BF44FE081EC931F5FCB
:10A70A00F1CF4FC2E63511F00C94D353E091420BCE
:10A71A00E13211F415DF41C0E33299F40E946A77FD
:10A72A0021F00E9475770E94AA180E945E77E08144
:10A73A00E63529F4E0913F0BEA930E94DD180CDF1D
:10A74A002CC0E63531F40E94AF5D9F012093300C96
:10A75A0024C0E53471F40E94AF5D9F0120932F0C51
:10A76A000E947B7729F00E94AF5D9F012093320CF3
:10A77A0014C0E43591F440E050E00E94AF5D9F01BF
:10A78A00022E032A11F042E050E00E947B7719F072
:10A79A000E94AF5DAF014093310C03C2E43511F062
:10A7AA000C948D54E091420BE33231F40E94AF5D78
:10A7BA003197E0933F0BABC0E03511F00C948C5409
:10A7CA0010E00E943F7750F00E944672AC91AD3380
:10A7DA0029F00E94437711F01E3008F005C00E944C
:10A7EA00AD700E948177EDCF0E94AD700E948A778A
:10A7FA00EDE30E948F7711F00C948C54E4E5E0931A
:10A80A00570B10E00E94C76F3496E491EF3F11F4A2
:10A81A000C948C540E94F9730E94C76F0E94E46CD6
:10A82A000E945868E03011F00C948A540E94C76F55
:10A83A003496E491E03851F40E94AF5DE058FF4F3E
:10A84A00E093650CE0E8E093660C5FC0E23839F407
:10A85A000E94AF5DE058FF4FE093660C56C0E138A6
:10A86A0039F40E94AF5DA8E0B0E00E942F7B4DC092
:10A87A00E03011F0E13051F40E94BD6FFF93EF9385
:10A88A000E94AF5DAF91BF91EC933FC0E23059F4A3
:10A89A000E94BD6FFF93EF930E94AF5DAF91BF918E
:10A8AA00ED93FC9332C0E33051F40E94BD6FFF93E5
:10A8BA00EF930E94905DAF91BF91EC9326C0E43074
:10A8CA0021F50E94C76F3596E491EA930E94605E73
:10A8DA000E94BD6FE093630CF093640C00E00E9449
:10A8EA00C76F3596E4910E1780F40E94EC6BED5B0E
:10A8FA00F44FE081A091630CB091640CEC93A3E651
:10A90A00BCE00E94E46D0F5FEACF1F5F7BCF49C1B5
:10A91A00E03511F00C94D655E091420BE33299F4EC
:10A92A000E946A7721F00E9475770E9417180E9488
:10A93A005E77E081E03529F4E0913F0BEA930E94CB
:10A94A00991A0ADE2EC1E13211F4FADD2AC1E13484
:10A95A00D1F40E94AF5D1E2F00E00D3098F40E94E2
:10A96A001674EA0FFB1F3396E491E11749F40E942B
:10A97A0016740E941A74A0919A0BEA2BE0939A0B10
:10A98A000F5FEBCF0EC1E63559F5E0E0E093400BDF
:10A99A00ADE9BBE00E949477FF93EF930E94AF5D0D
:10A9AA00AF91BF91EC93EBE2EA930E94245DE03011
:10A9BA0059F0A0EABBE00E949477FF93EF930E94BC
:10A9CA00AF5DAF91BF91EC930E949777A091400B36
:10A9DA00A33018F40E947B7709F401C0D9CFE1C0F3
:10A9EA00ED34D1F4E0E0E093400BA9EABBE00E9429
:10A9FA009477FF93EF930E94AF5DAF91BF91EC9371
:10AA0A000E949777A091400BA33018F40E947B779D
:10AA1A0009F401C0EACFC5C0E735D1F4E0E0E0931C
:10AA2A00400BA0EBBBE00E949477FF93EF930E9448
:10AA3A00AF5DAF91BF91EC930E949777A091400BC5
:10AA4A00A23018F40E947B7709F401C0EACFA9C0AA
:10AA5A00E434C9F5E0E0E093400B0E94AF5D9F014A
:10AA6A00E2E0EA930E94315DAF01E3E70E948F774B
:10AA7A0059F40E949D77BF01D9010E944C71E40FDD
:10AA8A00F51FDB01ED93FC93E9E40E948F7779F4DB
:10AA9A000E949D7720833183AAE9BBE00E949477C4
:10AAAA000F010E94A377EC91E160D001EC930E9420
:10AABA009777A091400BA33018F40E947B7709F492
:10AACA0001C0CBCF6EC0EE3499F40E94F57310E04A
:10AADA001A3068F4AAE8BBE0EE27A10FBE1F0E9455
:10AAEA00AD70ED5BF44FE081EC931F5FF1CF59C07D
:10AAFA00E33459F4E2E2EA930E94245D0E94AF5DD6
:10AB0A00E093950BF093960B4CC0E33589F40E94C1
:10AB1A00AF5D9F0100240216030624F42B30E0E007
:10AB2A003E070CF004C0F9013197E093970B39C046
:10AB3A00E53529F40E94AF5DE093990B32C0EF34FA
:10AB4A0091F40E94AF5D1E2FECE2EA930E94245D0D
:10AB5A00E12FE295E07FEF930E94AF5DAF91EA0F9C
:10AB6A00E093980B1EC0E035E1F4E0E0E093400B7F
:10AB7A00ACEABBE00E94A9770E94C770FF93EF93EB
:10AB8A000E943F5EAF91BF91ED93FC930E9497772D
:10AB9A00A091400BA23018F40E947B7709F401C0FF
:10ABAA00E7CF0E94145DE7CC0E94D67C26960895D2
:10ABBA000E94D17C0E94585DE13010F40C94B05888
:10ABCA00E091410BE332A9F4E091420BE03519F42C
:10ABDA00E9EDF7E109C0E83419F4EAEFF7E104C056
:10ABEA00E33531F4E5E1F8E1FA93EA930E948F5EE6
:10ABFA00AFC2E934C1F4E091420BE43499F40E9403
:10AC0A00700CC3D80E94AD7710E0183148F4A3E263
:10AC1A00B7E00E94E174EA930E94BF5E1F5FF5CF1E
:10AC2A000E94AD7795C2E43511F00C94B456E091C8
:10AC3A00420BE43229F4E8E2F0E00E94B1778EC0D8
:10AC4A00E33211F4B7D88AC0E03511F00C94B35648
:10AC5A009CD8A0913F0BA83210F00C94B3560E94D6
:10AC6A00B5770E94E46C0E948F5EEDE3EA930E943E
:10AC7A007F5E0E94B5773496E491E03839F40E94F9
:10AC8A00416D0E94D2730E94B15E68C0E23839F405
:10AC9A000E94B86F0E94D2730E94B15E5FC0E13811
:10ACAA0039F40E94CD730E94D2730E94B15E56C0DD
:10ACBA00E03011F0E13051F40E94B57732960E94EB
:10ACCA00FC7A0E94CC700E944C7648C0E23059F45B
:10ACDA000E94B57732960E94FC7ADF010E9438738F
:10ACEA000E94B15E3BC0E33051F40E94B5773296C0
:10ACFA000E94FC7AE081EA930E94CE5E2FC0E43083
:10AD0A0069F50E94B57732960E94FC7AE093630C4B
:10AD1A00F093640C10E00E94B5773596E4911E1703
:10AD2A0090F40E94AD70ED5BF44F0F01A091630C9B
:10AD3A00B091640CEC91D001EC93A3E6BCE00E94C4
:10AD4A00E46D1F5FE8CF0E94B5773596E491F0E095
:10AD5A000E948A770E94F9730E94175FF9C1E3354E
:10AD6A0081F5E0913F0BEA930E944618E091420B6D
:10AD7A00E43229F4EAE0F0E00E94B17721C0E3323C
:10AD8A0011F418D81DC0EE34D9F40E94CA4E10E04E
:10AD9A001A3068F40E94AD70ED5BF44F0F01A3EB1B
:10ADAA00BBE00E94E174D001EC931F5FF1CFE0E0B9
:10ADBA00E0934D0B0E94F9730E94175F0E94507630
:10ADCA00C7C1E63511F00C942957E0913F0BEA937D
:10ADDA000E94AA18E091420BE43229F40E94867478
:10ADEA000E94D54E30C0E33219F40E94DF4E2BC0C8
:10ADFA00E53459F40E94CA4EE0912F0C0E94D27396
:10AE0A000E94B977E091320C19C0E63529F40E9404
:10AE1A00CA4EE091300C12C0E435A9F40E94CA4E21
:10AE2A00E091310CE03011F0E1E301C0E0E3EA9394
:10AE3A000E947F5E0E94BF77E091310CF0E00E9491
:10AE4A004C760E94507684C1E03511F00C947A5801
:10AE5A00E0913F0BEA930E941718E091420BE4320B
:10AE6A0029F4E0E4F0E00E94B1773EC1E33219F43C
:10AE7A000E94DF4E39C1E13411F00C9486570E94CA
:10AE8A00CA4E12E0A0919A0BECEDEA233E2F00E0A5
:10AE9A000D3078F40E9416740E941A74E31739F47C
:10AEAA000E941674EA0FFB1F3396149102C00F5FBB
:10AEBA00EFCF0E94C76C0E94C676E091980BE030F3
:10AECA0089F0E0E3F8E10E9438720E94A16C0E94C6
:10AEDA00D2730E94B977E091980BEF700E94D273F7
:10AEEA000E94C676E091990BE03051F0E3E3F8E175
:10AEFA000E943872E091990B0E94D2730E94C67622
:10AF0A00F3C0E43479F50E94C377A091400BA330D3
:10AF1A0040F5E091400BE03011F00E94BF770E94AB
:10AF2A00A377EC91E17061F4A3EABBE00E94A977F0
:10AF3A000E942F6D0E9438730E94225FE3E70BC0C4
:10AF4A00A3EABBE00E94A9770E942F6D0E94387382
:10AF5A000E94B15EE9E4EA930E947F5E0E949777BD
:10AF6A00D4CFBEC0ED34C9F40E94C377A091400B80
:10AF7A00A33090F4E091400BE03011F00E94BF77CB
:10AF8A00A9EABBE00E94C977EC910E94D2730E94A1
:10AF9A00B15E0E949777EACFA3C0E735C9F40E9451
:10AFAA00C377A091400BA23090F4E091400BE030BF
:10AFBA0011F00E94BF77A0EBBBE00E94C977EC9129
:10AFCA000E94D2730E94B15E0E949777EACF88C02E
:10AFDA00E63531F50E94C377A091400BA330F8F40F
:10AFEA00E091400BE03011F00E94BF77ADE9BBE081
:10AFFA000E94C977EC910E94D2730E94B15EEBE283
:10B00A00EA930E947F5EA0EABBE00E94C977EC91B6
:10B01A000E94D2730E94B15E0E949777DDCF60C012
:10B02A00EE34D1F40E94CA4E10E01A3068F40E943D
:10B03A00AD70ED5BF44F0F01AAE8BBE00E94E1742A
:10B04A00D001EC931F5FF1CFE0E0E0934D0B0E943B
:10B05A00F9730E94175F44C0E33499F40E94CA4E00
:10B06A000E94F973EBE3F8E1FA93EA930E94406FC6
:10B07A000E9451730E94DC740E94F9730E94175F48
:10B08A002FC0E035A9F40E94CA4EE091AC0BF091B2
:10B09A00AD0BFA93EA930E943A5F0E94BF77E09160
:10B0AA00AE0BF091AF0BFA93EA930E943A5F18C085
:10B0BA00E33531F40E94CA4EE091970BEF5F0DC061
:10B0CA00EF3491F40E94CA4E0E94A16C0E94D2737E
:10B0DA000E94B977E091980BEF70F0E00E944C76ED
:10B0EA00EBE3EA930E947F5E33C0EB3489F5E0918B
:10B0FA003F0BEA930E946C18E091420BE43229F468
:10B10A00E0E8F0E00E94B17723C0E33219F40E942C
:10B11A00DF4E1EC0E134E1F40E94CA4EA091340C05
:10B12A00E1E0EA230E94D2730E94B977A091340C1D
:10B13A00E3E0EA230E94D2730E94B977E091350CCA
:10B14A000E94D2730E94B15EEEE3F8E10E94387267
:10B15A000E94145D2FCD0C94975C1A930E94817102
:10B16A00EFE3F9E00E9452720E94CD77E181E43464
:10B17A0071F40E94CD7702800E94416DE05DE01576
:10B18A0029F00E94CD77E281EA3209F401C05BC05E
:10B19A000E94D2770E94CD77E1810E94D6770E94E1
:10B1AA00CD77E2810E94D6770E9446721C910E9456
:10B1BA00CD7733960E945272E12FE23139F40E9420
:10B1CA0018771397E6E0EC93D4D93DC0E13139F40E
:10B1DA000E9418771397E2E1EC93EADC34C0EF306F
:10B1EA00B1F40E9418771397EEE0EC930E94F34EA5
:10B1FA00E13039F4A0913408A03019F00E94267683
:10B20A0009F402C00E94991B0E94D9771CC0EE3033
:10B21A00D1F40E9418771397EFE0EC930E94F34E53
:10B22A00E13089F4A0913408A03019F00E94267602
:10B23A0009F402C00E94991BE0E0E0933408EFEFA2
:10B24A00EA930E947A4F0E941877E0E0EC9371C269
:10B25A001A930E944C730E94976FEAE7EA930E943E
:10B26A007F5E0E94467211971C91E12FE23131F400
:10B27A00E6E0EA930E947F5E7CD931C0E13131F485
:10B28A00E2E1EA930E947F5E93DC29C0EF3089F401
:10B29A00EEE00E94E07739F4A0913408A03019F06A
:10B2AA000E94267609F402C00E94991B0E94D9774F
:10B2BA0016C0EE30A1F4EFE00E94E07781F4A0918D
:10B2CA003408A03019F00E94267609F402C00E94C0
:10B2DA00991BE0E0E0933408EA930E947A4F0E94B7
:10B2EA001877E0E0EC93A0913708AA3211F00E9497
:10B2FA00665F1FC2EFEFE093570BE093580B089578
:10B30A00AC81A03310F0AA3308F006C00E94E77798
:10B31A00E0530E94EF77ACC4AC81A13410F0A7349B
:10B32A0008F006C00E94E777E7530E94EF77A0C4AF
:10B33A00A881B981E0E0EC939BC4AA93EA93FA93BB
:10B34A00EFB7EA931A930A931BB10CB1E0919F0CE1
:10B35A00F0E0E359F34F0083A0919F0CAF5FA093F5
:10B36A009F0CA23319F4E0E0E0939F0C0991199124
:10B37A0004C31A93E091A00CA0919F0CEA17D1F391
:10B38A00F0E0E359F34F1081A091A00CAF5FA093B6
:10B39A00A00CA23319F4E0E0E093A00CC9C1A0917B
:10B3AA009F0CAE5CE091A00CAE1BE2E30E94A37A74
:10B3BA0008950A921A92FA926A937A938A939A93BE
:10B3CA00AA93BA93EA93FA93EFB7EA930E94F477AF
:10B3DA0049F0A0913809A03021F00E946A0CE130AE
:10B3EA0009F401C011C0E091060DF0E0EF55F34FEA
:10B3FA00E081ECB9A091060DAF5FA093060DA436CB
:10B40A0019F4E0E0E093060DE991EFBFF991E991B3
:10B41A00B991A9919991899179916991F990199024
:10B42A00099018951A930E94F47759F45D9B09C004
:10B43A00A0913809A13021F40E946A0CE03009F089
:10B44A0013C01091050D0E94AD70EF55F34FA981FD
:10B45A00A0831F5F143609F410E0E091060DE1178E
:10B46A00E1F31093050D02C0E981ECB9B2C20E9462
:10B47A00F47721F40E946A0CE13009F001C02AC372
:10B48A0060C10E94D17C8BDFE03011F40C94565BD2
:10B49A0070DF1E2FA0916A0CA53618F0E0E0E09349
:10B4AA00390930913909E0913909E03011F00C94E9
:10B4BA00BD5AA091E40BA63029F4163011F01531CB
:10B4CA0009F401C004C010933F09E2E4E0C0A0916E
:10B4DA00E40BA13041F0A091E40BA23021F0A0913D
:10B4EA00E40BA53031F4E12FEF77E0933F09EBE469
:10B4FA00CEC01A3521F4E1E0E0933909CAC012300E
:10B50A0049F4E4E1E0933909E0E0E0933A09E09391
:10B51A003C09BFC0A091E40BA33069F4173729F0A6
:10B52A001A3310F4103308F402C0E7E001C0E0E077
:10B53A00E0933B0905C01A930E941149E0933B0925
:10B54A00A0913B09AF3F99F010933F09E1E0E093E6
:10B55A003A0910933C09E0913B09E03011F4E5E423
:10B56A0004C0EAE0E0933909E0E0E0933E0991C0C3
:10B57A00E13069F4103039F4E2E0E0933909E0E0AF
:10B58A00E0933E0903C0E0E0E093390982C0E2306B
:10B59A0059F410933B0910933C09E0E0E0933A090F
:10B5AA00E3E0E093390975C0E330F1F40E94FA77D9
:10B5BA000E940078EA0F0E940A78A9F4E0913C09F7
:10B5CA00E03071F4E4E0E0933909E0913A090E942D
:10B5DA00E86E0E9413780E94FA77A0E0A08303C065
:10B5EA00E0E0E093390955C0E43049F41D3019F41C
:10B5FA00EAE5E0933E09E0E0E09339094AC0EA301F
:10B60A0079F40E94FA770E940078EA270E940A7861
:10B61A0031F4E0E0E0933909E5E4E0933E0939C00A
:10B62A00E431B9F40E94FA771083E12FA0913C0922
:10B63A00EA27E0933C09E0913A09EF5FE0933A097F
:10B64A00E0E0E093690C133019F4E5E1E09339097D
:10B65A0020C0E53111F0E63159F41A93E9E6FCE02D
:10B66A00FA93EA93E9E3F9E0FA93EA9349DE11C01F
:10B67A00E73179F4E0E0E0933909173131F4E091E8
:10B68A00690CA0913C09EA1709F003C0E3E4E093CE
:10B69A003E09A09139093A1719F0E0E0E0936A0CE3
:10B6AA00F2CE40C1AA93BA93EA93FA93EFB7EA9318
:10B6BA001A930A9310919B0000919C00E12FEC7160
:10B6CA00A9F4E091CF0DF091D00DE95FF24F00831C
:10B6DA00AFECBDE00E94E46DE83CA0E0FA0731F46B
:10B6EA00E0E0F0E0E093CF0DF093D00D09911991CD
:10B6FA00E991EFBFF991E991B991A99118951A9336
:10B70A000E9418780E941D78D9F30E941878E95F80
:10B71A00F24F1081A1EDBDE00E94E46DE83CA0E08B
:10B72A00FA0731F4E0E0F0E0E093D10DF093D20DA6
:10B73A00E12F199108950E9418780E941D7809F046
:10B74A00C9C1E0E008950E94D17CF5DFE03021F024
:10B75A00A091680CA03009F0E5C0D1DF1E2FA0919E
:10B76A00DB0DA53618F0E0E0E093D50D3091D50D4C
:10B77A00E091D50DE03059F4113019F4E4E0E0938A
:10B78A00D50D1A3519F4EAE0E093D50DC3C0E430BB
:10B79A00C1F4E0E0E093D50D1A3229F00E94416D20
:10B7AA00E05DE11769F4109337081093D60DE5E0D0
:10B7BA00E093D50DE0E0E093680CE1E0E093D80D6A
:10B7CA00A9C0E530A9F4E0E0E093D50D0E94416DEF
:10B7DA00E05DE11761F00E9424780E942D78E091E3
:10B7EA00D80DEF5FE093D80DE6E0E093D50D92C057
:10B7FA00E63091F4E091D80D0E942D780E942478C9
:10B80A00EF5FE093D80DE0E0E093D90D133019F41F
:10B81A00E7E0E093D50D7EC0E73011F0E83059F447
:10B82A001A93E9EDFDE0FA93EA93E5EDFDE0FA9368
:10B83A00EA9366DD6FC0E93081F4E0E0E093D50D6C
:10B84A00173131F4E091D90DA091D60DEA1709F01C
:10B85A0003C0E4E5E093680C5DC0EA3041F41030BF
:10B86A0011F4EBE001C0E0E0E093D50D53C0EB30FA
:10B87A0071F4E0E0E093D80D1093D70D1093D60D34
:10B88A00ECE0E093D50DE0E0E093680C43C0EC30C7
:10B89A00A1F5E091D80DF0E0E15CF64F10830E942B
:10B8AA002478EF5FE093D80DE091D70DE150E09353
:10B8BA00D70DA091D70DA03021F4A091D60DA030BC
:10B8CA0009F00EC0EDE0E093D50DE091D80D0E948D
:10B8DA00E86E0E941378E091D80DF0E00E94137888
:10B8EA00A091D70DA03021F4A091D60DA03009F473
:10B8FA0003C0E0E0E093D50D0DC0ED3059F4E0E06F
:10B90A00E093D50D1D3031F4EAE5E093680CEFEFD2
:10B91A00E093670CE091D50DE31719F0E0E0E093AE
:10B92A00DB0D13CF0E94D87C24960895AA93EA933C
:10B93A00FA93EFB7EA93E091DD0EA091DC0EEA17D5
:10B94A0091F0E0913608E03019F0E89426F80AC040
:10B95A000E943278F0E0E030A1E0FA0719F4E0E062
:10B96A00E093DD0E03C0E89425F826F8E091670C11
:10B97A00E03019F0E0E0E093D50DE991EFBFF991DD
:10B98A00E991A99118951A93E091DD0EA091DC0E28
:10B99A00EA1721F4E0919B00E072C1F4E091DC0E19
:10B9AA00F0E0E452F24FA981A0831091DC0E1F5FF0
:10B9BA000E94076CA030E1E0BE0709F410E0E091B4
:10B9CA00DD0EE117E1F31093DC0E03C0E981E09389
:10B9DA009C00188122960895E0E0E093DD0EA09184
:10B9EA00DC0EA13020F00E943278689426F808957F
:10B9FA00AA93BA93EA93EFB7EA93E091670CE0301F
:10BA0A0041F4E0E0E093DD0E0E94416DEF5FE093C8
:10BA1A003608E991EFBFE991B991A99118950E9469
:10BA2A003F7718F00E94437709F403C00E943D73E0
:10BA3A00F6CF0E94437711F40E943D7308950E9445
:10BA4A004672AC91E881EA1729F40E943D73319756
:10BA5A00E1E099C3E0E097C30E94D17C00E010E0E6
:10BA6A00EEE20E948F77E9F420E030E0EC810E9458
:10BA7A004078BCF4D8010E9408748F010E941477A0
:10BA8A0018F00E94457808F009C00E944672EC91AD
:10BA9A000E94E0720E0F1F1F0E943D732F5F3F4FDF
:10BAAA00E5CFF801E3C00E943F7728F00E94CD77E6
:10BABA00E181E03208F410C00E944672EC91E093F2
:10BACA00410B0E943D730E944672EC91E093420B37
:10BADA000E943D73E1E008950C946B621A930A93F5
:10BAEA0000E010E01230A8F40E9447770E94056433
:10BAFA00EF3F69F0E02FE295E07FEF930E944777EE
:10BB0A000E940564AF91EA0F0E2F0E943D731F5FDA
:10BB1A00E9CFE02FE5C31A930A9310E00E94467218
:10BB2A000C910B3311F0003208F412C0013310F0FB
:10BB3A00093308F007C0E02F0E94E072E853FF4F74
:10BB4A00E4911E2B0E943D730E9446720C91E9CF2C
:10BB5A00E12FC6C30E94D17C00E010E00E94467229
:10BB6A00AC91AD3221F40E943D7331E001C030E066
:10BB7A000E94147718F00E94457808F009C0D8018D
:10BB8A000E9408740E9449788F010E943D73F0CF89
:10BB9A00303029F4F8010E94D87C0C94AB62F80189
:10BBAA000E94E3790E94D87C0C94AB6224971A9382
:10BBBA00E0E0E983EA83EB83EC830E944672AC916E
:10BBCA00AD3221F40E943D7311E001C010E00E94E1
:10BBDA00147718F00E94457808F022C0A981BA812A
:10BBEA008B819C81EAE0F0E060E070E00E944E7A8E
:10BBFA007F936F93FF93EF930E944672EC91E05309
:10BC0A00AF91BF918F919F91FF27662777270E9457
:10BC1A00D979E983FA836B837C830E943D73D7CFFA
:10BC2A00103031F4E981FA816B817C81188120C05E
:10BC3A00E981FA816B817C810E94E779188118C0B9
:10BC4A000E94D17C20E030E000E010E0EC810E940C
:10BC5A0093755CF4D9010E9408740E9449789F0187
:10BC6A000E943D730F5F1F4FF1CFF9010E94D87CEC
:10BC7A00259608950E94D17C6DDF8F0120E030E087
:10BC8A00EEE20E948F7711F465DF9F01112322F4FF
:10BC9A00F9010E94E3799F01A0911B0CA13030F0B9
:10BCAA00D8010E944C71E20FF31F8F01F8010E9424
:10BCBA00D87C0C94AB621A9310E00E943977A1F0F9
:10BCCA000E943F7758F00E944672AC91A23231F03E
:10BCDA000E94437719F0E9811E1708F005C00E94F7
:10BCEA00AD700E948177ECCF0E94AD700E948A7776
:10BCFA000C94C562E8810E94D677E881A0915B0B1B
:10BD0A00EA0FE0935B0BE881A0915C0BEA27E093D2
:10BD1A005C0B39C21A9310E0E12FA981BA810E9403
:10BD2A001274E491E03049F0E12FA981BA810E94AE
:10BD3A001274E4910E944E78EFCF0BC01A9310E070
:10BD4A000E948475E03029F00E9484750E944E7822
:10BD5A00F7CF18812396089564970E949E740E94D3
:10BD6A005378E88DF98D0E9451730E94CE74E6DFF4
:10BD7A006696089564970E949E74E7E4F8E1FA9340
:10BD8A00EA93E88D0E94C46B0E949E74D7DF659681
:10BD9A0008951A93ECE3EA93ADDF11E0193080F4C9
:10BDAA000E94AD70E853FF4FE491A981EA2319F08C
:10BDBA00E12FE05D01C0E0E2EA939CDF1F5FEECF76
:10BDCA00EEE3EA9397DF0C94C56264971A930E9494
:10BDDA0058780E945378EA8DFB8D0E9451730E9415
:10BDEA00DC740E9458780E9480681E2FED891E1705
:10BDFA0020F40E9458761F5FF9CF0E9458789EDF80
:10BE0A0018810EC064970E949E740E945378E88D30
:10BE1A00F98D6A8D7B8D0E94A5730E949E748EDFB8
:10BE2A00689608950E94AD77E881F981FA93EA93BA
:10BE3A0085DF0E94AD770C94C662A881B981E4E6D9
:10BE4A00F0E00E94747A0E944C76EEE2EA9352DFA6
:10BE5A00A881B981E4E6F0E00E94A67AFA93EA930F
:10BE6A00E2E0EA93B2DF0C94C662A0911B0CA13007
:10BE7A0030F0E881F981FA93EA93DFDF06C00E9485
:10BE8A000C77ECE4F8E10E9438720C94C66225FE45
:10BE9A0006C0E5E0F0E00E94BF6DA895F8CFECED92
:10BEAA00FDE0E0935D0BF0935E0BE1E00E94887188
:10BEBA00E0935B0B0E945D780E94416D0E94DF76E1
:10BECA0062C11A930A93E091670CE03009F008C244
:10BEDA00E3E0EA930FDFE0915B0BE295EF70EA9300
:10BEEA000E941C641E2FE0915B0BEF70EA930E9484
:10BEFA001C640E2F1A93FEDE0A93FCDEE7E1EA9336
:10BF0A00F9DEECEDFDE00E9418770E94107BEA1B37
:10BF1A00E093DC0E689425F8E3C1EE81EA93B7DF7B
:10BF2A00EC81FD810E9438720E9461786BDFC9DF63
:10BF3A000C94F362EB81EA93AADF0E94A870EADE0E
:10BF4A000E945D78BEDF0C94AB62ED81EA939FDFBD
:10BF5A00EB81FC810E943872EA81EA93CBDEE981A7
:10BF6A00E03011F0EA93C6DEE881E03011F00E9479
:10BF7A005D78A7DF0C944D640E94CF7C10E0E0E569
:10BF8A00F8E1A885B985EA17FB0719F444E150E0FE
:10BF9A0002C048EC50E0EA85E0933709E89431F8AA
:10BFAA00EA93E985FA85FA93EA93EA85EA93EA85B8
:10BFBA00EA93E0E0EA93C9DF0E942D649F010E94A0
:10BFCA0052140E94C5750E9438640E2F31FC02C0BB
:10BFDA00003009F001C0F3CF31FE04C0E89431F813
:10BFEA00E1E004C01F5F1230B0F2E0E00E94D67CAC
:10BFFA002B9608951A930A93E0913F0AE03009F4C8
:10C00A006FC1E0E0E0933809E2E0EA930BDA10E06E
:10C01A0003E00E94AD700E94687861F00E94AD70E2
:10C02A000E9423760E94AD70E15CF54FE0810E27F5
:10C03A001F5FEFCFE3E0EA93F5D9E02FE295EF70C7
:10C04A000E946D78E02FEF700E946D78E7E1EA9325
:10C05A00E9D946C11A930A93E0913F0AE03009F4FC
:10C06A003FC10E94B86FE03021F0E091410AEA3204
:10C07A0009F405C00E94B86FE05DE093410AE0E070
:10C08A00E0933809EAE5EA93CDD9E0E0EA93CAD920
:10C09A0010E00E94AD700E94687811F01F5FF9CF1E
:10C0AA001F5F012F0A93BED910E00E94AD700E9453
:10C0BA00687861F00E94AD700E9423760E94AD708C
:10C0CA00E15CF54FE0810E0F1F5FEFCFE02FE195A6
:10C0DA00EA93A8D9EDE0EA93A5D902C11A930A9383
:10C0EA00F894E0E0E0933608E091DD0EE093DC0E90
:10C0FA007894E0913F0AE03009F4F2C0EAE5EA9365
:10C10A0042DCE0E0EA933FDC10E00E94AD700E945E
:10C11A00687811F01F5FF9CF1F5F012F0A9333DC94
:10C12A0010E00E94AD700E94687879F00E94AD70AC
:10C13A00E15CF54FE081EA9326DC0E94AD70E15C98
:10C14A00F54FE0810E0F1F5FECCFE02FE195EA93E8
:10C15A001ADCEDE0EA9317DCC3C0E881EA9397DEC4
:10C16A00EAE5EA93C7DDE0913F09EA93C3DD0E945D
:10C17A004672EC91E03031F00E944777BBDD0E94B5
:10C18A003D73F5CF9EDE219608951A930E94817120
:10C19A00E0913A08EA93AEDDE4E4EA93ABDDE0919C
:10C1AA003808EA93A7DD14E00E94AD70E95CF74F06
:10C1BA00E081E43040F00E94AD70E95CF74FE08125
:10C1CA000E944E78F1CFE0E0EA9394DD43DF79C133
:10C1DA001A930A9356D9E0913E09E03011F40C946F
:10C1EA007461A0913E09AA3541F4A0913A09A3309D
:10C1FA0020F0E0914009E43409F04BC00E94B86F86
:10C20A00E03021F0E0914109EA32C1F40E94416D27
:10C21A00E05DA0914109EA1721F0E0914109EA3273
:10C22A0021F40E94B25816DF08C0E2E4F9E00E9445
:10C23A005272E09141090E9473782BC00E94B86F34
:10C24A00E05DA0914109EA1721F50E94416D1E2F78
:10C25A00E0914209ED3421F4E0914309E33209F017
:10C26A0007C0E4E4F9E00E94527274DC1E2FD7DBA7
:10C27A000E94416DE11729F0E12FE05D0E94737879
:10C28A0008C00E94416DE05DE09341090E94B258E6
:10C29A00E1DEA0913E09A53449F4A091E40BA33054
:10C2AA0019F40E94342A02C00E94384AA0913E0919
:10C2BA00A33411F40E94E529A0913E09AB3411F48C
:10C2CA000E94E029A0913E09A23431F4A091E40B26
:10C2DA00A63011F40E94D849E0E0E0933E09E0E07C
:10C2EA000991199108952FDAA091680CA43529F4BF
:10C2FA00A0E025FCA1E0A03009F03AC0E09139089D
:10C30A00E03581F4E0913A08EA93E6E0EA930E9484
:10C31A003C42A0913A08A03820F0E0913A08E09314
:10C32A00650523C0E03721F4E0E0E09365051DC010
:10C33A00EA3519F40E942D5918C0EA3711F425DF9D
:10C34A0014C0E23519F40E94FB4B0FC0E23719F40E
:10C35A000E94304C0AC00E94BE2FE0913808A0917A
:10C36A003709EA1711F4689431F8E0E0E093680CB1
:10C37A00A091680CAA3531F40E94B258AFDEE0E011
:10C38A00E093680CA3C0A0916B0CA13050F0E0912F
:10C39A006B0CE150E0936B0CE03019F4E1E0E093B0
:10C3AA006C0CA0E025FCA1E0A13049F4A0E026FC39
:10C3BA00A1E0A03021F4A0913608A03009F001C014
:10C3CA000BDBE0913608E03019F0E150E0933608D3
:10C3DA000895E091DB0DEF5FE093DB0DE0916A0CCD
:10C3EA00EF5FE0936A0CE091670CE03019F0E150DE
:10C3FA00E093670C0895A091E40BA13041F0A0915D
:10C40A00E40BA23021F0A091E40BA53029F4E3E07B
:10C41A00E0939000E8E3E9B9A091E40BA63029F48F
:10C42A00E1E0E0939000ECE9E9B90895E091610B4D
:10C43A00E0937100E0E0E0937400E2B3E360E2BBF2
:10C44A00E1B3E360E1BB85E38A95F1F7E1B3EC7F01
:10C45A00E1BBE4E4E093740088EC90E00197F1F723
:10C46A000895E2E001C0E0E0E093610BDFDF0895A8
:10C47A001A931FEFF6DF16D0E03089F4E9810E94A3
:10C48A007A7841F4EDB7FEB7FA93EA931F930E94C4
:10C49A007F781F9118D080E991E00197F1F7E3DFE7
:10C4AA00E12F6EC01A9314EAE4EA0E94837841F4F9
:10C4BA000E948878183011F0103111F4E0E001C0C0
:10C4CA00E2E019910895E4E9E0937400E0E0089548
:10C4DA001A93E981E1600E948D7831F40E9488788C
:10C4EA00103411F4E0E04CC04AC01A93E9810E946A
:10C4FA008D7831F40E948878183111F4E0E040C058
:10C50A003EC01A93E9810E948D7831F40E9488789E
:10C51A00183211F4E0E034C032C01A93E981E030F5
:10C52A0011F0E4EC01C0E4E80E94837869F40E9407
:10C53A008878E0917300AA81BB81EC93103511F0E1
:10C54A00183511F4E0E001C0E1E01881249608955D
:10C55A001A93E981E093740010E0E0917400E078A6
:10C56A0011F4163908F005C08BE18A95F1F71F5FBF
:10C57A00F4CFE0917400E07811F0E0E001C0E1E06E
:10C58A001881229608950E94D17C3D810C8120E079
:10C59A0089DFE030F9F4EE810E94726ED9F43A93A1
:10C5AA00B0DFE030B9F40E949178A1F47BDFE0308B
:10C5BA0089F4EE810E947A7869F4EDB7FEB7FA93AE
:10C5CA00EA931F930E947F781F91E03019F47BDF72
:10C5DA00E12F02C02BDFDCCF0E94D87C279608957A
:10C5EA000E94D17C30E00E811D815CDFE03099F43D
:10C5FA00EF810E94726E79F40E94917861F41A9325
:10C60A0080DFE03041F4EC81EA937BDFE03019F41B
:10C61A005ADFE0E002C00ADFE8CF0E94D87C289601
:10C62A00089522970E94CF7C50E02B853A85A895E1
:10C63A0039DFE03011F00C947963EE850E94726E56
:10C64A0011F00C9479632A935CDFE03011F00C94BA
:10C65A0079633A9356DFE03011F00C94796322DF64
:10C66A00E03011F00C947963EE850E947A78E1F556
:10C67A00E0E0EE83EF83EC85FD8531970E945875E3
:10C68A0049F4EDB7FEB7FA93EA931F930E947F78B5
:10C69A001F9109C0EDB7FEB7FA93EA931F93E1E041
:10C6AA00EA933BDF1F910E2FEE81FF81A885B985A2
:10C6BA00EA0FFB1F1083EE81FF813196EE83FF8321
:10C6CA00003039F4EC85FD85AE81BF81AE17BF0716
:10C6DA0008F001C0D0CFEC85FD850E94587521F481
:10C6EA00F2DEE0E00C94C266A1DEA2CF68970E9457
:10C6FA00CF7C20E0E0E0EC8FED8F31E0A895E9A156
:10C70A00FAA1662777270E94A67BEA87FB876C87B0
:10C71A007D87EE8D0E949678EE83FF8368877987FE
:10C72A00AA85BB858C859D850E947C7CEA8BFB8BC8
:10C73A006C8B7D8B0E94007BFE017296FA93EA93C2
:10C74A000E94296BEE8BFF8B688F798F0E949C78F1
:10C75A000E946D7BAF010E949C78AE8DBB27882713
:10C76A0099270E94077B0E94AF78DE015A960E94A1
:10C77A006D7BED93FC930AA119A194DEE030D1F50B
:10C78A00EDA10E94726EB1F50E94917899F51A9303
:10C79A00B8DEE03079F5303051F14F5F5F4FEC8D04
:10C7AA00FD8D3196EC8FFD8FAC8DBD8D1197EBA170
:10C7BA00FCA1EA17FB0711F430E018C0EC8DFD8DDF
:10C7CA003197AF8DB8A10E9498759BDEEE8DDA0184
:10C7DA00F0E0EA17FB0751F476DEEA8DFB8DA9A19A
:10C7EA00BAA1EA0FFB1FE9A3FAA389CFD4CF6BDE64
:10C7FA00E0E002C01BDEC1CF0E94D67CA696089557
:10C80A00A881A03310F0AA3308F004C0E881E053ED
:10C81A000C94C168A881A13410F0A73408F004C0B0
:10C82A00E881E7530C94C168EFEF0C94C168A881C2
:10C83A00AA3020F4E881E05D0C94C168A881AA308E
:10C84A0020F0E881E95C0C94C168E8E50C94C168C1
:10C85A001A930A93F8940091620B1091630B7894DF
:10C86A00F8010C9437681A930A93F2DF8F01EA8170
:10C87A00FB81AC81BD81EA0FFB1FE01BF10BDF01DD
:10C88A000E94C57C14F4E0E001C0E1E0198108814E
:10C89A0026960895E4E6F8E0FA93EA93EAEBF0E0E4
:10C8AA00FA93EA930E948674E4E0EA93E6E2EA9352
:10C8BA00EEE0EA930E948F67ECEFF8E0FA93EA93CE
:10C8CA00EAEAF0E00E94B478E8E0EA93E0E2EA9368
:10C8DA00E1E0EA930E948F67ECEFF9E0FA93EA93BA
:10C8EA00E2EDF0E00E94A56BFA93EA93E2E0EA93A4
:10C8FA00E2E1EA93E1E0EA930E948F670E947E6B8D
:10C90A000E94D06DEFEAF0E00E94B478E3E0EA9387
:10C91A000E94D064EAE0F0E0FA93EA93E4E3F0E0FC
:10C92A000E94BB6DE0E0E0931004E4E5F8E10E94A8
:10C93A00E06CEFE0E093100408950895EA81F0E0D6
:10C94A00EBBBF5BBF7E1F09365001F98E6E1E093D6
:10C95A006500F0936500E881F981EBBBF5BBFFE167
:10C96A00F0936500EEE1E0936500F09365001F9A8D
:10C97A0023960895E2E2F0E0EBBBF5BBE7E1E09332
:10C98A0065001F98E6E1E0936500E7E1E093650042
:10C99A0008951F9A08950E94BB780E94FC7A8F011D
:10C9AA00AE85AA2362F0AD85BE85A03FE0E0BE0752
:10C9BA0034F4AB85BC85AF33E1E0BE070CF07CC034
:10C9CA00E985FA85AD85BE85AE0FBF1FA03FE0E0C1
:10C9DA00BE0744F0AD85BE85EFEEF0E0EA1BFB0B27
:10C9EA00E987FA87EF81F885AB85BC85AE0FBF1F53
:10C9FA00A034E1E0BE0744F0AB85BC85EFE3F1E08B
:10CA0A00EA1BFB0BEF83F8870E94C3780E94D27857
:10CA1A00E4E0EA93EA85FB850E94D678E5E0EA93AA
:10CA2A00EA85FB85AE85BF850E947A6C0E94A36465
:10CA3A000E94DE78E7E0EA93EC85FD850E94D278D1
:10CA4A00E8E0EA93E885F9850E94E578E9E0EA9367
:10CA5A00E885F985AC85BD850E947A6C0E94A3643D
:10CA6A0089DF0BBB15BB2EE13FE100E010E0EF814F
:10CA7A00F885E017F1078CF040E050E0E985FA8587
:10CA8A00E417F5073CF020936500309365004F5F8B
:10CA9A005F4FF4CF0F5F1F4FEACF7BDFE4E0EA93EB
:10CAAA000E947E6B0E94ED780E94836B0E94F2784E
:10CABA000E94F8780E94FD7860C10E94BB780E94AB
:10CACA00FC7A8F01E985FA85AD85BE85EA17FB07F1
:10CADA0011F00C94CC650E94007914F40E94077935
:10CAEA00E6E1EA93E8E2F0E00E94D278E4E0EA9331
:10CAFA000E94DB6C0E94ED780E94FD78E8E0EA93E0
:10CB0A000E947E6B0E94F8780E94836B0E94A36445
:10CB1A00E2E0EA93EC85FD850E941879E3E00E9441
:10CB2A001B79E6E0EA93EE85FF850E941879E7E033
:10CB3A00EA93EE85FF85F0700E94D2781BDF0BBB6B
:10CB4A0015BB2EE13FE10B851C85EF81F885E017C7
:10CB5A00F1073CF020936500309365000F5F1F4F8B
:10CB6A00F4CF17DFE6E1EA930E94D86B0E94A36430
:10CB7A00E4E0EA930E947E6B0E94ED780E94836B48
:10CB8A000E94F2780E94F8780E94FD78F6C0EF8140
:10CB9A00F885AB85BC85EA17FB0731F50E94207939
:10CBAA0014F40E9407790E94C378F0700E94D27828
:10CBBA000E94DE78E7E00E941B790E94BF640BBBEB
:10CBCA0015BB2EE13FE10D851E85E985FA85E01743
:10CBDA00F1073CF020936500309365000F5F1F4F0B
:10CBEA00F4CF0E94CE64C9C00E9427790E9496762B
:10CBFA00FF93EF930E942E790E949676AF91BF9190
:10CC0A00EA17FB0710F40C9454660E94007934F575
:10CC1A0020E030E00E943179E217F307F4F00E9435
:10CC2A0027790E9438790E9431790E943D790E94C1
:10CC3A004579E6E0EA93AC85BD85A21BB30BFD01FD
:10CC4A000E941879E7E0EA93AC85BD850E94517984
:10CC5A000E9458792F5F3F4FDDCF20C020E030E09F
:10CC6A000E942E79E217F307CCF00E9427790E94DE
:10CC7A0038790E942E790E943D790E944579E6E032
:10CC8A00EA93F9010E94E578E7E0EA93F9010E9444
:10CC9A005E790E9458792F5F3F4FE2CF6EC00E94A3
:10CCAA0027790E949676FF93EF930E942E790E942D
:10CCBA009676AF91BF91EA17FB0710F00C94C26603
:10CCCA000E94207964F520E030E00E946779E2173B
:10CCDA00F30724F10E942E790E9438790E9467791D
:10CCEA000E946E79AE85BF85A21BB30BFD010E941F
:10CCFA001879E3E0EA93AE85BF850E945179E6E0B0
:10CD0A00EA93FA010E94E578E7E0EA93FA010E94C1
:10CD1A005E790E9458792F5F3F4FD7CF2EC020E00F
:10CD2A0030E00E942779E217F3073CF10E942E793E
:10CD3A000E9438790E9427790E946E79F9010E942F
:10CD4A00D678E3E0EA93F901AE85BF85AE0FBF1F3F
:10CD5A00EFEFF0E0EA23FB230E94D278E6E0EA93C1
:10CD6A00FA010E94E578E7E0EA93FA010E945E7907
:10CD7A000E9458792F5F3F4FD4CF0E94D67C2F96BE
:10CD8A0008950E94CF7CEC85FD85309711F40C94B0
:10CD9A008B6700910D0410E0E0910E041E1710F04D
:10CDAA000C945167E6E0EA93E985FA850E941879BE
:10CDBA00E7E0EA93E985FA85F0700E94D2782C853B
:10CDCA003D854A855B85022E032A11F40C94496736
:10CDDA0037FF4CC0E2E0EA93FA010E941879E3E0D7
:10CDEA00EA93FA01F0700E94D278E2E2EBBBE0E04B
:10CDFA00E5BBE7E1E09365001F98F6E1F093650073
:10CE0A00E0936500EE81EBBBEF81E5BBEFE1FEE16C
:10CE1A00E0936500F0936500E0936500023050F0FE
:10CE2A00F0936500E0936500033020F0F09365000D
:10CE3A00E093650036FF19C0F0936500E093650042
:10CE4A00023070F0F0936500E09365004F5F5F4F2A
:10CE5A00033030F0F0936500E09365004F5F5F4F59
:10CE6A00220F331F4F5F5F4FE5CF1F9A220F331FE9
:10CE7A00023010F04F5F5F4F033010F04F5F5F4F8B
:10CE8A004F5F5F4F0C94E866E885F9853196E8872D
:10CE9A00F9871F5F0C94D16639C022970E94CF7C14
:10CEAA00E8850E9475790E94FC7AEE83FF83E98502
:10CEBA00A8E1EA9FF001E05EF54F8F0130E03830DB
:10CECA0028F5F801E4915E2F0F5F1F4FF801E491F6
:10CEDA004E2F407F0E947A790E947F79EA87FB87EA
:10CEEA00F801E4914E2F440F440F440F440F0F5F93
:10CEFA001F4FF801E4915E2F0F5F1F4F0E947A794E
:10CF0A000E947F79EA87FB873F5FD9CF0E94D67C50
:10CF1A002E96089524970E94CF7CEA850E947579FF
:10CF2A000E94FC7AEE83FF8300E010E0EB850E940A
:10CF3A009375C4F5EF85F889E887F98720E030E032
:10CF4A00EC850E9440781CF5E989FA8944915527B5
:10CF5A003196E98BFA8B5A934A930E94576CE98966
:10CF6A00FA89FA93EA93EC85FD85FA93EA930E948B
:10CF7A00C666E0910D04EE0FEE0FEE0FA885B98597
:10CF8A000E941274E887F9872F5F3F4FD9CFE0914B
:10CF9A000E04AD85BE850E941274ED87FE870F5F71
:10CFAA001F4FC4CF0E94D67C639608951A930A93A2
:10CFBA00EFE1E09365000E94576EEBE1E0936500B4
:10CFCA00E4E6F0E00E94BF6DEFE1E0936500E8EC73
:10CFDA00F0E00E94BF6DE8EFFFEFE093DE0EF09302
:10CFEA00DF0EE491EF3F39F0E091DE0EF091DF0EB3
:10CFFA00049000920403E0E4F6E18F01F801E49161
:10D00A00ED3F39F4F80131960E94E46C0E94C97927
:10D01A0019C0EC3F71F4F80131960E94FC7ADF01E5
:10D02A00E0910403F0E0EA17FB0711F00D5F1F4FD0
:10D03A0009C0F801E491EA93F80131960E94E46C80
:10D04A000E94A3640D5F1F4FF801E491EF3FB1F610
:10D05A000E94976CE1E0E0930E04E0930D04E4E192
:10D06A00E093130409911991089599818881009692
:10D07A0041F0BD81AC81FB81EA8105900D92019757
:10D08A00E1F7FD81EC810C94556BB981A88110966A
:10D09A0031F0FC81EB816A8161931197E9F7EB81A9
:10D0AA00FC8125960895E991F991A991B9911D906C
:10D0BA000590011421F40020D1F7EE2708951018E5
:10D0CA00E1F3E1E008F4E2500895E991F991A991B8
:10D0DA00B991CD0161916D936623E1F7FC01089541
:10D0EA00E991F991A991B991CD0105900D9200208C
:10D0FA00E1F7FC010895A991B991EE27FF276D91F7
:10D10A00662311F03196FBCF0895AA27BB27E99130
:10D11A00F9910590002011F01196FBCFFD010895B9
:10D12A007991E991F991A991B991CD01772351F0BA
:10D13A007A9561916D936623C9F7772319F07A95E9
:10D14A006D93FBCFFC0108956991E991F991A99139
:10D15A00B991CD01662351F06A9505900D92002090
:10D16A00C9F7662319F06A950D92FBCFFC01089561
:10D17A005D9BFECFE881ECB9219608951A930A9334
:10D18A00AC81BD810E94ED7A3097C1F0AA81BB8142
:10D19A000E94ED7A8F01309749F00230E0E01E07D5
:10D1AA0060F0F80131978F01ED93FC93AC81BD815A
:10D1BA000E94E46D3197AE81A08303C0EE81EA93A9
:10D1CA00D7DF19810881279608952C970E94CF7C72
:10D1DA0010E0E88DF98D3196E88FF98F3197E49157
:10D1EA002E2FE03011F40C94A86AE12FE03039F4C4
:10D1FA00253211F411E002C00E948C79A3C1E130FA
:10D20A00C1F4253219F40E948C799BC112E0E0E046
:10D21A00E98B00E02D3211F401E094C12B3219F4AC
:10D22A00EBE2E98B8FC1203219F4E0E2E98B8AC183
:10D23A0002C0E23039F450E013E0203311F4006800
:10D24A0081C102C0E330A1F4203310F02A3308F080
:10D25A0009C0A52FEAE0EA9FF0015E2FE22FE05312
:10D26A005E0F70C140E02E3211F414E06BC110C0A1
:10D27A00E430A1F4203310F02A3308F009C0A42FB7
:10D28A00EAE0EA9FF0014E2FE22FE0534E0F5AC117
:10D29A002C3619F4026015E055C104C0E53011F0CE
:10D2AA000C94A76AE22FE33649F40E949779EE8933
:10D2BA00FF89A481AA930E949D7943C1E33741F46F
:10D2CA000E9497790E94A7790E9480681E2F0AC03F
:10D2DA00E037A1F40E9497790E94A7790E948A6890
:10D2EA001E2F08600F77403011F0411708F001C077
:10D2FA00142F40E0E0E0E88B30E076C0E43611F02D
:10D30A00E93611F4046002C0E537A1F4EAE0E88BDB
:10D31A0001FF08C0E0E0FAEC6AE97BE30E949E6D37
:10D32A001AE023C0E0E1F7E260E070E00E949E6D3F
:10D33A0015E01BC0E83511F4086004C0E83711F0A5
:10D34A000C94A66AE0E1E88B01FF08C0E0E0F0E097
:10D35A0060E070E10E949E6D18E007C0E0E0F0E135
:10D36A0060E070E00E949E6D14E0403011F00F778B
:10D37A0001C041E001FF08C00E949779AE89BF89C8
:10D38A0014960E94F17A13C002FF08C00E9497798E
:10D39A00AE89BF8914960E94346D09C00E9497799C
:10D3AA00AE89BF8914960E94ED7A66277727EC87A3
:10D3BA00FD876E877F8702FF16C0AF85AA2362F4B6
:10D3CA00EC85FD856E857F850E94E779EC87FD8770
:10D3DA006E877F87EDE2E98BE989E03019F01F5FFC
:10D3EA004F5F01C00B7F342F00FD14C0151710F4D6
:10D3FA00351708F00FC007FF08C002FF04C00B7FF3
:10D40A002989115001C020E301C020E20E948C79D1
:10D41A005150ECCF1417B0F4006102FF0AC00B7F21
:10D42A00E989EA930E949D79503009F051501150D0
:10D43A004150E0E3EA930E949D79503009F051503F
:10D44A004150E8CF312FE889E030D1F43030B9F0DB
:10D45A0003FF08C0EE81FF813196EE83FF83319787
:10D46A00E49105C0AE81BF81ED91AE83BF83EA939B
:10D47A000E949D79503009F051503150E7CF57C082
:10D48A000E94AF790E94797A2E2F2A3030F003FF5A
:10D49A0002C0295C01C0295A01C0205D04FD25C0D3
:10D4AA00213360F4A885B9858A859B85A130E0E09F
:10D4BA00BE07E0E08E07E0E09E0709F40BC04317C1
:10D4CA0040F4531710F000FF01C014C020E207FF18
:10D4DA000CC020E3006102FF08C00B7FE989EA93D0
:10D4EA000E949D79503009F051500E948C79503039
:10D4FA0009F0515031500E94AF790E94B47AEC87FA
:10D50A00FD876E877F87E889A885B9858A859B8587
:10D51A00FF27662777270E94797A0E949E6DE88501
:10D52A00F9856A857B850E94C17C09F0A9CF00FF35
:10D53A0008C0503031F05150E0E2EA930E949D79E0
:10D54A00F8CF10E046CE0E94D67C6A960895FF92E4
:10D55A00F82E22971A930A93DE010E94D5798D013B
:10D56A00DE0116960E94D5790E94ED7AEA83FB8342
:10D57A00DE0114960E94D5790E9438731A930A9391
:10D58A00FE0136960E94AA6B20DEAA81BB81E0E0EA
:10D59A00EC93198108812496FF9008957B816A8112
:10D5AA00F981E88177FB770F67FD7160972F9E57A6
:10D5BA0081F078F0983190F4AA27BB27882708943D
:10D5CA008795B795A7959A95D1F7EA23FB23682300
:10D5DA0005C0E8947727EE27FF2766276F777695A9
:10D5EA0008F4606877F9A991B99189919991EA1734
:10D5FA00FB076807790797FB08950E9461780E94E4
:10D60A00B87919F40E94BF791DC0E6F7A881B981DB
:10D61A008A819B81E0E0F0E060E87FE30E94AF78D6
:10D62A0011C00E9461780E94B87919F40E94BF79EA
:10D63A0009C0E6F30E94BF79A0E0B0E080E89FE36A
:10D64A000E94E07B249608950E94C4790E94C17CBE
:10D65A0039F4A881B9810E946B6F0E94F77A20C0C1
:10D66A00AA81BB818C819D810E94C97C34F40E946D
:10D67A00C4790E94007BC1DF05C00E94C4790E9460
:10D68A00007BCFDFA881B9810E94F77AA881B9818E
:10D69A000E94F17AAA81BB818C819D810E94AF7818
:10D6AA0026960895E991F99130971AF4E095F09544
:10D6BA00319608950E943662E0EBEA93E8E1F0E0E1
:10D6CA00FA93EA93E1E0F0E0FA93EA93E3E2F7E00F
:10D6DA00FA93EA930895E0EBEA93E0E0F0E0FA9334
:10D6EA00EA930E94C8620C943862E0E2EA930C94CE
:10D6FA007B63E0E0F0E0FA93EA930895EFEEF0E05E
:10D70A00FA93EA930895FA93EA93E0E0EA930C9481
:10D71A00D064FA93EA930C94F142E12FA6E3B3E0C2
:10D72A00F0E00E94FB79EA0FFB1F0895A12FB0E0F9
:10D73A00ECE3F0E00E94497A3896FA93EA93089566
:10D74A00FA93EA93E2E3F0E00895FA93EA93D1CFE9
:10D75A00E0911004E0930F0408950E94980C0C9431
:10D76A00A248E32FF0E0EE5AFC4FE4910895EA93C1
:10D77A000E94AE0CFE013696FA93EA930895FF27AB
:10D78A00662777270E94007B84E00E94AC6A28966D
:10D79A000895FE017196FA93EA930C9410430E943D
:10D7AA00D17C0C941946E8E0F0E0FA93EA930895E4
:10D7BA00E4E0F0E0FA93EA930895FA93EA93E8E34F
:10D7CA00F0E0FA93EA9308950E94FC7ABECFE02F24
:10D7DA00F0E00895A0913A0CB0913B0CBD01A3E092
:10D7EA00B0E00E94217AE60FF71FE491E030089535
:10D7FA00E091C005EE0FEE0FEF5F3E2F0895E32F85
:10D80A00F0E00895A12FB0E00895A0913A0CB091EC
:10D81A003B0CBD01A3E0B0E00E94217AE60FF71F9E
:10D82A0008950E94F979EA54FD4F0895FA93EA930C
:10D83A00E22FF0E008950E94CF7CA0911908089584
:10D84A00E091C20BF0E00895AFE3B1E00E94747A70
:10D85A00089530911E08E1E0E0930D04E2E0E093C0
:10D86A000E043A930E941718E091980BE295EF7014
:10D87A00E0930F04E091980BEF70E0931004089581
:10D88A00FA93EA93E52FF0E0FA93EA930895E7E32F
:10D89A00F0E0FA93EA930895E22FE450F0E0FA9365
:10D8AA00EA930895EA85FB85FA93EA930895E32FAC
:10D8BA00E058EA931ECFEAE8FBE0FA93EA930C9465
:10D8CA0010433A930E941718A0918A0BAD3208951B
:10D8DA00E091980BE295EF70E0930F04E091980BBA
:10D8EA00EF700895E52FF0E00895EA0FFB1FFA9311
:10D8FA00EA930895EF5EFC4FBF01E081E058DB0137
:10D90A00EC930895E0E0EC93AE81BF810895E3E0E3
:10D91A00F0E0FA93EA930895E52FE450F0E0FA93E1
:10D92A00EA930895E0E0E0930F04EFE0E093100437
:10D93A000895E550F0E00895E091980BE295EF70B4
:10D94A000895EA1BA2E5B7E0F0E00E94FB7908958A
:10D95A00F0E0EE0FFF1FE85BFC4F0895A6E4B3E08A
:10D96A00F0E0EE0FFF1FEA0FFB1F0895FA93EA9308
:10D97A00E12FF0E0FA93EA9308950E941946E0E055
:10D98A00EA930895E12FF0E0FA93EA930895FA935F
:10D99A00EA93E2E0F0E0FA93EA930895EAE8FBE01A
:10D9AA00FA93EA93EAE0EA930C94B845E1E0F0E0EE
:10D9BA00FA93EA930895FA93EA930C94A1450E9484
:10D9CA00FC7AFA93EA930895ABE0EA9FF001E252F7
:10D9DA00FA4F08951A930A9333CF1A930A93E0E001
:10D9EA00EA930E94D064E2CFE1E0E0933C0C0E940B
:10D9FA002D64E0933E0CF0933F0C0895BD01AAE01C
:10DA0A00B0E00E94217AE60FF71F0895FA93EA938D
:10DA1A00EAE0EA930C94B845E1E0E0930E0469CE9B
:10DA2A000E94F2450C94D345E0E2EA930C948B45AC
:10DA3A00A3E2B7E0E881F0E0EE0FFF1FAE0FBF1FD1
:10DA4A000E94ED7A0895FA93EA930C94A240E88131
:10DA5A00F0E00895EE0FFF1FAE0FBF1F08950E945A
:10DA6A00ED7A0E940B7A08950E94007B0C94834001
:10DA7A00FA93EA930C94F245A9E0B0E00E941B7B6A
:10DA8A000895A7E11A9FF001EF5CF94FE08108952C
:10DA9A00E12FEF5FEA930C94B840F0E0D4CFE8E0CE
:10DAAA00F0E053CEEA93E6E0EA930E946E407BCE22
:10DABA00E093620088EC90E00197F1F70895E09313
:10DACA00610088EC90E00197F1F70895E0916D0507
:10DADA00F0916E050895E0916905F0916A0508953F
:10DAEA00AE0FBF1FE3E0F0E00E94747A0895FA9344
:10DAFA00EA931A930A930C94D311FA93EA933A93FA
:10DB0A002A930C94D311A0917105B09172050895CE
:10DB1A00A0917305B09174050895A0E0B0E00E9449
:10DB2A00177B08950E94107BEA1BFB0B0E940B7A5D
:10DB3A000895E887F9876A877B870895A885B98554
:10DB4A008A859B85EFEEF0E060E070E008950E9420
:10DB5A000B7A0E949E7A0895A4E0B0E00E94177B97
:10DB6A000895EC83FD836E837F830895FA93EA9385
:10DB7A000C940D46FA93EA930C94C979A9E01A9F7A
:10DB8A00F001EA50FC4F089537960E94FC7ADF01B3
:10DB9A000E94ED7A0895E2E3F0E0FA93EA93089599
:10DBAA000A921A92FA926A937A938A939A93AA9306
:10DBBA00BA93EA93FA93EFB7EA931A930895ED9119
:10DBCA00FD913196FE93EE930895ADE01A9FF00110
:10DBDA00EB5FFC4FE08108951A93E1E0EA930C941D
:10DBEA007C46ADE01A9FF001DF01EB5FFC4FE0815C
:10DBFA00E0300895E2E0EA930C947C46FA93EA93C3
:10DC0A00E4E6F0E0FA93EA930E943864E03008957B
:10DC1A00E1E0E0930D04E0930E040895E0912808F2
:10DC2A00F091290860912A0870912B080895E091D3
:10DC3A002008E150A3EAB6E0F0E00E94FB79AE0FBB
:10DC4A00BF1F0E94F17A0895E12FEF5FF0E010CF35
:10DC5A00E0912108EA93E0911E08EA930E94241AAF
:10DC6A00A0911E0CB0911F0C10970895A091200C42
:10DC7A00B091210C8091220C9091230C0E94C97CB6
:10DC8A000895E0911E0CF0911F0C0895E091200C6C
:10DC9A00F091210C6091220C7091230C0895EAE016
:10DCAA00F0E068CFE2E3F0E065CF1A93E0EAEA93A6
:10DCBA00EA81F0E0E054F14FFA93EA930E94C862D5
:10DCCA001E2F0895E0EAEA93EA81F0E0E054F14F6A
:10DCDA00FA93EA931A930C94F562EA930E947A6291
:10DCEA00E0300895E0EAEA93EEE5F0E0FA93EA9389
:10DCFA00E0E0FFE0FA93EA93EEEBFBE00895FA9393
:10DD0A00EA93F3CCE0EAEA93E981FA81E050FE4E25
:10DD1A00FA93EA930895EA81F0E0A8E2B0E00E945B
:10DD2A00497A0895E0EAEA93E2E0F0E0FA93EA93A6
:10DD3A001A930A930895FA93EA930C941663FA9342
:10DD4A00EA930C94C862E0EAEA93E8E2F0E0FA9314
:10DD5A00EA931A930A93EAE8FBE00895EAE8FBE0FB
:10DD6A00FA93EA930895EDE2EA93EAE0F0E0FA938F
:10DD7A00EA930E944A68E0E00895EA81F0E0ABE0A5
:10DD8A00B0E00E94497AE050F24F8F01AA81AA308E
:10DD9A000895E0EAEA93EBE0F0E0FA93EA931A9343
:10DDAA000A93E2EBFBE00895E3EBFBE0FA93EA93D4
:10DDBA000895EA81F0E0EE0FFF1FE050F04F8F0167
:10DDCA00AA81A0380895E150F0E00895EA81F0E0D0
:10DDDA000E94FB79E058F14F8F01AA81A53008957E
:10DDEA00EFE2FCE0FA93EA93E0E0EA93E1CCECE1BB
:10DDFA00FCE0FA93EA93E0E0EA93D5CC0E94FB793F
:10DE0A000E94F779DF01EA85F0E0AE0FBF1FE8E074
:10DE1A00F0E00E94497AE050FA4E8F01E0EAEA9374
:10DE2A00C2CC1A930A93ECE1FCE085CFAE81BF81A4
:10DE3A00888599850E94D979EE83FF8368877987D7
:10DE4A00089540931E0C50931F0CEE81FF81688544
:10DE5A007985E093200CF093210C6093220C709347
:10DE6A00230C0895F0E0AE0FBF1F0895EA930E94B5
:10DE7A0017180C94E61EE091950BF091960B0895F5
:10DE8A00FA93EA930C94B617ED81EA93ED81EA933B
:10DE9A000895E091AC0BF091AD0B0E940B7A0895B6
:10DEAA00E0912608F09127080895E093270CF09353
:10DEBA00280C0C947C1BE3EAF6E0FA93EA93E0E080
:10DECA00EA930895FA93EA930C944A68E0E0F0E042
:10DEDA0060E070E00895E0932808F09329086093C1
:10DEEA002A0870932B080895E091970BA3EAB6E0ED
:10DEFA00F0E00E94FB790895AE0FBF1F0E94F17AED
:10DF0A000895ED5EF94FE081E1300895FA93EA93BE
:10DF1A00E0912108E05DEA930895EA930E94C15FC7
:10DF2A00E1300895EBE3F8E0E0935F0BF093600BC8
:10DF3A000895E12FA3EAB6E0F0E00E94FB79089584
:10DF4A00A881AF5FEAE00E94537AE05D0895A88154
:10DF5A00AF5FEAE00E94A37AE05D0895FA93EA933C
:10DF6A00E0E0EA930895AAE0B0E00E941B7B0895DE
:10DF7A00E12FF0E00E94F979EE52FF4F32960E94AB
:10DF8A00FC7A0895E12FF0E00E94F979EE52FF4FF2
:10DF9A0008953696E491D901EC930895E0EAEA935C
:10DFAA00E5E0F0E0FA93EA930895EA930E946D1B84
:10DFBA00FA93EA93E4E2FCE00895FA93EA93EFEF26
:10DFCA00EA93E5E0F0E07ECFE093250CF093260C8F
:10DFDA0008950E94107BEA1BFB0B0895E9E2FCE01E
:10DFEA00ECCFA0912A0CB0912B0C0895E0E0E093BD
:10DFFA00380CE093390C0895A0912C0CB0912D0C9B
:10E00A000895E0912C0CF0912D0CAC81BD81EA0FA2
:10E01A00FB1F0895E0932C0CF0932D0C08951A938E
:10E02A000E94071C1E2F0895E0932A0CF0932B0CD4
:10E03A000895FA93EA930E943864E0300895ABE0B9
:10E04A001A9FF001E452FA4F08951A930E94F61D9E
:10E05A00D3CFE0912A0CF0912B0C0895EA930E94F9
:10E06A00F61D0E94931DE0300895EB81EA930E9409
:10E07A002E1CFA93EA93E9E2FCE008951A930A93B4
:10E08A00A09119080895E0E0E0934F0CE0934E0C3C
:10E09A0008951A930A93E0911208ABE0EA9FF001FF
:10E0AA00E752F84F8F01D80111960895E0E0F0E0A9
:10E0BA00ED93FC930895EA81D801EC93E2E1F8E04C
:10E0CA00FA93EA930E94D732198108810895E12FC1
:10E0DA00A6EAB0E0F0E0EE0FFF1FEA0FFB1F0E9476
:10E0EA00FC7A0895E150ADE0EA9FF0010895A6EAAE
:10E0FA00B0E0F0E0EE0FFF1FEA0FFB1F0E94FC7A70
:10E10A000895A0911608B0911708EA2BFB2BE0930B
:10E11A001608F09317080895E150A7E1EA9FF00165
:10E12A000895A7E10A9FF001E15DF94FAF01089553
:10E13A00F0E0A4E6B0E00E94497A0895ED55F94F5F
:10E14A00E081E0300895E981FA81FA93EA9308952B
:10E15A00E12FF0E00895E2E0F0E00E94747A089579
:10E16A00AAE9BBE0E0911A080895ADE9BBE0E091A5
:10E17A001A0878CEA0EABBE0E0911A0873CEA3E2AF
:10E18A00B7E0B0CBEE0FFF1FEA0FFB1F0895E08147
:10E19A00F0E00895A7E11A9FF001E15DF94FEE83DF
:10E1AA00FF83AE81BF810895EE81FF81A481AA9386
:10E1BA000C943C1F0D901C90AE81BF811296EC917D
:10E1CA00F0E0E00DF11DDB01ED93FC930895ED9174
:10E1DA00FD913197FE93EE9308950E94E120EF7727
:10E1EA000E2EAA85BB851296EC91E0150895A3E23E
:10E1FA000A9FF001E855F94F0895E0911208ABE043
:10E20A00EA9FF001E752F84FEC87FD87AC85BD85A0
:10E21A00119608951296EC91AC85BD851696EC93ED
:10E22A000895D001F0E00895A885B98518960E944E
:10E23A00ED7A0895AC85BD85EC93E2E1F8E0FA93B6
:10E24A00EA930C94D732E885F985A281AA930895B6
:10E25A00AA85BB85EC91EA93E3E0EA930C943C42ED
:10E26A00AA85BB85E0E0EC93E2E0E09324060895FA
:10E27A00BF0100801180AE81BF811296EC91089592
:10E28A00DB01ED93FC93AE81BF8112963BCBE4E6B2
:10E29A00F0E00E94497A0895F0E0ED93FC93089526
:10E2AA00E2E1F8E0FA93EA930C94D732E091190884
:10E2BA00A0911808EA170895F0E0E00DF11D0895FD
:10E2CA00A3EABBE045CFADE9BBE0EE27A10FBE1F35
:10E2DA00EC910895A0EABBE0EE27A10FBE1FEC91D6
:10E2EA000895BD01AAE0B0E00E94217ADB010895F9
:10E2FA00E081EA930C94175AEFE3FAE0E0935D0B9E
:10E30A00F0935E0B0895EA930E947F5EE0E0089521
:10E31A00EA930E947F5E0C94FF5FADE9BBE0EE27B3
:10E32A00A00FBE1FEC910895A0EABBE0EE27A00F54
:10E33A00BE1FEC910895AAE9BBE0EE27A00FBE1F0D
:10E34A00EC91E1700895A3EABBE041CAA0EBBBE0FF
:10E35A00EE27A00FBE1FEC910895A9EABBE0EE27B5
:10E36A00A00FBE1FEC910895EA81ADE0EA9FF0018B
:10E37A00E15FFC4FA0E0A083EA81EA930895ADE053
:10E38A00EA9FF001EB5FFC4F0895ABE00A9FF001B2
:10E39A00E452FA4F0895ABE00A9FF001EE51FA4FAA
:10E3AA000895FA93EA930C946434FA93EA930E94D8
:10E3BA00B2423A931FCCE0912C0CF0912D0C30977D
:10E3CA000895AFEFBFEFA083B18308950E942D6433
:10E3DA00E093540CF093550C0895FA93EA93E0E015
:10E3EA00F0E80895E0911208ABE0EA9FF001E752E5
:10E3FA00F84FFA93EA930E94492852CFE091100805
:10E40A00ABE0EA9FF0010895E0E1F8E0FA93EA93BD
:10E41A000C94D732FA93EA930C94A54EE88DABE0AC
:10E42A00EA9FF0010895FA93EA93D1C9E0E1EA93E9
:10E43A00E0912506EA930E94EA171E2F089530DD1F
:10E44A00FA93EA930895FA93EA930C94C11DE09320
:10E45A002506E0E0E093510CE1E3E093520C0E94C0
:10E46A0088290C945525FA93EA930C948F5EE0E47C
:10E47A00F9E0E0935F0BF093600BE3E0EA930C940E
:10E48A00255EA0915F0BB091600B08950E942D64E8
:10E49A00E093490CF0934A0C0895E0935F0BF093D4
:10E4AA00600B0895E3E0EA930C94255EE093260856
:10E4BA00F09327080895E0E0F0E0E0932408F09351
:10E4CA002508E2E0E0930E040895E091130431CAAE
:10E4DA00E0912408F0912508B6CAE0915D05F09113
:10E4EA005E0531970895FA93EA930C94E644A0E006
:10E4FA0024FCA1E0A0300895E7E0EA93E0E0EA9383
:10E50A00F8C8E0913208F0913308FA93EA93089533
:10E51A00FA93EA930E943864E13008950E942D64C8
:10E52A00E0933208F09333080895E0E0E0934E0C4C
:10E53A000895EF5CEA930C948B45A3EEB6E05FC9AD
:10E54A00A3EABBE0E0911A08F0E01CCE0E94ED7A43
:10E55A00D001ED93FC9304CEF0E0EA0FFB1F0F010C
:10E56A00FFCDA3E2B7E04BC9E0911908EA93E0E0D6
:10E57A00EA930C94002BEA930E9416400E944F42A1
:10E58A001E2F0895EAE2EA93E0E3F7E1E7CC0E945E
:10E59A00872BE1E0EA930C946F2B1F771A930C9464
:10E5AA001718A0912408B09125080895E8EEF3E021
:10E5BA000E94A67A0895E053F0E00895F2DFEA1780
:10E5CA00FB070895E0931808E0E0E0932F08089508
:10E5DA000E949F5F0E94A72CE093230808950E943F
:10E5EA0017180C9419460E94FB270E94C61E0E9407
:10E5FA004C42E03008950E944F421E2F1A930E9407
:10E60A00DA2C103808951A93E091C605EA93089512
:10E61A00E091890BEA930E942417E03008950E9442
:10E62A002D64E093560CF093570C0895FA93EA93ED
:10E63A00F7C9D90118960E94ED7A0895E4E6F0E048
:10E64A0060E070E00E949E7A08950E94171813CC29
:10E65A000A93E091C605EA930895E0912E08EA9399
:10E66A000A930C9448190E94ED7AFA93EA93089552
:10E67A00AFE5BBE0A4CAE0913B08E053E093210870
:10E68A000895FA93EA93E0E3EA930C949F5FE0918A
:10E69A003808EA930C944C5F0E940B7A0E94007B24
:10E6AA0008950E94075FEBE3EA930C947F5EE89477
:10E6BA0023F8E0E0F0E0FADEE0E0E0931E080A93D7
:10E6CA00E1E0EA930C94002BE89423F8E0E0F0E010
:10E6DA00EDDEE0E0E0931E08EA930C946F2BE091E4
:10E6EA001208ABE0EA9FF0010895A881B981EC9184
:10E6FA00EF5FEC930895ABE00A9FF001E352FA4F03
:10E70A000895A083ABE00A9FF0010895ABE00A9F49
:10E71A00F001E152FA4F0895EDE4F7E1FA93EA9332
:10E72A00EA85ABE0EA9FF0010895AC81BD81EE274E
:10E73A00A00FBE1F0895E02FAC81BD81F0E00895BF
:10E74A000E94007B84E00E94AC6A28960895EE2716
:10E75A00A30FBE1FEC91D001EC930895A2E5B7E098
:10E76A000C94046C0E94FB79EA0FFB1FAF01089519
:10E77A00E0912C0CF0912D0C0895E32FA0911E0826
:10E78A00EA0F0895ADE02A9FF001E35FFC4F089578
:10E79A00A8E0B0E00E941B7B0895F0E0FA93EA93A8
:10E7AA0008950E94C0410C948D41F0E00E94FB79CB
:10E7BA0008950E94007B0E94AA410C948D410E94F8
:10E7CA00C041E0E5F7E1CACB0E948D410C948D412E
:10E7DA0020E030E0E12FE05DEA93E3E5F7E196CB54
:10E7EA00EAE0EA930C94605EE3E4FBE0FA93EA93CE
:10E7FA00089510915D0500915F0508950E944F42AA
:10E80A003E2F0C943445EAE0F0E00E94497A0895DC
:10E81A00DF01EE27A30FBE1F0895F0E0EA0FFB1FEA
:10E82A000895E02FA4E2B2E0C0CFEA0FFB1F3296B0
:10E83A00E4910895FA93EA93E0911B0CEA930E94FB
:10E84A00AB37E1320895EA930E945137E1320895D5
:10E85A00E6E0F0E00C94AA6BEAE3EA930C948B45A9
:10E86A000E94F245AAE9BBE0EE27A10FBE1FEC9178
:10E87A00E1700895EE0FFF1F0C947A6CEA930E94E0
:10E88A00AB37E13208950E94C10C0C947E6B0E9452
:10E89A00007B0C949740EEE5F7E08DC8EA23EA93F3
:10E8AA000E94BE40C1C8EA930E94BE40BDC8DF01B3
:10E8BA00329685C80E94F979EE52FF4F0895ECEC22
:10E8CA00F7E0E0933A0CF0933B0C08950E94A819E4
:10E8DA00E0E0E09320080E94EA140E94C10CE1E003
:10E8EA00E0931B0808950E9419460E94630F0E9434
:10E8FA004F420E2F0D330895EE81FF81FA93EA936A
:10E90A000895E5E0F0E0FA93EA930895E0E0EA93E7
:10E91A000C947E6BEAE2EA93E5E6F7E10895EA935E
:10E92A000E943A150C94C10CE093C105F093C205FC
:10E93A000895FE01FA93EA930895E6E7F7E1FA9358
:10E94A00EA93EE85FF8568897989FACEEAE7F7E1E5
:10E95A00FA93EA93AE85BF85888999896FCE0E941A
:10E96A00007BAA89BB898C899D89E4E6F0E060E096
:10E97A0070E00E94B87A0E94007B88E00E94AC6A2C
:10E98A002C960895E3E8F7E1FA93EA93EE85FF857A
:10E99A0083CE84E00E94AC6A2896CBCFFA93EA939E
:10E9AA00EE85FF8508950E94665F0C942D6484E0CD
:10E9BA000E94AC6A28960895EE27A10FBE1FEC911B
:10E9CA000895EA930E9429411F5F0895E091C405C2
:10E9DA00A7ECB5E0F0E00895AF5FEAE00E94A37A01
:10E9EA000895E091C305A7ECB5E0F0E0CBCBA0E039
:10E9FA00A083E981ADE0EA9FF0010895EF73A5E1F4
:10EA0A00EA9FF001E051FB4F0895EF73ABE0EA9FF4
:10EA1A00F001EC5EFB4F0895AC81BD81EE27A30F98
:10EA2A00BE1FAC91A0300895ABE00A9FF001EC5EE6
:10EA3A00FB4F0895EA0FFB1F0F01AC81BD8187CE02
:10EA4A00A5E10A9FF001E051FB4F0895EE81FF8195
:10EA5A0001801280AE81BF8115960E94ED7AD001A5
:10EA6A000895FE013896FA93EA930895EAA5FBA55C
:10EA7A00FA93EA930895FA93EA93FE013A96FA937F
:10EA8A00EA930E946A6830E0E02F0895E091C10598
:10EA9A00F091C2050895A1ECB5E0ED91FD91329691
:10EAAA00FE93EE930895AE81BF81EA17FB0708959E
:10EABA00E0E0E0936505E093660508951A930A93EA
:10EACA003A932A930895FA93EA93E0910E040895EB
:10EADA00A0910003B09101030895E0910003F09121
:10EAEA000103FA93EA93E0910203F0910303FA9384
:10EAFA00EA930895E0930003F09301030895A9812E
:10EB0A00BA815ACFF801AA81BB81EA0FFB1FE491AF
:10EB1A000895AE0FBF1FAC91A0300895D801F0E060
:10EB2A00AE17BF070895AE0FBF1FEC91EA93089581
:10EB3A00A0910E04E4E1EA9FF0012E2F3327CDCFF6
:10EB4A00E0E0EA930E94D0640E94D87C0895ECE049
:10EB5A00EA9FF001A0910D04EA9FF00108951A932B
:10EB6A00E1E0E0930E04E0930D0410E00895EF81D4
:10EB7A00F885EA1BFB0B0895EA9FF001F0E008957F
:10EB8A003A932A935A934A930895EAA5FBA5E20F6A
:10EB9A00F31FFA93EA930895ECA1EA930C94626541
:10EBAA003A932A93EEA1FFA1E40FF51F0895FA9371
:10EBBA00EA93EBCFEAA5FBA5E40FF51FFA93EA93D4
:10EBCA00EBCFE20FF31FFA93EA930895FA93EA93CD
:10EBDA005A934A930895EA9FF001AEA1BFA1F0E0CB
:10EBEA000895E2E0E0930E04E0E2F0E0EAA3FBA37A
:10EBFA000895AE1BBF0BAFCAEE8DF0E00895E20F89
:10EC0A00F31F3196FA93EA93ECA1FDA1E40FF51FE5
:10EC1A0031960C94BB6DECA1FDA1E40FF51F0C9489
:10EC2A00BB6DE9A1F0E0DE0116960895ED8DEA9339
:10EC3A000E944145E9A1EF5FE9A30895E15CF54F20
:10EC4A0057CBE091370CA091360CEA170895E09162
:10EC5A001108ABE0EA9FF001E655F84F0895F096E7
:10EC6A00EA930E944C5FE2E7EA930C947F5EEA9390
:10EC7A000E947F5EEEE0EA930C947F5EE6E9F7E19C
:10EC8A00F2CBE0911108ABE0EA9FF0010895FA9304
:10EC9A00EA930C94B15EEBE3EA930C947F5EEC5535
:10ECAA00F84FDF01E0CCE0E3EA930C947F5EE09159
:10ECBA001008A0911108EA170895E1E1F8E0FA9323
:10ECCA00EA930C94D732EA930E947F5EE2E0E093E3
:10ECDA003408D7CFED55F84FA2E0A0830C94FC4836
:10ECEA00E3E0EA930E94EA5ECCCFA091250CB091B2
:10ECFA00260C0895E2E5EA930E947F5E0C94FC4894
:10ED0A001A93E985FA85FA93EA930895E552F84F3A
:10ED1A00A885B985A083B183E2CCE2E5EA930C9495
:10ED2A007F5EFA93EA930C94576B1A93E091380832
:10ED3A00E0531E2FECE3F8E0B0CBE0911208A0916B
:10ED4A001308EA170895E3E1F8E0FA93EA930C94BA
:10ED5A00D732E0911308ABE0EA9FF0010895A09141
:10ED6A00740B3ACEE093740BEAE2EA930E944C5F8A
:10ED7A00D4CFE091740BE05A7ACFD9011696EC9170
:10ED8A000CCD0E94B15E87CFF901A281B381BA93FB
:10ED9A00AA9308950E94B15EEAE3EA930C947F5E17
:10EDAA00D9011196E0E0EC930E94665FCCCFD901BD
:10EDBA00EC91F3CCE05DEA930C947F5EE05DEA931C
:10EDCA000E944C5FAACFEB58F44FE081E05D4FCF31
:10EDDA00EAE3EA930E947F5EF9010895E0935E0CEC
:10EDEA00F0935F0CE2E0E0933508D9011196EC93B9
:10EDFA000895EA930E944C5F90CF0E94B15ED3CDF2
:10EE0A00E091190CDBCFE091190CF0E0DCCFE8813E
:10EE1A00F9813DCFECE2EA930E947F5EF8CF31DBC5
:10EE2A00AC91A0330895A0915D0BB0915E0B08954B
:10EE3A00EE81FF81E093270CF093280C1093240CA9
:10EE4A000E947C1BE1E3089541E050E00E94AF5D1F
:10EE5A00E887F987EAE3EA930E94245DE13008959E
:10EE6A001A93E985FA85B2CEE2E2EA930E94245D1A
:10EE7A00E030089506DBAC91A032089502DBAC9134
:10EE8A00AB330895FEDAEC91EA930895EAE3EA9344
:10EE9A000C94245D0E94AF5D3197E887F987E88575
:10EEAA0008950E94ED7AE40FF51FD001ED93FC93CB
:10EEBA000895E0913F0BF0E0ED55F94F0895E0E039
:10EECA00E093650CE093660C08950E94AF5D31975C
:10EEDA00E0933F0BE091580BA0913F0BEA1708957E
:10EEEA000E946552E0913F0BEA930895ECE2EA939F
:10EEFA000E94245DE0300895ED5BF44F0F01C1DA02
:10EF0A00EC91D001EC931F5FB3CBED5BF44FA0E023
:10EF1A00A0830895EA930E94245DE1300895E09168
:10EF2A00400B7BCCE091400BEF5FE093400B0895E0
:10EF3A00A3EABBE0E091400BF0E024C9AAE9BBE0F8
:10EF4A00E091400B0C94376FE091400BF0E008958C
:10EF5A00E2E2EA930C947F5EFA93EA930C94D54E1C
:10EF6A00E0913F0BF0E0A6CC0E94B15EECE2EA939E
:10EF7A000C947F5EECE2EA930C947F5E0E94CA4E88
:10EF8A00E0E0E093400B0895E091400B0C94376F5A
:10EF9A00E0915F0BF091600B0895ADE5BBE00C9436
:10EFAA00E46D41DFEC93F9CFE0E0EA930E942E4F43
:10EFBA00E09334080895EA930E947F5E0E94F34E1C
:10EFCA00E1300895AA81BB81EC91E295E07FAE2FF2
:10EFDA00EC810895EA0FAA81BB81EC9386CBE0917C
:10EFEA00060DA091050DEA170895E0913A09F0E09F
:10EFFA00E15CF64F08951083E0913A09EF5FE093E0
:10F00A003A09E12FA0913C090895E0933C09E09167
:10F01A003B09E150E0933B09E0300895E15CF64F8B
:10F02A00A0E0A0830895E091D10DF091D20D08954A
:10F03A00A091CF0DB091D00DEA17FB070895E12FEB
:10F04A00A091D60DEA0FE093D60DE091D80D089560
:10F05A00F0E0E95CF74F10830895E091DD0EF0E0EF
:10F06A00E452F24FE081E0939C00E091DD0EEF5F05
:10F07A00E093DD0E0895D901F0E0AE17BF070895B9
:10F08A0000DAAC91AA3308950F01FBD9EC91E05351
:10F09A0013C9EA930E947F5E1F5F0895E4E4F8E1D2
:10F0AA00FA93EA930895FE013196FA93EA93089542
:10F0BA00E881EA930C947F5EE881F9816A817B8119
:10F0CA000E94007B0895E15CF54FE081E0300895ED
:10F0DA00EA930E941C64EA930C94175AEA930E94DA
:10F0EA00B260EAE5E0933D090895EA930E946D62F1
:10F0FA00E0300895E0E0EA930C949262EA930E9469
:10F10A00AD62E0300895E0917100E87F1E2F089506
:10F11A00E0937300E4E8F2CF0A930E948662E0303B
:10F12A000895FF27662777270E94A67B0895EE8D0C
:10F13A00AE85BF8588899989F4DF0E942E7CA9A1B2
:10F14A00BAA1882799270E94077B0E940A7B0E94FE
:10F15A00D97B08950E940A7B0E94D97B0895FA936D
:10F16A00EA93E2E1F0E0FA93EA9308950E94CF7CF1
:10F17A00EE81A0E2B6E1F0E00C94C770E2E0EA9317
:10F18A00EE85FF850E94007AFA93EA930E94A364AF
:10F19A00E3E0EA93EE85FF850895FA93EA930C94E7
:10F1AA00A364AE85BF85AE0FBF1FFD010E94007A22
:10F1BA00F4CFE6E0EA93EC85FD850E94007AEDCF74
:10F1CA00AC85BD85AE0FBF1FFD010E94007AE5CF59
:10F1DA000E94A364E5E0EA9308950E94A364E8E02C
:10F1EA00EA930C94DB6C0E94A364E9E0EA93089525
:10F1FA00EFE3F1E0D2CFEB85FC85AF81B885AE179E
:10F20A00BF0708950D851E85ED85FE85E987FA8776
:10F21A000D871E870B851C85EB85FC85EF83F88798
:10F22A000B871C8708950E94007AB7CFEA93EC8572
:10F23A00FD85F070B2CFED85FE85A985BA85AE173A
:10F24A00BF070895AD85BE85E985FA85EA1BFB0BE4
:10F25A000895AB85BC858BCCAF81B885EB85FC85E1
:10F26A00EA1BFB0B0895D9010E94497A0F01089500
:10F27A00D0010E94747AAF01E2E0EA93FA0191CFD9
:10F28A00E3E0EA93FA01AE85BF85AE0FBF1FEFEF49
:10F29A00F0E0EA23FB2381CFA21BB30BEFEFF0E0F0
:10F2AA00EA23FB237ACFE2E2EA931A930A930C94B5
:10F2BA00A364AC85BD85AE0FBF1FEFEFF0E0EA2374
:10F2CA00FB236BCFA985BA85ED85FE85EA1BFB0B6F
:10F2DA000895D0010E94747AAF01E2E0EA9308959A
:10F2EA00A0E2B6E1F0E00C94C7705A934A93EE8517
:10F2FA00FF8554CBFA93EA93EC85FD85FA93EA935A
:10F30A000E94C666E0910E04AA85BB8586CA2A9326
:10F31A00ED89FE89FA93EA93FE017596FA93EA93C8
:10F32A000C94C368EE89FF893497EE8BFF8B08959E
:10F33A00ED89FE89FA93EA93FE017596FA93EA93A8
:10F34A000C94C368AE89BF8914960E94ED7AEE8345
:10F35A00FF83D2CAE885F9856A857B85AC85BD8538
:10F36A008E859F8508950E94D36AE883F9836A830C
:10F37A007B830895E881F9816A817B810895EA8116
:10F38A00FB816C817D810895E991F991309639F07C
:10F39A0080EA9FE00197F1F7A8953197C9F7089598
:10F3AA000024AF0DB01D0895EA0FFB1F681F791FD7
:10F3BA000895EA1BFB0B680B790B0895F195E1950B
:10F3CA00F0400895F09560957095E195FF4F6F4F65
:10F3DA007F4F0895EE230E2EEA2F19F0EE0F0A94AE
:10F3EA00E9F70895EE0FFF1FEE0FFF1FEE0FFF1F45
:10F3FA00EE0FFF1F0895EF2FFF27E7FDFFEF089598
:10F40A00FE2FFF0FFF0B6F2F7F2F08956F2F660FB1
:10F41A00660B762F0895BA2FBB0FBB0B8B2F9B2F32
:10F42A0008958B2F880F880B982F0895EA17FB07EA
:10F43A00E1E00CF0EE270895FA9FF02DEB9FF00D16
:10F44A00EA9FE02DF10D08957A9F702D6B9F700D44
:10F45A00F89F700DE99F700D6A9F602D710DFB9FDB
:10F46A00600D711DE89F600D711D8827FA9FF02DB0
:10F47A00610D781FEB9FF00D611D781FEA9FE02D4B
:10F48A00F10D681F781F089582D0D6DF0EF496DF3B
:10F49A0008958BD0D9DF0EF495DF0895002498E003
:10F4AA00AA0F001C0E1A10F40E0E01C0A1609A9544
:10F4BA00B9F7EA2FA02D08950024112490E1AA0F8C
:10F4CA00BB1F001C111C0E1A1F0A18F40E0E1F1E59
:10F4DA0001C0A1609A9599F7FD01D001089557D00E
:10F4EA00EBDF0EF46BDF08953F934F935F93002495
:10F4FA0011244427552730E2AA0FBB1F881F991FE2
:10F50A00001C111C441F551F0E1A1F0A460B570BCD
:10F51A0028F40E0E1F1E461F571F01C0A1603A9500
:10F52A0059F7FD01BC01D001CA015F914F913F918A
:10F53A0008953BD0D9DF0EF445DF0895AFDFEA2FF7
:10F54A000895E894B7FF04C0A095B0951196689401
:10F55A00F7FD34DFB1DFFD010EF430DF0895C4DFBB
:10F56A00FD01BC010895E89497FF09C0A095B095E4
:10F57A0080959095AF5FBF4F8F4F9F4F689477FDEF
:10F58A0021DFB2DFFD01BC010EF41CDF0895E8940F
:10F59A00F7FF02C013DF6894B7FF06C0A095B095C5
:10F5AA00119600F8039400FA0895E89477FF02C0D0
:10F5BA0009DF689497FF0BC00024A095B095809549
:10F5CA0090951196801D901D00F8039400FA0895F5
:10F5DA00ED91FC9111970895ED91FD916D917C91BA
:10F5EA0013970895ED93FD936D937C930895059079
:10F5FA00F491E02D08957A936A93FA93EA93089521
:10F60A00689401C0E89401D09DD0182E862F612DF0
:10F61A00192E972F712D1B2EBF2FF12D1A2EAE2FBB
:10F62A00E12D0895119602D0FE2F1197E199FECF90
:10F63A00FF93FFB7F894AEBBBFBBE09AEDB3FFBF31
:10F64A00FF91089507D01196EF93EF2F03D0EF9112
:10F65A0011970895E19B02C0A895FCCF9FB7F89433
:10F66A00AEBBBFBBE09A8DB3E81719F0EDBBE29AC7
:10F67A00E19A9FBF0895552342F4503811F4E0FFF0
:10F68A0004C03196691F791F6BF050E8572711F4AF
:10F69A005F93CDC05F3F31F0660F000C57956795B9
:10F6AA00752F08955F9300200AF0CDC0C6C050E8B8
:10F6BA00192E1522880F991F9527550F879550E8FF
:10F6CA00072E0522660F771F7527550F6795089530
:10F6DA00689401C0E8945F93F2DF703818F07F3FB6
:10F6EA0008F4A5C056E1571BAAF4519558300EF4F8
:10F6FA00593030F0EFEFFFEF6FEF7FE777F91AC07D
:10F70A0077275523B9F0EE0FFF1F661F771F5A950B
:10F71A00D1F710C07727583028F0EF2FF62F672F30
:10F72A005850F9CF552331F076956795F795E795B7
:10F73A005A95D1F700200AF445DE5F91089568943E
:10F74A0001C0E894309760407040B1F0002426F080
:10F75A00772312F4009436DE172E7EE1112032F060
:10F76A007A95EE0FFF1F661F111CF9CFEF2FF62FA8
:10F77A00612D5F938ADF5F9108954F93AF01FD0179
:10F78A00DA01AB01BC01CA01402D012C142E4F91A4
:10F79A000895EA0FFB1F681F0895E095F09560959C
:10F7AA00EF5FFF4F6F4F08955F9381DF903871F1DC
:10F7BA0050E8152604C05F937ADF903839F1703823
:10F7CA0021F1572F591B13F112F4D7DFFACF583111
:10F7DA0018F0AA27BB278827583028F0AB2FB82F54
:10F7EA0088275850F9CF552329F08695B795A795BC
:10F7FA005A95D9F7502D512562F0CBDF38F4679529
:10F80A00F795E795739513F41EC0B7DF3EDF5F9156
:10F81A000895EA1BFB0B680B51F010F40094BDDF4E
:10F82A006623A2F3EE0FFF1F661F7A95CBF7EE272A
:10F83A00FF27662777275F910895EFEFFFEF6FE7BE
:10F84A007FEF5F910895EFEFFFEF6FE77FE75F913B
:10F85A0008955F932CDF703851F3903841F30124F7
:10F86A000894791F23F41CF300203AF3ECCF0F928B
:10F87A001F932F933F934F93112722279927689F0E
:10F88A00A0018F9F302D410D591F6B9F300D411DD7
:10F89A00591F8E9F27D0BF9F25D06A9F23D0BE9F16
:10F8AA001DD0AF9F1BD0AE9F110D291F391F491FB5
:10F8BA00591FE32FF42F652F522F4F913F912F910C
:10F8CA001F910F9066232AF0550FEE1FFF1F661F28
:10F8DA0002C073954BF2CFDE5F910895100D211D82
:10F8EA00391F02C0200D311D491F591F08955F930A
:10F8FA00DEDE703821F411200AF49FCFA4CF9038AD
:10F90A0009F495CF01240894970B1BF4D4F3002033
:10F91A00F3CF792F1F932F933F934F9311241127DE
:10F92A00222733274427552790E2AE17BF078607B9
:10F93A00410730F0AE1BBF0B860B410B089401C088
:10F94A008894551F221F331F111CAA1FBB1F881F13
:10F95A00441F9A9551F7F901612D4F913F912F91CB
:10F96A001F91662332F0550FEE1FFF1F661F7A950F
:10F97A0043F281DE5F9108953097604070400895A8
:10F98A0000240A160B06089500240A160B06080618
:10F99A00090608955A934A933A932A931A930A9313
:10F9AA0008955D814C813B812A81198108810895DE
:00000001FF
